:100000000C94AC540C9451550C9451550C9451557E
:100010000C9451550C9451550C9451550C945155C8
:100020000C9451550C9451550C9451550C945155B8
:100030000C9451550C949A570C9451550C9451555D
:100040000C9451550C9451550C9451550C94515598
:100050000C9451550C9451550C9451550C94515588
:100060000C9451550C9451550C9451550C94515578
:100070005A5501200201003808000000000000006D
:100080000000000000565E645E375FDB62C7626797
:100090005E765E855EAF62935EA15E5B5B525B5B8C
:1000A0005252095B52A45252A4A45252A45B52A4CD
:1000B0005B5B5B525B5B52A45B5B5B095252525BC6
:1000C0005B5B525252A4A4525B5B5252A45B5B5BDB
:1000D000525252525B5B5B52A4A4520952A4A45BDD
:1000E000525B5B52A45B5B5B525B5B52A45B5B5BF2
:1000F0005B525252525B5B5B5B0909A4A4525B5298
:1001000052A4A4A45B5B5252A45B5BA45B5B520948
:10011000525B5B5B5B525B5B5B5252525B5B52A41C
:100120005B5B5BA45252525B5B5B52A45B5B525BBA
:100130005B52A45B5B5B525209095B5B5B52A4A4FC
:100140005209525252A45B5B5B52A4A4A4525B5B63
:100150005B52A45B5B525B5B5B525B5252525B5BDC
:100160005B5B52A4A4A4525B5B5B525B5B5B525231
:100170005B5B525B5B52A4A45252525252A45B5B33
:100180005B5B525B52A45B5B5B5B525B5B525B5B9A
:100190005B52A45B5B52525252A45B000000000011
:1001A0000000000000898989898900008992929263
:1001B0009289920089929292928992008992929267
:1001C000899B9200899292899B9292008989899B4E
:1001D00092929200009B9B929292920000000000EB
:1001E00000000089898989898989899292929292ED
:1001F00092929292929292929292929292929292DF
:1002000092929292929292929292929292929292CE
:100210009292929292929292929292009292929250
:1002200092929200899292929292920089929292E4
:1002300092929200899292929292920089929292D4
:1002400092929200899292929292920089929292C4
:100250009292920089929292929292929292929219
:100260009289899292929289899B9B929292899B80
:100270009B92929292899B9292929292899B929255
:1002800092929292899B9292929292899B9292924E
:10029000929292899B929292929292000000000018
:1002A0000000000000898989898900008992929262
:1002B0009289920089929292928992008992929266
:1002C000899B9200899292899B923F008989899BA0
:1002D000923F3F00009B9B923F3F3F000000000089
:1002E00000000089898989898989899292929292EC
:1002F00092929292929292929292929292929292DE
:100300009292923F929292929292923F3F929292C6
:100310009292923F3F3F9292929292009292929248
:100320003F3F3F0089929292923F3F008992929282
:1003300092923F0089929292929292008992929226
:1003400092929200899292929292920089929292C3
:1003500092929200899292929292923F3F3F929211
:100360009289893F3F929289899B9B3F9292899B78
:100370009B92929292899B9292929292899B929254
:1003800092929292899B9292929292899B9292924D
:10039000929292899B9292929292920909090909EA
:1003A000090909092E2E2E2E2E2E2E092E1C1C1C5C
:1003B0001C1C1C092E131313131313092E1C1C1CB5
:1003C0001C1C1C092E1C1C1C1C1C1C092E1313138A
:1003D00013132E092E1C1C1C1C2E1C0909090909AB
:1003E0000909092E2E2E2E2E2E13091C1C1C2E1C24
:1003F0002E130913132E1C132E13091C2E1C131C51
:100400002E13092E1C131C1C2E13091C131313135B
:100410002E1309131C1C1C1C2E1309092E1C1C1C3A
:100420002E1C13092E13132E1C1313092E1C2E1C05
:10043000131C1C092E2E1C131C1C2E092E1C1313FE
:10044000131313092E2E2E2E2E2E2E0913131313D3
:1004500013131309090909090909091C1C1C1C1C8F
:100460002E130913131313132E13091C1C1C1C1C0D
:100470002E13091C2E2E1C1C2E13091313131313D9
:100480002E13092E2E2E2E2E2E1309131313131393
:1004900013130909090909090909090101010101E0
:1004A000010101011717171717171701170606067D
:1004B00006060601170202020202020117060606DC
:1004C00006060601170606060606060117020202C0
:1004D00002021701170606060617060101010101AF
:1004E000010101171717171717020106060617064D
:1004F000170201020217060217020106170602067A
:10050000170201170602060617020106020202027E
:100510001702010206060606170201011706060663
:100520001706020117020217060202011706170634
:100530000206060117170602060617011706020231
:1005400002020201171717171717170102020202FA
:10055000020202010101010101010106060606066F
:10056000170201020202020217020106060606062F
:1005700017020106171706061702010202020202FD
:1005800017020117171717171702010202020202BA
:1005900002020101010101010101015353535353AF
:1005A00053535353AEAEAEAEAEAEAE53AEAEAEAE32
:1005B000AEAEAE53AEAEA5AEAEA5A553AEAEA5A53E
:1005C000AEA55C53AEAEA5A55C5CA553AEAE5C5CBF
:1005D0005CA55C53AEAEA5A5A5A5A5535353535337
:1005E000535353AEAEAEAEAEAEA553AEAEAEAEAEA0
:1005F000A55C535C5CA55C5C5C5C535CA5A5AE5CD7
:10060000535C53A5A5AEAEA55C53535CAEAEA5A599
:100610005C5C53AE5C5CA5A55C5C5353AEAEAEA512
:10062000A5A5AE53AEAEA5AEAEAEA553AEAEAEA5CD
:10063000A5A5A553AEAEAEA5A5A5A553AEAEA5A5E1
:100640005C5C5C53AEA55C5C5C535353A55C5C5C2A
:1006500053535C5353535353535353AEA55C5C5C99
:10066000535353A5AEA55C5C535353A55C5CA5A541
:100670005C5C535C5CA5AEAEA55C535CA5A5A5AE69
:10068000A55C535C5C5C5C5C5CA5535C5C5C5C5C2A
:100690005C5C5353535353535353531B5C1B5C5C6D
:1006A0005C5C131B1B5C1B5C5C5C131B5C5C5C1B61
:1006B0005C5C135C5C1B5C5C5C131B1B5C5C1B5C10
:1006C0005C13135C1B5C5C5C5C131B1B5C5C5C5C08
:1006D000131B135C5C1B5C5C131B5C1B5C1B5C5C7A
:1006E0005C5C131B1B5C1B5C5C5C131B5C5C1B1B62
:1006F0005C5C135C5C1B5C5C5C131B1B5C5C1B5CD0
:100700005C13135C1B5C5C5C5C131B1B5C1B5C5C08
:10071000131B135C5C1B5C5C131B5C5C5C5C5C1300
:100720001B131B5C5C5C131B131B5C5C5C13131BBB
:100730001B5C1B5C13131B135C1B5C5C131B131BEC
:100740005C5C5C13131B1B5C1B5C5C131B131B5C52
:100750005C5C5C131B1B5C1B5C5C5C5C5C5C5C132E
:100760001B131B1B5C1B131B5C1B5C5C5C13131BB4
:100770001B5C1B5C135C1B135C1B5C5C131B131B63
:100780005C5C5C135C1B1B5C1B5C5C131B131B5CC9
:100790005C1B5C131B1B5C1B5C5C1B0101010101EE
:1007A000010101011818181810010101181010108A
:1007B00010100101011010101010011001010101B1
:1007C000010101181010011818181010101001184C
:1007D0001010101010010101101010010101010191
:1007E00001010118181818181810101810101010FE
:1007F0001010101010101010100101010101010162
:100800000101011001010118180118101001181040
:100810001001101010011010101001010101010150
:1008200001010118101810100118181010101010E4
:100830000118101010100101011010010101011028
:1008400010010101101818181010100110181010C4
:100850001010100101101010101010010101010101
:1008600001010118181010011018181010101001B3
:1008700010181010101001010110100101011010CA
:100880001001011001101818181010100110181084
:1008900010101001010110101010010101010101DF
:1008A0000101010118181818100101011810101089
:1008B00010100101011010101010011001010101B0
:1008C0000101011810100118181837101010011824
:1008D00010373710100101013737370101010101CD
:1008E00001010118181818181810101810101010FD
:1008F0001010101010101010100101010101010161
:1009000001010137010101181801183737011810CA
:1009100010011037373710101010010101010101CB
:100920003737371810181010013737101010101003
:100930000118371010100101011010010101011000
:1009400010010101101818181010100110181010C3
:10095000101010010110101010101037373701015E
:10096000010101373710100110181837101010014D
:1009700010181010101001010110100101011010C9
:100980001001011001101818181010100110181083
:1009900010101001010110101010010000000000E3
:1009A000000000007676767676767600761B1B6DF4
:1009B0006D1B1B007624246D6D1B2400766D6D6D00
:1009C0006D1B2400766D6D6D6D6D1B00766D1B6D5E
:1009D0006D6D1B00761B241B6D6D1B00000000005D
:1009E00000000076767676766D1B001B6D6D1B6DB4
:1009F000241B00246D6D1B6D241B00241B6D6D6D6D
:100A0000241B0024246D6D6D241B0024241B6D6D9C
:100A1000241B002424246D6D241B00007624242430
:100A20006D6D1B00766D6D6D6D6D1B00761B1B1B58
:100A30006D1B6D00766D6D6D1B6D1B00766D6D6DA4
:100A40006D6D6D006D242424242424001B1B1B1BAE
:100A50001B1B1B00000000000000002424241B6D51
:100A6000241B001B2424246D241B001B6D24246DD7
:100A7000241B001B6D6D246D241B006D6D6D6D6D51
:100A8000241B002424242424241B001B1B1B1B1BAD
:100A90001B1B00000000000000000001010101011B
:100AA0000101010117171717171717011701010681
:100AB00006010101170202060601020117060606D9
:100AC00006010201170606060606010117060106C1
:100AD00006060101170102010606010101010101DB
:100AE0000101011717171717060101010606010674
:100AF00002010102060601060201010201060606C4
:100B000002010102020606060201010202010606B6
:100B1000020101020202060602010101170202029D
:100B20000606010117060606060601011701010166
:100B3000060106011706060601060101170606064C
:100B4000060606010602020202020201010101017B
:100B5000010101010101010101010102020201067D
:100B6000020101010202020602010101060202065F
:100B7000020101010606020602010106060606063A
:100B8000020101020202020202010101010101014E
:100B90000101010101010101010101262626261C96
:100BA000012626262626261C01262626261C1C1360
:100BB00001261C26261C1C1301261C26261C13138A
:100BC00001261C261C131C1301261C1C13131313B3
:100BD000011C13010101010101010126262626261F
:100BE000261C0126262626261C13011C1C1C1C1C48
:100BF0001313011C1C1C1C1C1313011C1C1C1C1398
:100C00001313011C131C131C1313011313131313BD
:100C100013130101010101010101012626262626E7
:100C200026262626261C1C1C1C1C1C26261C1C1CBE
:100C30001C1C1C26261C1C1C1C1C1C26261C1C1CCC
:100C40001C131C261C1313131313131C131313133D
:100C50001313130101010101010101261C012626C4
:100C6000261C011C1301261C1C13011C1301261C2D
:100C7000131301131301261C1313011C1301261C4B
:100C80001313011313011C131313011313011C136A
:100C900013130101010101010101010B0B0B0B0AEF
:100CA0000B0B140B0B140B0B0B0B0A140B0A0A0B7C
:100CB0000B0B0B0A0B0B140B0B0B0B0B0B0B0A0B7D
:100CC0000B0B140B140B0B0B140B0A0B0B0B0B0B5A
:100CD0000A0B0B0B0A0B0A140B0B0B0A0B0B0B0A60
:100CE0000B0B140B0B140B0B0B0B0A140B0A0B0B3B
:100CF0000B0B0A0A0B0B140B0B0B0B0B0B0B0A0B3E
:100D00000B0B140B140B0B0B140B0A0B0B0B0B0B19
:100D10000A0B0B0B0A0B0B140B0B0B0B0B0A0B0A1E
:100D20000B0B140B0B140B0B0B0B0A140B0A0B0BFA
:100D30000B0B0B0A0B0B140B0B0B0B0B0B0B0A0BFC
:100D40000B0B140B140B0B0B140B0A0B0A0B0B0BDA
:100D50000A0B0B0B0A0B0B140B0B0B0B0B0B0B0ADD
:100D60000B0A140B0B140B0B0B0B0A140B0A0B0BBB
:100D70000B0B0B0A0A0B140B0B0B0B0B0B0B0A0BBD
:100D80000A0B140B140B0B0B140B0A0B0B0B0B0B9A
:100D90000A0B0B0B0A0B0B140A0B0B0000000000D4
:100DA00000000000080808080808080008111111D0
:100DB0001111110008111111121111000811121254
:100DC0001212120008111111121111000811121241
:100DD000121212000811111111111100000000006F
:100DE000000000080808080808080811111111116E
:100DF00011111111111112111111111112121212DE
:100E000012111111111112111111111112121212CC
:100E100012111111111111111111110008111212D9
:100E200012121200081112111111120008111212DF
:100E300012121200081111111211110008111212D0
:100E400012121200081111111211110008111212C0
:100E50001212120008111111111111111212121295
:100E6000121111111211111112111111121212126B
:100E7000121111111111121111111111121212125C
:100E8000121111111111121111111111121212124C
:100E90001211111111111111111111000000000096
:100EA00000000000080808080808080008111111CF
:100EB0001111110008111111121111000811121253
:100EC000121212000811111112113F000811121212
:100ED000123F3F00081111113F3F3F00000000008A
:100EE000000000080808080808080811111111116D
:100EF00011111111111112111111111112121212DD
:100F00001211113F111112111111113F3F12121242
:100F10001211113F3F3F111111111100081112124E
:100F20003F3F3F0008111211113F3F0008111212FC
:100F300012123F00081111111211110008111212A2
:100F400012121200081111111211110008111212BF
:100F500012121200081111111111113F3F3F12120C
:100F60001211113F3F1111111211113F12121212E1
:100F7000121111111111121111111111121212125B
:100F8000121111111111121111111111121212124B
:100F9000121111111111111111111108080808086D
:100FA00008080808F6F6F6F6F6F6F608F6ADADAD62
:100FB000AD5A5A08F6ADAD5A5AAD5A08F6AD5AAD0B
:100FC000AD5A5A08F6AD5AAD5AADAD08F65AAD5AFB
:100FD000AD5A0808F65A5A5AAD08AD08080808086C
:100FE000080808F6F6F6F6F6AD5A085AADADADADFE
:100FF000AD5A08AD5A5AADADAD5A085AADAD5AAD5D
:10100000AD5A08AD5AAD5AADAD5A085AAD5AAD5A9F
:10101000AD5A0808AD5A5A5AAD5A0808F65AAD5A90
:10102000AD5A0808F6AD5AAD5AADAD08F6AD5AAD99
:10103000AD5A5A08F6ADAD5A5AAD5A08F6ADADAD37
:10104000AD5A5A08F6ADADADADADAD08AD5A5A5A70
:101050005A5A5A08080808080808085AAD5AAD5ADA
:10106000AD5A08AD5AAD5AADAD5A085AADAD5AADEC
:10107000AD5A08AD5A5AADADAD5A085AADADADAD89
:10108000AD5A08ADADADADAD5A5A085A5A5A5A5A72
:101090005A080808080808080808080101010101A1
:1010A000010101011717171717171701170707076E
:1010B00007020201170707020207020117070207CA
:1010C00007020201170702070207070117020702BA
:1010D00007020201170202020702070101010101D2
:1010E0000101011717171717070201020707070762
:1010F00007020107020207070702010207070207AA
:10110000070201070207020707020102070207029E
:101110000702010207020202070201011702070289
:101120000702020117070207020707011707020754
:101130000702020117070702020702011707070744
:101140000702020117070707070707010702020244
:10115000020202010101010101010102070207026D
:101160000702010702070207070201020707020739
:101170000702010702020707070201020707070724
:101180000702010707070707020201020202020223
:10119000020101010101010101010125252525258A
:1011A0002525251C252525252525251C1C1C251C1C
:1011B0002525251C1C1C251C2525251C1C1C251C27
:1011C0002525251C1C1C251C2525251C1C1C251C17
:1011D0002525251C1C1C251C2525252525252525E3
:1011E000251C00252525251C1C13001C1C1C1C135C
:1011F0000A00001C131C13130A00001C131C1313F9
:101200000A00001C131C13130A00001C131C1313E8
:101210000A00001C131C13130A00001C1C1C251CB4
:101220002525251C1C1C251C2525251C1C1C251CB6
:101230002525251C1C1C251C2525251C1C1C251CA6
:101240002525251C1C1C13131313131C1313131314
:1012500013131300000000000000001C131C1313E4
:101260000A00001C131C13130A00001C131C131388
:101270000A00001C131C13130A00001C131C131378
:101280000A000013131C13130A0000131313131383
:101290000A00000000000000000000515B515B519B
:1012A000515B5B5B51515B5151515B515B5B5B51DE
:1012B000515B51515B5B51515B51515B5B515B5BCE
:1012C000515B5B515B5B515B5B5B51515B515B5BAA
:1012D000515B5B515B5B5B515B515B51515B5151AE
:1012E0005B515151515B515B5B5B515B5B5B5B5B8A
:1012F0005B5B5B515B5151515B51515B5B515B518E
:101300005B51515B5B515B515B5B5B5B5B5B515169
:10131000515151515B5B5B5B5B5B5B5B51515B5B59
:10132000515B5B5B5B51515B5B5B51515B5B5B5B3F
:10133000515B5B5B515B5B51515B515B5B5B515B39
:10134000515B5151515B5B5B515B5B515B5B5B5133
:101350005B5B5B515B5B51515B5B515B5B515B5B0F
:101360005151515B515B5B51515B5B5B5B5B51511D
:101370005B5B515B515B5B5B515B515B5B515B51F9
:1013800051515B5B5B515B515B5B5B5B515B515BE9
:101390005151515B51515B515B5B5149494949493D
:1013A000494949DADADADADADADADADADADADADA50
:1013B000DADADADADAEBEBEBEBEBEBDADAEBEBEBF4
:1013C000EBF4F4DADAEBEBEBF4F4F4DADAEBEBF47B
:1013D000F4F4EBDADAEBF4F4F4EBF4494949494973
:1013E000494949DADADADADADADA49DADADADADAA1
:1013F000DADA49EBEBEBEBEBEBEB49F4EBF4F4EB88
:10140000EBEB49EBF4F4EBEBEBF449F4F4EBEBEB43
:10141000F4F449F4EBEBEBF4F4F449DADAEBF4F43A
:10142000EBF4F4DADAEBF4EBF4F4EBDADAEBEBF41A
:10143000F4EBEBDADAEBF4F4EBEBEBDADAEBF4EB1C
:10144000EBEBF4DADAEBEBEBEBF4F4DADAEBEBEB15
:10145000F4F4F4DADAEBEBF4F4F4EBEBEBEBF4F4B6
:10146000F4EB49EBEBF4F4F4EBEB49EBF4F4F4EBD1
:10147000EBEB49F4F4F4EBEBEBEB49F4F4EBEBEBD3
:10148000EBEB49F4EBEBEBEBEBEB49EBEBEBEBEBE7
:10149000EBEB49EBEBEBEBEBEBEB4949494949490A
:1014A000494949DADADADADADADADADADADADADA4F
:1014B000DADADADADAEBEBEBEBEBEBDADAEBEBEBF3
:1014C000EBF4F4DADAEBEBEBF43F3FDADAEBEBF4E4
:1014D0003F3F3FDADAEBF43F3F3F3F494949494953
:1014E000494949DADADADADADADA49DADADADADAA0
:1014F000DADA49EBEBEBEBEBEBEB49F4EBF4F4EB87
:10150000EBEB49EBF4F4EBEBEBF4493FF4EBEBEBF7
:10151000F4F4493F3FEBEBF4F4F449DADAEBF43F4F
:101520003F3F3FDADAEBF4EB3F3F3FDADAEBEBF445
:10153000F43F3FDADAEBF4F4EBEBEBDADAEBF4EB73
:10154000EBEBF4DADAEBEBEBEBF4F4DADAEBEBEB14
:10155000F4F4F4DADAEBEBF4F4F4EB3F3FEBF4F40D
:10156000F4EB493FEBF4F4F4EBEB49EBF4F4F4EB7C
:10157000EBEB49F4F4F4EBEBEBEB49F4F4EBEBEBD2
:10158000EBEB49F4EBEBEBEBEBEB49EBEBEBEBEBE6
:10159000EBEB49EBEBEBEBEBEBEB49494949494909
:1015A00049494949FFFFFFFFFFFFFF49FFADADADCF
:1015B000ADADAD49FFADADADADADAD49FFADADAD7F
:1015C000ADADAD49FFADADADADADAD49FFADADAD6F
:1015D000ADADAD49AD9B9B9B9B9B9B4949494949FF
:1015E000494949FFFFFFFFFFFFAD499BADADADADE1
:1015F000AD9B499BADADADADAD9B499BADADADAD2B
:10160000AD9B499BADADADADAD9B499BADADADAD1A
:10161000AD9B499B9B9B9B9B9B9B4949FFADADAD64
:10162000ADADAD49FFADADADADADAD49FFADADAD0E
:10163000ADADAD49FFADADADADADAD49FFADADADFE
:10164000ADADAD49FFADADADADADAD49AD9B9B9B76
:101650009B9B9B49494949494949499BADADADAD22
:10166000AD9B499BADADADADAD9B499BADADADADBA
:10167000AD9B499BADADADADAD9B499BADADADADAA
:10168000AD9B499BADADADADAD9B499B9B9B9B9BE2
:101690009B9B49494949494949494901010101017E
:1016A000010101011717171717171701170606066B
:1016B00006060601170606060606060117060606B2
:1016C00006060601170606060606060117060606A2
:1016D00006060601060202020202020101010101E0
:1016E000010101171717171717060102060606064C
:1016F00006020102060606060602010206060606A4
:101700000602010206060606060201020606060693
:101710000602010202020202020201011706060687
:101720000606060117060606060606011706060641
:101730000606060117060606060606011706060631
:10174000060606011706060606060601060202023E
:101750000202020101010101010101020606060661
:101760000602010206060606060201020606060633
:101770000602010206060606060201020606060623
:101780000602010206060606060201020202020223
:101790000202010101010101010101E4E4E4E4E4C8
:1017A000E4E4E4E4E4E4DBE4DBE4DBE4E4DBE4DB26
:1017B000DBDBE4E4DBDBDBDBDBDBDBE4E4DBDBDB55
:1017C000DB92DBE4DBDB92DB92DB92DB92929292A8
:1017D0009292928989898989898989E4E4E4E4E497
:1017E000E4DB89E4DBE4DBE4DB9289DBDBDBE4DB09
:1017F000929289DBDBDBDBDBDB9289DB92DB92DB4A
:10180000929289DBDB92DB92DB92899292929292A6
:101810009292898989898989898989E4E4E4E4E45F
:10182000E4DB89E4DBE4DBE4DB9289DBDBDBE4DBC8
:10183000929289DBDB92DB92DB9289DB92DB92DB9B
:10184000929289DBDB92DB92DB9289929292929266
:101850009292898989898989898989E4E4E4E4E41F
:10186000E4E4E4E4E4E4DBE4DBE4DBE4E4DBE4DB65
:10187000DBDBE4E4DBDBDBDBDBDBDBE4E492DB9226
:10188000DB92DBE4DBDB92DB92DB92DB92929292E7
:1018900092929289898989898989891818181810DA
:1018A00018181A18101A18181818101A18101810D2
:1018B00018181A1018181A181818181818181018B4
:1018C00018181A181A1818181A181018181818189A
:1018D00010181818101A181A1818101818181810A4
:1018E00018181A18181A18181818101A1810181882
:1018F0001818181018181A1018181818181810187E
:1019000018181A181A1818101A1810181818181861
:10191000101818181018181A18181818181818105D
:1019200018181A18181A18181818101A1810181841
:101930001810181018181A10181818181818101845
:1019400010181A181A1818181A1810181818181821
:10195000101818181018181A18181818181818101D
:1019600018181A18101A1818181A101A1810181807
:101970001018181018181A181818181818181018FD
:1019800018181A1A1A1818181A18101A18181818D5
:10199000101018181018181A181818000000000055
:1019A00000000000525252525252520052494949CC
:1019B0004949490052494949494949000000000044
:1019C000000000525252524952525249494949006C
:1019D000524949494949490052494900000000001B
:1019E0000000004952525252525252005249494943
:1019F0004949490052494949494949000000000004
:101A0000000000525252524952525249494949002B
:101A10005249494949494900524949490000000091
:101A20000000004952525252525252005249494902
:101A300049494900524949494949490000000000C3
:101A400000000052525252495252524949494900EB
:101A50005249494949494900524949000000004951
:101A600000000049525252525252520052494949C2
:101A70004949490052494949494949000000000083
:101A800000000052525252495252524949494900AB
:101A9000524949494949490052494900000000005A
:101AA0000000004952525252525252005249494982
:101AB0004949490052494949494949000000000043
:101AC0000000005252525249525237494949490086
:101AD000523737494949490037373700000000007D
:101AE0000000004952525252525252005249494942
:101AF0004949490052494949494949000000000003
:101B00000000003752525249525252373749490069
:101B1000524949373737490052494900000000000F
:101B20003737374952525252523737005249494992
:101B300049493700524949494949490000000000D4
:101B400000000052525252495252524949494900EA
:101B500052494949494949005249493737370000F4
:101B600000000037375252525252523752494949B7
:101B70004949490052494949494949000000000082
:101B800000000052525252495252524949494900AA
:101B900052494949494949005249490A0A0A0A0A27
:101BA0000A0A0A0A661466666666660A140A0A0A59
:101BB0000A0A0A0A660A1D661D141D0A660A0A1D1B
:101BC00066141D0A660A1D0A1D661D0A660A1D1492
:101BD0000A1D660A660A1D141D661D0A0A0A0A0AFB
:101BE0000A0A0A666666660A66140A0A0A0A0A0A7F
:101BF000140A0A141D661D0A66140A14661D0A0AD0
:101C000066140A661D0A1D0A66140A1D0A141D0AB6
:101C100066140A0A1D141D0A66140A0A660A1D14AF
:101C2000661D0A0A660A1D661D0A1D0A660A661DE9
:101C30000A141D0A660A1D0A1D141D0A140A0A0A3E
:101C40000A0A0A0A661466666666660A140A1414A4
:101C50001414140A0A0A0A0A0A0A0A1D66141D0A3A
:101C600066140A0A1D661D0A66140A140A1D660A0D
:101C700066140A141D0A1D0A66140A0A0A0A0A0AC8
:101C8000140A0A666666661466140A141414140AA2
:101C900014140A0A0A0A0A0A0A0A0A0101010101BD
:101CA000010101011702171717171701020101019E
:101CB00001010101170106170602060117010106BD
:101CC0001702060117010601061706011701060291
:101CD000010617011701060206170601010101019D
:101CE0000101011717171701170201010101010175
:101CF000020101020617060117020102170601017F
:101D0000170201170601060117020106010206016A
:101D1000170201010602060117020101170106025E
:101D2000170601011701061706010601170117061C
:101D30000102060117010601060206010201010166
:101D400001010101170217171717170102010202FB
:101D5000020202010101010101010106170206014F
:101D600017020101061706011702010201061701F9
:101D7000170201020601060117020101010101011A
:101D800002010117171717021702010202020201CE
:101D90000202010101010101010101646464646442
:101DA000646464646464646464646464645B5B5B0E
:101DB0005B5B5B64645B5B5B5B5B5B64645B5B5B4F
:101DC0005B5B5B645B5B5B5B5B5B5B5B09090909A2
:101DD00009090909090909090909096464646464AC
:101DE00064641264646464645B12125B5B5B5B5BDF
:101DF0005B12125B5B5B5B5B5B12125B5B5B5B5B57
:101E00005B12125B5B5B5B5B5B12120909090909E0
:101E10000912120909090909090912646464646450
:101E2000646412646464645B5B12125B5B5B5B5BA7
:101E30005B12125B5B5B5B5B5B12125B5B5B5B5B16
:101E40005B12125B5B5B5B5B5B12120909090909A0
:101E50000912120909090909090912646464646410
:101E6000646464646464646464646464645B5B5B4D
:101E70005B5B5B64645B5B5B5B5B5B645B5B5B5B97
:101E80005B5B5B645B5B5B5B5B5B5B5B09090909E1
:101E90000909090909090909090909FFFFFFFFFFE4
:101EA000FFFFFFFFFFFFFFFFFFFFFF5B5B5B5B5B76
:101EB0005B5B5B8080808080808080808080808091
:101EC000808080C0C0C0C0C0C0C0C0C0C0C0C0C0D2
:101ED000C0C0C0C0C0C0C0C0C0C0C0C0C0C0C0C002
:101EE000C0C0C0C0C0C0C0C0C0C0C0C0C0C0C0C0F2
:101EF000C0C0C0C0C0C0C0C0C0C0C0C0C0C0C0C0E2
:101F0000C0C0C0FFFFFFFFFFFFFFFFFFFFFFFFFF9E
:101F1000FFFFFF5B5B5B5B5B5B5B5BFFFF5B808093
:101F2000C0C0C0FFFF5B8080C0C0C0FFFF5B80807F
:101F3000C0C0C0FFFF5B8080C0C0C0FFFF5B80806F
:101F4000C0C0C0FFFF5B8080C0C0C0FFFF5B80805F
:101F5000C0C0C0FFFF5B8080C0C0C0C0C0C0C0C0E8
:101F6000FFFF5BC0C0C0C0C0FFFF5BC0C0C0C0C03F
:101F7000FFFF5BC0C0C0C0C0FFFF5BC0C0C0C0C02F
:101F8000FFFF5BC0C0C0C0C0FFFF5BC0C0C0C0C01F
:101F9000FFFF5BC0C0C0C0C0FFFF5BFFFF008080D1
:101FA000C0C0C0FF00F60000C0C0C0FF00F6F6F6DB
:101FB00000C0C0FF00F6F6F6F600C0FF00F6F6F629
:101FC00000C0C0FF00F60000C0C0C0FFFF0080805E
:101FD000C0C0C0FFFF5B8080C0C0C00000FFFFFF2B
:101FE000FFFFFF00FFFFFFFFFFFFFFFFFFFFFFFF00
:101FF0005B5B5BFFFFFF5B5B808080FFFF5B5B8069
:10200000808080FFFF5B808080C0C0FFFF5B80809E
:10201000C0C0C0FFFF5B8080C0C0C0FFFFFFFFFFEC
:102020005B0000FFFFFFFFFF5B5B005B5B5BFFFF95
:10203000FF5B5B8080805B5BFFFF5B808080805B01
:10204000FFFF5BC0C0C0C080FFFF5BC0C0C0C0C09E
:10205000FFFF5BC0C0C0C0C0FFFF5BFFFF5B8080B5
:10206000C0C0C0FFFF5B8080C0C0C0FFFF5B80803E
:10207000C0C0C0FFFF5B5B80C0C0C0FFFFFF5B5BF9
:1020800080C0C0FFFFFFFFFFFFFFFF00FFFFFFFF5C
:10209000FFFFFF00005B5B5B5B5B5BC0C0C0C0C061
:1020A000FFFF5BC0C0C0C0C0FFFF5BC0C0C0C0C0FE
:1020B000FFFF5BC0C0C0C0FFFFFF5BC0C0C0FFFF31
:1020C000FFFF5BFFFFFFFFFFFF5B5BFFFFFFFFFF0C
:1020D0005B5B005B5B5B5B5B5B0000000000000028
:1020E00000000000000000000000000000000000F0
:1020F00000000000000000000000000000000000E0
:1021000000000000000000000000000000000000CF
:102110000000000000000000000000C0C0C0C0C0FF
:10212000C0C0C0C0C0C0C0C0C0C0C0C0C0C0C0C0AF
:10213000C0C0C0C0C0C0C0C0C0C0C0C0C0C0C0C09F
:10214000C0C0C0C0C0C0C0C0C0C0C0C0C0C0C0C08F
:10215000C0C0C0C0C0C0C0C0C0C0C0C0C0FFFFFFC2
:1021600080C0C0C0C0FFFFFF80C0C0C0C0FFFFFF75
:1021700080C0C0C0C0FFFF8080C0C0C0C0FFFF8063
:10218000C0C0C0C0C0808080C0C0C0C0C0FFFF80D1
:10219000C0C0C0C0C0C0C0C0C0C0C0C0C0C0C0C03F
:1021A000C0C0C0C0C0C0FFC0C0C0C0C0FFC0FFC072
:1021B000FFC0C0C0C0FFFFFFC0C0C0C0FFC0FFC0A5
:1021C000FFC0C0C0C0C0FFC0C0C0C0C0C0C0C0C091
:1021D000C0C0C0C0C0C0C0C0C0C0C0C0C0C0C0C0FF
:1021E000C0C0C0C0C0C0C0C0C0C0C0C0C0C0C0C0EF
:1021F000C0C0C0C0FFFFFFFFFFC0C0C0C0C0C0C0A4
:10220000C0C0C0C0C0C0C0C0C0C0C0C0C0C0C0C0CE
:10221000C0C0C0C0C0C0C0C0C0C0C0C0C0FFFFFF01
:10222000C0C0C0C0FF8080FFFFC0C0FFFF80C08073
:10223000FFFFC0FFFF80C0C0FFFFC0FFFF80C0C026
:10224000FFFFC0C0FFFF80C0FF80C0C0C0FFFFFF16
:1022500080C0C0C0C0C0C0C0C0C0C0C0C0C0FFFF40
:10226000C0C0C0C0C0FFFFFF80C0C0C0C0C0FFFF73
:1022700080C0C0C0C0C0FFFF80C0C0C0C0C0FFFFE2
:1022800080C0C0C0C0C0FFFF80C0C0C0FFFFFFFF54
:10229000FFFFC0C0C0808080808080C0FFFFFFFF44
:1022A000FF80C0FFFFC0C0C0FFFF80C0C0C0C0FF34
:1022B000FFFF80C0C0FFFFFFFF80C0C0FFFFFFFF28
:1022C00080C0C0FFFFFF8080C0C0C0FFFFFFFFFFD6
:1022D000FFFFC0C080808080808080C0FFFFFFFF44
:1022E000FFFFC0C0C08080FFFF80C0C0C0C0FFFF34
:1022F00080C0C0C0C0FFFFFFFFC0C0C0C0C0C0C022
:10230000FFFFC0FFFFC0C0C0FFFFC0C0FFFFFFFF57
:10231000FF80C0C0C080808080C0C0C0C0C0FFFF40
:10232000FF80C0C0C0FFFFFFFF80C0C0FFFF80FF75
:10233000FF80C0FFFF80C0FFFF80C0FFFFFFFFFFE7
:10234000FFFFC0C0808080FFFF8080C0C0C0C0FF92
:10235000FF80C0C0C0C0C0C08080C0FFFFFFFFFFC3
:10236000FFC0C0FFFF80808080C0C0FFFFFFFFFF75
:10237000FFC0C0C080808080FFFFC0C0C0C0C080E0
:10238000FFFFC0FFFFC0C080FFFFC0C0FFFFFFFF17
:10239000FFC0C0C08080808080C0C0C0C0FFFFFF81
:1023A000FFC0C0C0FFFF8080C0C0C0FFFF80C0C0B2
:1023B000C0C0C0FFFFFFFFFFFFC0C0FFFF808080E5
:1023C000FFFFC0FFFF80C0C0FFFFC0C0FFFFFFFFD7
:1023D000FF80C0C0C080808080C0C0FFFFFFFFFFC3
:1023E000FFFFC0FFFF808080FFFFC0C0C0C0C0FFF4
:1023F000FF80C0C0C0C0FFFF80C0C0C0C0FFFF8062
:10240000C0C0C0C0C0FFFF80C0C0C0C0C0FFFF8050
:10241000C0C0C0C0C0C0C0C0C0C0C0C0FFFFFFFFC0
:10242000C0C0C0FFFF808080FFC0C0FFFFFF80C032
:10243000FFC0C0C0FFFFFFFFC0C0C0FF8080FFFF24
:10244000FFFFC0FF80C0C0C0FFFFC0C0FFFFFFFF95
:10245000FF80C0C0C0C0C0C0C0C0C0C0FFFFFFFF81
:10246000FFC0C0FFFF808080FFFFC0FFFF80C0C0B3
:10247000FFFFC0C0FFFFFFFFFFFFC0C0C0C0C0C064
:10248000FFFFC0C0C0C0C0FFFF80C0C0FFFFFFFF94
:1024900080C0C0C0C0808080C0C0C0C0C0FFFFFF7F
:1024A00080C0C0C0FFFF80FFFF80C0FFFF80C080F2
:1024B000FFFFC0FFFF80C0C0FFFF80FFFFFFFFFFE7
:1024C000FFFF80FFFF808080FFFF80FFFF80C0C094
:1024D000FFFF80808080C0C0C08080FFFFFFFFFFC3
:1024E000FFC0C0FFFF808080FFFFC0FFFF80C0C033
:1024F000FFFFC0FFFFFFFFFFFF80C0FFFF80808066
:10250000FFFFC0FFFF80C0C0FFFFC0FFFFFFFFFF56
:10251000FF80C0C08080808080C0C0C0C0FFFFFF3F
:10252000FF80C0C0FFFF8080FFFFC0FFFF80C0C0F2
:10253000C0C0C0FFFF80C0C0C0C0C0FFFF80C0C01F
:10254000C0C0C0C0FFFF8080FFFFC0C080FFFFFF92
:10255000FF80C0C0C080808080C0C0FFFFFFFFFF41
:1025600080C0C0FFFF8080FFFF80C0FFFF80C0C031
:10257000FFFFC0FFFF80C0C0FFFFC0FFFF80C0C0E3
:10258000FFFFC0FFFF80C0FFFF80C0FFFFFFFFFF16
:1025900080C0C0C080808080C0C0C0FFFFFFFFFF40
:1025A000FFFFC0FFFF80808080C0C0FFFF80C0C0F1
:1025B000C0C0C0FFFFFFFFFFFFC0C0FFFF808080E3
:1025C000C0C0C0FFFF80C0C0C0C0C0FFFFFFFFFF92
:1025D000FFFFC0C0808080808080C0FFFFFFFFFFC2
:1025E000FFFFC0FFFF80808080C0C0FFFF80C0C0B1
:1025F000C0C0C0FFFFFFFFFFFFC0C0FFFF808080A3
:10260000C0C0C0FFFF80C0C0C0C0C0FFFF80C0C04E
:10261000C0C0C0C0C0C0C0C0C0C0C0C0C0FFFFFFFD
:10262000FFFFC0C0FFFF808080C0C0FFFF80C0C030
:10263000C0C0C0FFFF80C0FFFFFFC0FFFF80C080A1
:10264000FFFFC0C0FFFF8080FFFFC0C0C0FFFFFFD3
:10265000FF80C0C0C0C0C0C0C0C0C0FFFFC0C0C0FD
:10266000FFFFC0FFFF80C0C0FFFF80FFFF80C0C032
:10267000FFFF80FFFFFFFFFFFFFF80FFFF808080E5
:10268000FFFF80FFFF80C0C0FFFF80FFFF80C0C052
:10269000FFFF80C08080C0C0C08080C0FFFFFFFF00
:1026A000FFFFC0C0C0C0FFFF80C0C0C0C0C0FFFFF0
:1026B00080C0C0C0C0C0FFFF80C0C0C0C0C0FFFF9E
:1026C00080C0C0C0C0C0FFFF80C0C0C0FFFFFFFF10
:1026D000FFFFC0C0C08080808080C0C0C0C0FFFF3E
:1026E000FFFF80C0C0C0C0FFFF80C0C0C0C0C0FF2F
:1026F000FF80C0C0C0C0C0FFFF80C0C0C0C0C0FF5E
:10270000FF80C0FFC0C0C0FFFF80C0C0FFFFFFFF51
:1027100080C0C0C0C080808080C0C0FFFFC0C0C07B
:10272000FFFFC0FFFF80C0FFFF80C0FFFF80FFFFF3
:1027300080C0C0FFFFFFFF80C0C0C0FFFFFFFFFFE2
:10274000C0C0C0FFFF80FFFFFFC0C0FFFF80C0FF11
:10275000FFFFC0C08080C0C08080C0C0FFFFC0C07D
:10276000C0C0C0C0FFFF80C0C0C0C0C0FFFF80C0ED
:10277000C0C0C0C0FFFF80C0C0C0C0C0FFFF80C0DD
:10278000C0C0C0C0FFFF80C0C0C0C0C0FFFFFFFF0F
:10279000FFFFC0C0C08080808080C0FFFF80C0C0BD
:1027A000FFFFC0FFFFFF80FFFFFF80FFFFFFFFFF76
:1027B000FFFF80FFFFFFFFFFFFFF80FFFF80FF8025
:1027C000FFFF80FFFF80C0C0FFFF80FFFF80C0C011
:1027D000FFFF80C08080C0C0C08080FFFFC0C0C03D
:1027E000FFFFC0FFFFFF80C0FFFF80FFFFFFFF80F4
:1027F000FFFF80FFFFFFFFFFFFFF80FFFF80FFFF66
:10280000FFFF80FFFF80C0FFFFFF80FFFF80C0C091
:10281000FFFF80C08080C0C0C08080C0FFFFFFFF7E
:10282000FFC0C0FFFF808080FFFFC0FFFF80C0C0EF
:10283000FFFFC0FFFF80C0C0FFFFC0FFFF80C0C020
:10284000FFFFC0FFFF80C0C0FFFFC0C0FFFFFFFF52
:10285000FF80C0C0C080808080C0C0FFFFFFFFFF3E
:10286000FFC0C0FFFF808080FFFFC0FFFF80C0C0AF
:10287000FFFFC0FFFF80C0C0FFFFC0FFFFFFFFFFE3
:10288000FF80C0FFFF80C0C0C0C0C0FFFF80C0C0CD
:10289000C0C0C0C0C0C0C0C0C0C0C0C0FFFFFFFF3C
:1028A000FFC0C0FFFF80C0C0FFFFC0FFFF80C0C0EF
:1028B000FFFFC0FFFF80C0C0FFFFC0FFFF80FFFF22
:1028C000FFFFC0FFFF80C0FFFF80C0C0FFFFFFFF12
:1028D00080FFC0C0C0C0C0C0C0C0C0FFFFFFFFFFBE
:1028E000FFC0C0FFFF808080FFFFC0FFFF80C0C02F
:1028F000FFFFC0FFFF80C0FFFFFFC0FFFFFFFFFF24
:1029000080C0C0FFFF80FFFFFF80C0FFFF80C0FFCF
:10291000FFFF80C0C0C0C0C0C0C0C0C0FFFFFFFF7D
:1029200080C0C0FFFF8080FFFFC0C0FFFF80C0C02D
:10293000C0C0C0C0FFFFFFFFFFC0C0C0C0C08080DC
:10294000FFFFC0FFFFC0C0C0FFFFC0C0FFFFFFFF11
:10295000FF80C0C0C0C0C0C0C0C0C0FFFFFFFFFF3D
:10296000FF80C0C0C0FFFF80C0C0C0C0C0FFFF80EC
:10297000C0C0C0C0C0FFFF80C0C0C0C0C0FFFF80DB
:10298000C0C0C0C0C0FFFF80C0C0C0C0C0FFFF80CB
:10299000C0C0C0C0C0C0C0C0C0C0C0FFFF80C0C0F9
:1029A000FFFF80FFFF80C0C0FFFF80FFFF80C0C02F
:1029B000FFFF80FFFF80C0C0FFFF80FFFF80C0C01F
:1029C000FFFF80FFFF808080FFFF80C0FFFFFFFFD1
:1029D000FF80C0C0C0C0C0C0C0C0C0FFFF80C0C0BA
:1029E000FFFF80FFFF80C0C0FFFF80FFFF80C0C0EF
:1029F000FFFF80FFFFFF80FFFFFF80C0FFFFFFFFA3
:102A0000FF80C0C0C0FFFFFF80C0C0C0C0C0FF804B
:102A1000C0C0C0C0C0C0C0C0C0C0C0FFFFC0C0C038
:102A2000FFFFC0FFFF80C0C0FFFF80FFFF80FF806F
:102A3000FFFF80FFFFFFFFFFFFFF80FFFFFFFFFFA4
:102A4000FFFF80FFFFFF80FFFFFF80FFFF80C08050
:102A5000FFFF80C080C0C0C0C08080FFFF80C0C0BA
:102A6000FFFF80FFFFFF80FFFFFF80C0FFFFFFFF32
:102A7000FF80C0C0C0FFFFFF80C0C0C0FFFFFFFFDE
:102A8000FF80C0FFFFFF80FFFFFF80FFFF80C0C00F
:102A9000FFFF80C0C0C0C0C0C0C0C0C0FFFF80C0BA
:102AA000FFFF80C0FFFF80C0FFFF80C0FFFF80C02E
:102AB000FFFF80C0C0FFFFFFFF80C0C0C0C0FFFF9E
:102AC00080C0C0C0C0C0FFFF80C0C0C0C0C0FFFF8A
:102AD00080C0C0C0C0C0C08080C0C0FFFFFFFFFF7B
:102AE000FFFF80C0808080FFFFFF80C0C0C0FFFF6D
:102AF000FF80C0C0C0FFFFFF80C0C0C0FFFFFF80DD
:102B0000C0C0C0FFFFFF80C0C0C0C0FFFFFFFFFF0D
:102B1000FFFF80C0808080808080800000008282F3
:102B200082828200008207070707070082070707E3
:102B3000070707821717171717171782171717177F
:102B4000171782821F1F1F1F1F1F8200821F1F1F38
:102B50001F1F820000822727272782828200000011
:102B600000000082078282000000008207070782BF
:102B700000000082171717820000001717828200DA
:102B80000000001F820000000000001F8200000003
:102B90000000002727820000000000000000000065
:102BA000008282000000000082070700000082828D
:102BB00007070700008282171717170000821717F0
:102BC0001717170082821F1F1F1F1F00821F1F1F42
:102BD0001F1F1F82822727272727278282828200A2
:102BE000000000078207078200000007820707072E
:102BF00082000017821717171782008217171717FE
:102C0000178200821F1F1F1F1F1F82821F1F1F1F6F
:102C10001F1F828227272727272782000000000006
:102C20008282820000000082070707000000008205
:102C3000070707000000008217171700000082171F
:102C4000171717000000821F1F1F1F000000821FA0
:102C50001F1F1F000000822727272782828282826F
:102C60008282000782070707070782078207070794
:102C70000782001782171717178200821717171776
:102C8000820000821F1F1F1F820000821F1F1F82E1
:102C900000000082272727820000000000000000BB
:102CA0008282820000000082070707000000008285
:102CB000070707000000008217171700000082179F
:102CC000171782000000821F1F1F82000000821F52
:102CD0001F1F8200000082272727828282828200B3
:102CE000000000820707078200000082070707072D
:102CF0008200008217171717178200171717171768
:102D00001782001F1F1F1F1F1F82001F1F1F1F1F53
:102D10008200002727272782000000000000000013
:102D2000008282000000000082070700000000000F
:102D300082070700000000008217170000000082D1
:102D400017178200000000821F1F8200000000820F
:102D50001F1F8200000082822727828282000000DB
:102D6000000000820782000000000082078200004D
:102D70000000008217820000000000171717820071
:102D80000000001F1F1F82000000001F1F1F820085
:102D900000000027272782820000000000000000BA
:102DA0008282820000000082070707000000008284
:102DB00007070700000000821717170000000082B5
:102DC000171717000000821F821F1F000000821FBC
:102DD000821F1F000082272782272782008282828B
:102DE0008282000782070707070782078207070713
:102DF000070782178217171717828217821717176C
:102E00001782001F1F821F1F8282001F1F821F1F29
:102E1000820000272782278282000000000082278C
:102E20002782270000000082278227000000822FCF
:102E30002F822F0000822F2F2F822F00822F2F2FE3
:102E4000822F2F00823F3F3F823F3F0000823F3F63
:102E5000823F3F00000082828282822727278200F1
:102E600000000027272727820000002F2F2F2F2F59
:102E70008200002F2F2F2F2F8200002F2F2F2F2F78
:102E80008200003F3F3F3F820000003F3F3F820003
:102E9000000000828282000000000082272727278E
:102EA0002727828227272727272782822F2F2F2F26
:102EB0002F2F8200822F2F2F2F2F8200822F2F2F34
:102EC0002F822F0000823F3F3F823F000000823F61
:102ED0003F823F0000000082828282272727272727
:102EE00027278227272727272782822F2F2F2F2F39
:102EF0002F82002F2F2F2F2F2F82002F2F2F2F2F9A
:102F00008200003F3F3F3F820000003F3F8282003F
:102F100000000082820000000000000000822727DD
:102F200027278200008227272727820000822F2F51
:102F30002F2F820082822F2F2F2F8200822F2F2F60
:102F40002F822F00823F3F3F3F823F00823F3F3F23
:102F50003F823F0000828282828282272782820013
:102F600000000027278200000000002F2F2F820082
:102F70000000002F2F2F82000000002F2F2F2F8204
:102F80000000003F3F3F3F828200003F3F3F3F3F06
:102F9000820000828282828200000000000082277C
:102FA0002782270000008227278227000000822F27
:102FB0002F822F000000822F2F822F0000822F2FC0
:102FC000822F2F0000823F3F823F3F0000823F3F21
:102FD000823F3F0000828282828282272782820093
:102FE00000000027272727820000002F2F2F2F2FD8
:102FF0008200002F2F2F2F2F8200002F2F2F2F2FF7
:103000008200003F3F3F3F3F8200003F3F3F3F8203
:1030100000000082828282000000000000008227FF
:103020002782270000008227278227000000822FA6
:103030002F822F000082822F2F822F0000822F2FBD
:10304000822F2F0000823F3F823F3F0000823F3FA0
:10305000823F3F00000082828282822727272782C8
:1030600000000027272727820000002F2F2F2F8204
:103070000000002F2F2F2F828200002F2F2F2F2FA5
:103080008200003F3F3F3F3F8200003F3F3F3F3FC6
:103090008200008282828282000000000082272754
:1030A000822727000082272782272700822F2F2FA1
:1030B000822F2F00822F2F2F2F822F00822F2F2F32
:1030C0002F822F823F3F3F3F82823F823F3F3F3FE1
:1030D00082823F000082828200008227278227822C
:1030E00000000027278282820000002F2F2F82827B
:1030F0000000002F2F2F82000000002F2F2F8200B2
:103100000000003F3F8200000000003F3F820000BF
:1031100000000082820000000000000000000000AB
:10312000000000000000000000000000000000009F
:10313000000000000000000000000000000000008F
:10314000000000000000000000000000000000007F
:1031500000000000000000000000008282828282E5
:10316000008282820707070782070782070707078F
:103170008207078217171717821717821717171753
:1031800082171700821F1F1F1F821F00821F1F1F11
:103190001F821F00822727272782278282008282A0
:1031A00082828207078207070707820707820707CD
:1031B0000707821717821717171782171782171713
:1031C0001717821F1F1F821F1F82821F1F1F821F30
:1031D0001F8200272727822782820000000000002C
:1031E000008282000000000082070700000000004B
:1031F000820707000000000082171700000000820D
:1032000017171700000000821F1F1F000000008218
:103210001F1F1F0000000082272727828200000056
:10322000000000070782000000000007078200007E
:103230000000001717820000000000178200000045
:103240000000001F820000000000001F820000003C
:10325000000000278200000000000082828282823B
:1032600000000007820707078200000782070707A0
:103270000782001782171717178200821717171770
:10328000171782821F1F1F1F1F1F82821F1F1F1FD2
:103290001F1F828227272727272782008227272789
:1032A000278227008227272727822700822F2F2F78
:1032B0002F822F0000822F2F2F2F820000822F2F8E
:1032C0002F2F820000823F3F3F82820000823F3FDB
:1032D0003F82820000008282820000272727822707
:1032E00082000027272782828200002F2F2F2F8223
:1032F0008200002F2F2F2F820000002F2F2F2F82D0
:103300000000003F3F3F82000000003F3F3F82003F
:103310000000008282820000000000000082272757
:1033200027822700008227272782270000822F2F4D
:103330002F822F0000822F2F2F822F00822F2F2FDE
:10334000822F2F00823F3F3F823F3F00823F3F3F1F
:10335000823F3F00008282828282820000008227B8
:103360002727270000008227272727000000822F19
:103370002F2F2F000000822F2F2F2F0000822F2FA2
:103380002F2F820000823F3F3F3F820000823F3F5D
:103390003F3F820000008282828282820000000021
:1033A000000000820082828200000082822F2F8231
:1033B000000000822F2F2F820000002F2F2F2F823E
:1033C0000000003F3F3F82820000003F3F3F8200FD
:1033D0000000008282820000000000000082272797
:1033E00027278200008227272727820000822F2F8D
:1033F0002F2F820000822F2F2F2F8200822F2F2F1E
:103400002F822F00823F3F3F3F823F00823F3F3F5E
:103410003F823F00008282828282822727272727DD
:1034200027278227272727272727822F2F2F2F2F4E
:103430002F82002F2F2F2F2F2F82002F2F2F2F2F54
:103440008200003F3F3F3F820000003F82828200B7
:1034500000000082000000000000000F30F037C0C4
:1034600001020304050603040708090A0B0C0D0EEC
:103470000F1011120F1013141516171819191A1B03
:10348000030407081C1D051E191919191F200F1008
:1034900021122223242519191711030005003008D1
:1034A00004000400271103010500000904000400C2
:1034B0003708040104000809040104002808040076
:1034C0000400090E020004002F080401040038085B
:1034D00006000800160E0201040081000000000032
:1034E000008142810000000081422442810000816D
:1034F0004224184281818181421800244281814303
:1035000024180018428181424200000024424224D3
:103510003C0000001C2424000000000000181818C3
:10352000000080000000000000004080000000005B
:1035300000002040800000000000102040800000BB
:103540000000081020408000000004081020408087
:10355000000002040810204080000102040810202E
:10356000408000010204081020400000010204080D
:1035700010200000000102040810000000000102F9
:103580000408000000000001020400000000000028
:103590000103F0000000000000000F000000000028
:1035A0000000000101010100000000000000000116
:1035B0000103000000000000003C0000000000804B
:1035C00080C0008080808000000000780000000043
:1035D00000000006020200000000000000000202DD
:1035E000060000000000000078000000404040405D
:1035F000000000003C000000000000000004040C7B
:103600000000000000202030000000000018080822
:10361000000000000000101000008080808080808A
:1036200080804040404040404040202020202020DA
:10363000202010101010101010100808080808089A
:10364000080804040404040404040202020202023E
:1036500002020101010101010101FF00000000005F
:10366000000000FF0000000000000000FF0000005C
:103670000000000000FF0000000000000000FF004C
:1036800000000000000000FF00000000000000003B
:10369000FF0000000000000000FF1000000000001C
:1036A000001028100000000010284428100000100E
:1036B0002844824428101028448201824428284447
:1036C00082010000000081000000000000814281B2
:1036D000000000008142244281000909090909090A
:1036E0000909092E2E2E2E2E2E2E092E1C1C1C1CD6
:1036F0001C1C092E131313131313092E1C1C1C1C42
:103700001C1C092E1C1C1C1C1C1C092E131313131F
:10371000132E092E1C1C1C1C2E1C09090909090941
:1037200009092E2E2E2E2E2E13091C1C1C2E1C2E8B
:10373000130913132E1C132E13091C2E1C131C2EDD
:1037400013092E1C131C1C2E13091C131313132EE8
:103750001309131C1C1C1C2E1309092E1C1C1C2EC7
:103760001C13092E13132E1C1313092E1C2E1C13AD
:103770001C1C092E2E1C131C1C2E092E1C1313138B
:103780001313092E2E2E2E2E2E2E09131313131360
:10379000131309090909090909091C1C1C1C1C2E01
:1037A000130913131313132E13091C1C1C1C1C2E9A
:1037B00013091C2E2E1C1C2E130913131313132E66
:1037C00013092E2E2E2E2E2E13091313131313133B
:1037D00013090909090909090909FEFEFEFEFEFE91
:1037E0000000FEFEFEFE000037FFFEFEFE00161685
:1037F00037FFFEFE00166F1637FFFE0000166F162D
:103800003737001600166F163737006F00166F6FC8
:103810001637FE0000166F6F6F1600FEFEFEFEFEEE
:10382000FEFE370000FEFEFEFEFE37161600FEFE10
:10383000FEFE37166F1600FEFEFE37166F160000EE
:10384000FEFE37166F16001600FE166F6F16006F1D
:1038500000FE6F6F6F160000FEFEFE00FF00166F89
:103860006F6FFE00FF0000161616FEFE00D0D0009F
:103870000000FEFE00D0D0D0D0D0FEFEFE00D0D0A2
:10388000D0D0FEFE000700000000FEFE0007070784
:1038900000FEFEFEFE000000FEFE6F6F1600FFFF42
:1038A00000FE161600D0FF0000FE0000D0D000077A
:1038B00000FED0D0D0D0000700FED0D0D000FE0057
:1038C000FEFE000000FEFEFEFEFEFEFEFEFEFEFE12
:1038D000FEFEFEFEFEFEFEFEFEFEFEFEFEFEFE0006
:1038E0000000FEFEFEFE000737FFFEFEFE0007079B
:1038F00037FFFE000007070737FF0007000707072D
:1039000037370007000707070737FE0000070707DC
:103910000707FE00FF00070707070000FEFEFEFE88
:10392000FEFE370700FEFEFEFEFE37070700FEFE26
:10393000FEFE370707070000FEFE370707070007F0
:1039400000FE07070707000700FE0707070700003C
:10395000FEFE07070700FF00FEFEFE00D00007077F
:103960000707FE00D0D000000000FE00D0D0D0D06D
:10397000D0D0FE00D0D0D0D0D0D0FEFE00D0D0D05D
:10398000D0D0FE00070000000000FE00070707007F
:10399000FEFEFEFE000000FEFEFE0700D000FEFE62
:1039A000FEFE00D0D000FEFEFEFED0D0D000FEFE17
:1039B000FEFED0D0D000FEFEFEFED0D000FEFEFE09
:1039C000FEFE0000FEFEFEFEFEFEFEFEFEFEFEFE13
:1039D000FEFEFEFEFEFEFEFEFEFEFEFEFEFEFEFE07
:1039E0000000FEFEFEFE000037FFFEFEFE00161683
:1039F00037FFFEFE00166F163737FE0000166F6F9A
:103A00001637006F00166F6F6F16006F00166F008D
:103A10006F6FFE0000166FFF006F00FEFEFEFEFEE1
:103A2000FEFE370000FEFEFEFEFE37161600FEFE0E
:103A3000FEFE37166F1600FEFEFE166F6F160000B4
:103A4000FEFE6F6F6F16001600FE6F006F16006FA0
:103A500000FE00FF6F16000000FEFE00D00016FF03
:103A6000006FFE00D0D000166F6FFEFE00D0D000B9
:103A70000000FEFE00D0D0D0D0D0FEFEFE00D0D0A0
:103A8000D0D0FEFE000700000000FEFE0007070782
:103A900000FEFEFEFE000000FEFE00FF1600FFFF1F
:103AA00000FE6F1600D0FFFF00FE0000D0D0000720
:103AB00000FED0D0D000000700FED0D000FEFE00F7
:103AC000FEFE0000FEFEFEFEFEFEFEFEFEFEFEFE12
:103AD000FEFEFEFEFEFEFEFEFEFEFEFEFEFEFEFE06
:103AE000FEFEFEFEFEFEFEFE0000FEFEFEFE0000EE
:103AF00037FFFEFEFE00070737FFFEFE0007070741
:103B00003737FE00000707073737000700070707AA
:103B100007370007000707000707FEFEFEFEFEFE50
:103B2000FEFE00FEFEFEFEFEFEFE370000FEFEFE76
:103B3000FEFE37070700FEFEFEFE3707070700FE02
:103B4000FEFE370707070000FEFE0707070700070E
:103B500000FE07000707000700FEFE00000707FF42
:103B60000007FE00070707FF0007FE00070707071B
:103B70000707FE00000707070707FE00FF00000712
:103B80000707FE00000000000000FE006F6F00FE4F
:103B9000FEFEFEFE0000FEFEFEFE00FF0707000028
:103BA000FEFE00FF07070700FEFE070707070700E6
:103BB000FEFE070707070000FEFE07070000FF00E4
:103BC000FEFE000000000000FEFEFEFE006F6F0023
:103BD000FEFEFEFEFE0000FEFEFEFEFEFEFEFE00FF
:103BE0000000FEFEFEFE00373737FEFEFEFE00162A
:103BF0001616FEFEFE006F6F006FFEFEFE006F00E9
:103C0000FF6FFEFEFE006F00FF6FFEFEFE006F6F97
:103C10006F6FFEFEFEFE006F6F00000000FEFEFEF6
:103C2000FEFE37373700FEFEFEFE1616373700FE63
:103C3000FEFE6F6F163700FEFEFE6F6F6F1600FE02
:103C4000FEFE006F161600FEFEFE006F001600FE60
:103C5000FEFE6F6F0000FEFEFEFEFEFE0000D000C6
:103C60000000FEFE0000D0D000FFFEFEFE00D0D01F
:103C700000FFFEFEFE00D0D00007FEFEFEFE0000AC
:103C80000000FEFEFE0007070700FEFEFEFE00002D
:103C900000FEFEFEFEFEFEFEFEFE00000000FEFE3A
:103CA000FEFEFF00D000FEFEFEFEFF00D000FEFE86
:103CB000FEFE0700D000FEFEFEFE000000FEFEFE3F
:103CC000FEFEFEFEFEFEFEFEFEFEFEFEFEFEFEFE14
:103CD000FEFEFEFEFEFEFEFEFEFEFEFEFEFEFEFE04
:103CE000FEFEFEFEFEFEFE000000FEFEFEFE0037B3
:103CF0003737FEFEFEFE00161600FEFEFE006F6F5A
:103D0000006FFEFEFE006F00FF6FFEFEFE006F0004
:103D1000FF6FFEFEFE006F6F6F6FFEFEFEFEFEFE8B
:103D2000FEFE000000FEFEFEFEFE37373700FEFE00
:103D3000FEFE1616373700FEFEFE6F6F163700FECA
:103D4000FEFE6F6F6F1600FEFEFE6F6F161600FE12
:103D5000FEFE006F001600FEFEFEFEFEFEFE006F81
:103D60006F00FEFEFE00D0000000FEFEFE00D00050
:103D7000FFFFFEFEFE00D000FFFFFEFE0007000773
:103D80000700FEFEFE0000000000FEFEFEFEFEFE3E
:103D90000007FEFEFEFEFEFEFE006F6F0000FEFE50
:103DA000FEFE00000000FEFEFEFE00D0D000FEFE83
:103DB000FEFE00D0D000FEFEFEFED00000FEFEFEA5
:103DC000FEFE000700FEFEFEFEFE0700FEFEFEFEFB
:103DD000FEFE00FEFEFEFEFEFEFEFEFEFEFE0000FD
:103DE0000000FEFEFE0037373737FEFE00070707EC
:103DF0000707FEFE000707070707FE000707000783
:103E00000707FE000700FF070700FE000700FF0787
:103E10000007FE000707070700070000FEFEFEFE82
:103E2000FEFE373700FEFEFEFEFE07373700FEFEC1
:103E3000FEFE07073700FEFEFEFE07070700FEFE38
:103E4000FEFE00070700FEFEFEFE07000700FEFE66
:103E5000FEFE070000FEFEFEFEFEFEFE0007070758
:103E600000070000000000000000006F00FFFFFFDF
:103E7000FF00FE000000000000D0FEFEFEFEFE007F
:103E8000D0D0FEFEFEFEFEFE0000FEFEFEFEFEFEAA
:103E9000FEFEFEFEFEFEFEFEFEFE00D000FEFEFE6C
:103EA000FEFED0D0D000FEFEFEFED0D0D000FEFE42
:103EB000FEFED00000FEFEFEFEFE000700FEFEFE3F
:103EC000FEFE070700FEFEFEFEFE0000FEFEFEFEFA
:103ED000FEFEFEFEFEFEFEFEFEFEFEFEFEFEFEFE02
:103EE000FEFEFEFEFEFE00000000FEFEFE00373776
:103EF0003737FEFE000707070707FEFE0007070724
:103F00000707FE00070700000707FE000700FF077E
:103F10000700FE000700FF070007FEFEFEFEFEFE94
:103F2000FEFE0000FEFEFEFEFEFE373700FEFEFE39
:103F3000FEFE07373700FEFEFEFE07073700FEFED7
:103F4000FEFE07070700FEFEFEFE00070700FEFE5E
:103F5000FEFE07000700FEFEFEFEFE000707070745
:103F60000007FEFE00070707000700000000000032
:103F70000000006F00FF00FFFF00FE000000FF00D8
:103F800000D0FEFEFEFEFE00D000FEFEFEFEFEFEA7
:103F90000007FEFEFEFEFEFEFE00070000FEFEFE27
:103FA000FEFE00D000FEFEFEFEFED0D0D000FEFEE3
:103FB000FEFED0D0D000FEFEFEFE000000FEFEFEA3
:103FC000FEFE0700FEFEFEFEFEFE0700FEFEFEFEFB
:103FD000FEFE00FEFEFEFEFEFEFE000000000000F3
:103FE0000000007676767676767600761B1B6D6D11
:103FF0001B1B007624246D6D1B2400766D6D6D6D8A
:104000001B2400766D6D6D6D6D1B00766D1B6D6DE7
:104010006D1B00761B241B6D6D1B00000000000053
:10402000000076767676766D1B001B6D6D1B6D2419
:104030001B00246D6D1B6D241B00241B6D6D6D24F6
:104040001B0024246D6D6D241B0024241B6D6D2426
:104050001B002424246D6D241B0000762424246D71
:104060006D1B00766D6D6D6D6D1B00761B1B1B6DE2
:104070001B6D00766D6D6D1B6D1B00766D6D6D6D2E
:104080006D6D006D242424242424001B1B1B1B1B8A
:104090001B1B00000000000000002424241B6D24D2
:1040A0001B001B2424246D241B001B6D24246D2461
:1040B0001B001B6D6D246D241B006D6D6D6D6D24DB
:1040C0001B002424242424241B001B1B1B1B1B1B40
:1040D0001B000000000000000000FEFEFEFE0000CD
:1040E0000000FEFE00001C2E2E2EFE001C2E1C2E9C
:1040F0002E2EFE001C2E001C1C1CFE001C2E2E0052
:104100000000001F001C2E2E1C2E006F00001C1C27
:104110002E2EFE00001F00001C1C000000FEFEFEF4
:10412000FEFE2E2E1C0000FEFEFE2E2E1C2E1C005F
:10413000FEFE1C1C002E1C00FEFE00002E1C1C009F
:10414000FEFE2E1C2E1C001F00FE2E2E1C00006FDB
:1041500000FE1C1C001F0000FEFEFE006400001F8D
:104160001F00FEFE007676000000FEFE00647676FC
:104170007676FEFEFE0064646464FEFE0098000035
:104180000000FEFE0098989800FEFEFEFE00000073
:10419000FEFEFEFEFEFEFEFEFEFE760000006476E3
:1041A00000FE64007676000000FE00767664006F04
:1041B00000FE64646400FE0001FE000000FEFEFEDE
:1041C000FEFEFEFEFEFEFEFEFEFEFEFEFEFEFEFE0F
:1041D000FEFEFEFEFEFEFEFEFEFEFEFEFEFE0000FB
:1041E0000000FEFE00001C2E2E2EFE001C2E1C2E9B
:1041F0002E2EFE001C2E001C1C1C00001C2E2E004F
:104200000000001F001C2E2E1C2EFE0000001C1C97
:104210002E2EFE006F0000001C1C000000FEFEFEA3
:10422000FEFE2E2E1C0000FEFEFE2E2E1C2E1C005E
:10423000FEFE1C1C002E1C00FEFE00002E1C1C009E
:1042400000FE2E1C2E1C001F00FE2E2E1C00000047
:10425000FEFE1C1C00006F00FEFEFEFE0064000E51
:104260000000FEFE006476000000FEFE006476762C
:104270007600FEFE006464767676FEFEFE006464E0
:104280006464FEFE009800000000FEFE009898980E
:1042900000FEFEFEFE000000FEFE0000006400FEC8
:1042A000FEFE7600766400FEFEFE6400766400FE8C
:1042B000FEFE0076646400FEFEFE64646400FEFEA2
:1042C000FEFE000000FEFEFEFEFEFEFEFEFEFEFE08
:1042D000FEFEFEFEFEFEFEFEFEFEFEFEFE000000F8
:1042E0000000FEFE001C001C2E2EFE001C1C2E00DA
:1042F0000000FE001C1C2E1C2E2EFE00001C1C2E7E
:104300002E2E006F000000000000006F001F6F00E5
:104310006F6FFE00001F6FFF006F00000000FEFEC9
:10432000FEFE1C002E1C00FEFEFE002E2E1C1C009D
:10433000FEFE2E1C2E1C1C00FEFE2E1C1C1C000053
:10434000FEFE00000000001F00FE6F006F1F006FE8
:1043500000FE00FF1F1F0000FEFEFE002E001FFFDC
:10436000006FFE007676001F1F1FFEFE00767600AF
:104370000000FEFE006476767664FEFEFE00646455
:104380006464FEFE009800000000FEFE009898980D
:1043900000FEFEFEFE000000FEFE00FF1F001C1CD3
:1043A00000FE1F1F0064006400FE00007664000031
:1043B00000FE76766400006F00FE646400FEFE007E
:1043C000FEFE0000FEFEFEFEFEFEFEFEFEFEFEFE09
:1043D000FEFEFEFEFEFEFEFEFEFEFEFEFEFEFEFEFD
:1043E000FEFEFEFEFE0000000000FEFE001C2E0091
:1043F0001C2EFE001C1C2E2E0000FE001C1C2E1C61
:104400002E2EFE00001C1C1C2E2E000E0000000094
:104410000000001F000E1F001F1FFEFEFEFEFEFE1E
:10442000FEFE00000000FEFEFEFE2E1C001C00FE34
:10443000FEFE00002E1C1C00FEFE2E1C2E1C1C006E
:10444000FEFE2E2E1C1C0000FEFE00000000001FC1
:1044500000FE1F001F0E001F00FEFE00000E1FFFCB
:10446000001FFE000E1F1FFF001FFE000E1F1F1F5C
:104470001F1FFE00000E1F1F1F1FFE006F00000EFB
:104480000E0EFE006F0000000000FE006F6F00FEC9
:10449000FEFEFEFE0000FEFEFEFE00FF1F0E000000
:1044A000FEFE00FF1F1F0E00FEFE1F1F1F1F0E003F
:1044B000FEFE1F1F0E0E0000FEFE0E0E00006F001F
:1044C000FEFE000000006F00FEFEFEFE006F6F00AB
:1044D000FEFEFEFEFE0000FEFEFEFEFEFEFEFE00F6
:1044E0000000FEFEFEFE001C2E2EFEFEFE001C2E18
:1044F0002E1CFEFEFE001C1C1C00FEFEFE0000002A
:104500000000FEFEFE006F00FF6FFEFEFE006F6FFC
:104510006F6FFEFEFEFE006F6F0000000000FEFEEB
:10452000FEFE1C001C1C00FEFEFE2E2E2E001C009B
:10453000FEFE1C1C00001C00FEFE00000000001C13
:1045400000FE6F00001F002E00FE6F6F001F002E88
:1045500000FE6F1F0000001C00FEFEFE0000760043
:104560000000FEFE00007676006FFEFEFE00647620
:10457000006FFEFEFE006464006FFEFEFE000000A1
:104580000000FEFEFE0098989800FEFEFEFE000071
:1045900000FEFEFEFEFEFEFEFEFE00000000FE002F
:1045A00000FE6F007600FEFEFEFE6F007600FEFE4F
:1045B000FEFE6F006400FEFEFEFE000000FEFEFE3A
:1045C000FEFEFEFEFEFEFEFEFEFEFEFEFEFEFEFE0B
:1045D000FEFEFEFEFEFEFEFEFEFEFEFEFEFEFEFEFB
:1045E000FEFEFEFEFEFEFE000000FEFEFEFE001CC5
:1045F0002E2EFEFEFE001C2E2E1CFEFEFE001C1C9F
:104600001C00FEFEFE0000000000FEFEFE006F002B
:10461000FF6FFEFEFE006F6F6F6FFEFEFEFEFEFE82
:10462000FEFE00000000FEFEFEFE1C001C1C00FE44
:10463000FEFE2E2E2E001C00FEFE1C1C00001C0088
:10464000FEFE00000000002E00FE6F00001F0000B4
:104650002E006F6F001F00001C00FEFEFEFE006FAC
:104660006F00FEFEFE0076000000FEFEFE007600FB
:104670006F6FFEFEFE0064006F6FFEFE006F006F46
:104680006F00FEFEFE0000000000FEFEFEFEFEFECD
:104690000098FEFEFEFEFEFEFE006F1F0000FEFE06
:1046A00000FE00000000FEFEFEFE00767600FEFE2C
:1046B000FEFE00766400FEFEFEFE64000000FEFECC
:1046C000FEFE006F00FEFEFEFEFE9800FEFEFEFEF9
:1046D000FEFE00FEFEFEFEFEFEFEFEFE00000000F0
:1046E0000000FE001C2E2E1C001C001C2E2E1C2E5A
:1046F0002E2E001C1C1C001C1C00000000000000D2
:104700000000001F00FF1F1F0000001F00FF1F0010
:104710001F1F001F1F1F1F001F0E00FEFEFEFEFEBC
:10472000FEFE1C00FEFEFEFEFEFE001C00FEFEFE67
:10473000FEFE001C00FEFEFEFEFE00001C00FEFE53
:10474000FEFE0E002E00FEFEFEFE00002E00FEFE0F
:10475000FEFE00001C00FEFEFEFEFE001F1F1F1FCF
:10476000000E0000000000000000006F6F6F6F6F10
:104770006F00FE00000000000076FEFEFEFEFE0060
:104780006464FEFEFEFEFEFE0000FEFEFEFEFEFE79
:10479000FEFEFEFEFEFEFEFEFEFE0000000000FE2F
:1047A000FEFE00006400FEFEFEFE76646400FEFE77
:1047B000FEFE640000FEFEFEFEFE009800FEFEFE11
:1047C000FEFE989800FEFEFEFEFE0000FEFEFEFECF
:1047D000FEFEFEFEFEFEFEFEFEFEFEFEFEFEFEFEF9
:1047E000FEFEFEFE000000000000FE001C2E2E1C3F
:1047F000001C002E2E2E1C2E2E2E001C1C1C001CFD
:104800001C000000000000000000001F00FF1F1F30
:104810000000001F00FF1F001F1FFEFEFEFEFEFE29
:10482000FEFE00FEFEFEFEFEFEFE1C00FEFEFEFE86
:10483000FEFE001C00FEFEFEFEFE001C00FEFEFE54
:10484000FEFE00001C00FEFEFEFE0E001C00FEFE32
:10485000FEFE0E002E00FEFEFEFEFE001F1F1F1FAE
:10486000001FFE001F1F1F1F000E000000000000A1
:10487000000000006F6F6F6F6F00FE00000000000F
:104880000076FEFEFEFEFE000098FEFEFEFEFEFE30
:104890009898FEFEFEFEFEFE00000E00001C00FECC
:1048A000FEFE0000000000FEFEFE00006400FEFEB2
:1048B000FEFE76766400FEFEFEFE640000FEFEFE56
:1048C000FEFE00FEFEFEFEFEFEFE00FEFEFEFEFE04
:1048D000FEFEFEFEFEFEFEFEFEFE080808080808BC
:1048E000080808F6F6F6F6F6F6F608F6ADADADAD44
:1048F0005A5A08F6ADAD5A5AAD5A08F6AD5AADAD92
:104900005A5A08F6AD5AAD5AADAD08F65AAD5AAD81
:104910005A0808F65A5A5AAD08AD08080808080897
:104920000808F6F6F6F6F6AD5A085AADADADADADDF
:104930005A08AD5A5AADADAD5A085AADAD5AADADE3
:104940005A08AD5AAD5AADAD5A085AAD5AAD5AAD26
:104950005A0808AD5A5A5AAD5A0808F65AAD5AAD17
:104960005A0808F6AD5AAD5AADAD08F6AD5AADAD20
:104970005A5A08F6ADAD5A5AAD5A08F6ADADADADBE
:104980005A5A08F6ADADADADADAD08AD5A5A5A5A4A
:104990005A5A08080808080808085AAD5AAD5AAD0E
:1049A0005A08AD5AAD5AADAD5A085AADAD5AADAD73
:1049B0005A08AD5A5AADADAD5A085AADADADADAD10
:1049C0005A08ADADADADAD5A5A085A5A5A5A5A5A4C
:1049D00008080808080808080808FEFEFEFEFEFE93
:1049E0000000FEFEFEFE00008080FEFEFE008080D5
:1049F00080FFFEFE008080808080FE00008080803E
:104A00008080001E000080808080006F00FF00809A
:104A10008080FE000000FF00000000FEFEFEFEFEA3
:104A2000FEFE800000FEFEFEFEFE80808000FEFE98
:104A3000FEFE8080808000FEFEFE80808080000080
:104A4000FEFE80808000001E00FE808000FF006F60
:104A500000FE0000FF000000FEFEFE00FF0000FF61
:104A6000FFFFFE00FF2200000000FEFE00222200E9
:104A70000000FEFE002222222222FEFEFE00222252
:104A80002222FEFE000700000000FEFE00070707CE
:104A900000FEFEFEFE000000FEFEFFFF0000FFFF26
:104AA00000FE00000022FF0000FE00002222006F36
:104AB00000FE22222222006F00FE22222200FE009F
:104AC000FEFE000000FEFEFEFEFEFEFEFEFEFEFE00
:104AD000FEFEFEFEFEFEFEFEFEFEFEFEFEFEFE00F4
:104AE0000000FEFEFE00008080FFFEFE0080808051
:104AF000808000000080808080800007000080802F
:104B00008080000700FF00808080FE000000FF0022
:104B10000000FE00FF0000FFFFFF0000FEFEFEFEA3
:104B2000FEFE80800000FEFEFEFE8080808000FE93
:104B3000FEFE80808080000000FE808080000007F4
:104B400000FE808000FF000700FE0000FF00000064
:104B5000FEFEFFFF0000FF00FEFEFEFEFE00220044
:104B60000000FEFEFE0022220000FEFEFE002222C9
:104B70002222FEFEFE0022222222FEFEFEFE002255
:104B80002222FEFEFE0007000000FEFEFE000707D8
:104B90000700FEFEFEFE000000FE000000002200F6
:104BA000FEFE000000222200FEFE2222222222001F
:104BB000FEFE222222222200FEFE2222222200FECD
:104BC000FEFE00000000FEFEFEFEFEFEFEFEFEFEFD
:104BD000FEFEFEFEFEFEFEFEFEFEFEFEFEFEFEFEF5
:104BE0000000FEFEFEFE000080FFFEFEFE00808054
:104BF0008080FEFE000080808080FE0000FF0000BC
:104C00000000001E0000FFFFFFFF006F001E0000FD
:104C10000000FE00001E6FFF006F00FEFEFEFEFEA5
:104C2000FEFE800000FEFEFEFEFE80808000FEFE96
:104C3000FEFE8080800000FEFEFE000000FF0000FF
:104C4000FEFEFFFFFF00001E00FE0000001E006FC2
:104C500000FE00FF6F1E0000FFFEFE00FF006FFF62
:104C6000006FFE00FF22006F6F6FFEFE0022220029
:104C70000000FEFE0022222222FFFEFEFE00222273
:104C800022FFFEFE000700000000FEFE00070707EF
:104C900000FEFEFEFE000000FEFE00FF6F00FFFFB4
:104CA00000FE6F6F0022FF0000FE00002222006F56
:104CB00000FE22222222006F00FE22222200FE009D
:104CC000FEFE000000FEFEFEFEFEFEFEFEFEFEFEFE
:104CD000FEFEFEFEFEFEFEFEFEFEFEFEFEFEFEFEF4
:104CE000FEFEFEFEFEFEFEFE0000FEFEFEFE0000DC
:104CF00080FFFEFEFE0080808080FEFE000080803F
:104D00008080FE0000FF0000000000070000FFFFA1
:104D1000FFFF0007000700000000FEFEFEFEFEFE93
:104D2000FEFE00FEFEFEFEFEFEFE800000FEFEFE1B
:104D3000FEFE80808000FEFEFEFE8080800000FE81
:104D4000FEFE000000FF0000FEFEFFFFFF00000768
:104D500000FE00000007000700FEFE00000707FF3E
:104D60000007FE00070707FF0007FE00071E0707F2
:104D70000707FE00000707070707FE00FF00000700
:104D80000707FE00000000000000FE006F6F00FE3D
:104D9000FEFEFEFE0000FEFEFEFE00FF0707000016
:104DA000FEFE00FF07070700FEFE0707071E0700BD
:104DB000FEFE070707070000FEFE07070000FF00D2
:104DC000FEFE000000000000FEFEFEFE006F6F0011
:104DD000FEFEFEFEFE0000FEFEFEFEFEFEFEFE00ED
:104DE0000000FEFEFEFE008080FFFEFEFE008080D2
:104DF0008080FEFEFE00FF808080FEFEFE0000FF41
:104E0000FFFFFEFEFE006F000000FEFEFE006F00D2
:104E1000FF00FEFEFEFE006F6F00000000FEFEFEC3
:104E2000FEFE80808000FEFEFEFE8080808000FE10
:104E3000FEFE808080FF00FEFEFEFFFFFF0000FE02
:104E4000FEFE0000006F00FEFEFE1E6F006F00FE03
:104E5000FEFE6F6F0000FEFEFEFEFEFE0000FF0085
:104E60000000FEFE0000FF2200FFFEFEFE002222E8
:104E70000000FEFEFE002222006FFEFEFE0000008B
:104E80000000FEFEFE0007070700FEFEFEFE00001B
:104E900000FEFEFEFEFEFEFEFEFE00000000FEFE28
:104EA000FEFEFF002200FEFEFEFE00002200FEFECF
:104EB000FEFE6F002200FEFEFEFE000000FEFEFE73
:104EC000FEFEFEFEFEFEFEFEFEFEFEFEFEFEFEFE02
:104ED000FEFEFEFEFEFEFEFEFEFEFEFEFEFEFEFEF2
:104EE000FEFEFEFEFEFEFE000000FEFEFEFE008058
:104EF00080FFFEFEFE0080808080FEFEFE00FF80C0
:104F00008080FEFEFE0000FFFFFFFEFEFE006F0041
:104F10000000FEFEFE006F00FF00FEFEFEFEFEFE35
:104F2000FEFE000000FEFEFEFEFE80808000FEFE13
:104F3000FEFE8080808000FEFEFE808080FF00FEFE
:104F4000FEFEFFFFFF0000FEFEFE0000006F00FE01
:104F5000FEFE1E6F006F00FEFEFEFEFEFEFE006FF8
:104F60006F00FEFEFE00FF000000FEFEFE00FF00E0
:104F7000FFFFFEFEFE00220000FFFEFE0007006FA6
:104F80006F00FEFEFE0000000000FEFEFEFEFEFEC4
:104F90000007FEFEFEFEFEFEFE006F6F0000FEFE3E
:104FA000FEFE00000000FEFEFEFE00222200FEFECD
:104FB000FEFE00222200FEFEFEFE22000000FEFE9B
:104FC000FEFE000700FEFEFEFEFE0700FEFEFEFEE9
:104FD000FEFE00FEFEFEFEFEFEFEFEFEFEFE0000EB
:104FE0000000FEFEFE008080FF80FEFE00808080CC
:104FF0008080FEFE00FF80808080FE000700FFFFB3
:10500000FFFFFE00070000000000FE000700FF0792
:105010000007FE000707070700070000FEFEFEFE70
:10502000FEFE808000FEFEFEFEFE80808000FEFE12
:10503000FEFE8080FF00FEFEFEFEFFFF0000FEFE83
:10504000FEFE00000700FEFEFEFE07000700FEFE5B
:10505000FEFE070000FEFEFEFEFEFEFE0007070746
:1050600000070000000000000000006F00FFFFFFCD
:10507000FF00FE00000000000022FEFEFEFEFE001B
:105080002222FEFEFEFEFEFE0000FEFEFEFEFEFEF4
:10509000FEFEFEFEFEFEFEFEFEFE000700FEFEFE23
:1050A000FEFE00222200FEFEFEFE22222200FEFE66
:1050B000FEFE22220000FEFEFEFE22000700FEFE93
:1050C000FEFE00070700FEFEFEFEFE0000FEFEFEE6
:1050D000FEFEFEFEFEFEFEFEFEFEFEFEFEFEFEFEF0
:1050E000FEFEFEFEFEFE00000000FEFEFE008080D2
:1050F000FF80FEFE008080808080FEFE00FF8080BA
:105100008080FE000700FFFFFFFFFE000700000099
:105110000000FE000700FF070007FEFEFEFEFEFE89
:10512000FEFE0000FEFEFEFEFEFE808000FEFEFE95
:10513000FEFE80808000FEFEFEFE8080FF00FEFE00
:10514000FEFEFFFF0000FEFEFEFE00000700FEFE6A
:10515000FEFE07000700FEFEFEFEFE000707070733
:105160000007FEFE00070707000700000000000020
:105170000000006F00FFFFFFFF00FE0000000000C6
:105180000022FEFEFEFEFE002222FEFEFEFEFEFECF
:105190000000FEFEFEFEFEFEFEFE070000FEFEFE1E
:1051A000FEFE002200FEFEFEFEFE22222200FEFE89
:1051B000FEFE22222200FEFEFEFE220000FEFEFE79
:1051C000FEFE000700FEFEFEFEFE070700FEFEFEDE
:1051D000FEFE0000FEFEFEFEFEFE49494949494929
:1051E000494949FFFFFFFFFFFFFF49FFADADADADEF
:1051F000ADAD49FFADADADADADAD49FFADADADAD03
:10520000ADAD49FFADADADADADAD49FFADADADADF2
:10521000ADAD49AD9B9B9B9B9B9B494949494949E6
:105220004949FFFFFFFFFFFFAD499BADADADADAD00
:105230009B499BADADADADAD9B499BADADADADADAE
:105240009B499BADADADADAD9B499BADADADADAD9E
:105250009B499B9B9B9B9B9B9B4949FFADADADADE8
:10526000ADAD49FFADADADADADAD49FFADADADAD92
:10527000ADAD49FFADADADADADAD49FFADADADAD82
:10528000ADAD49FFADADADADADAD49AD9B9B9B9B0C
:105290009B9B49494949494949499BADADADADAD94
:1052A0009B499BADADADADAD9B499BADADADADAD3E
:1052B0009B499BADADADADAD9B499BADADADADAD2E
:1052C0009B499BADADADADAD9B499B9B9B9B9B9B78
:1052D0009B494949494949494949FEFEFEFEFEFEAE
:1052E0000000FEFEFEFE0000E8E8FEFEFE00D8E83C
:1052F000F8F8FEFE00D8E8F8F8F8FE00D8E8E8F87C
:10530000F8F8FE00D8E8E8E8F8F8FE00D8D8E8E8B1
:10531000E8E8FE0000D8D8E8E8E800FEFEFEFEFE61
:10532000FEFEE80000FEFEFEFEFEF8E8D800FEFEEF
:10533000FEFEF8F8E8D800FEFEFEF8F8E8E8D8002F
:10534000FEFEF8E8E8E8D800FEFEE8E8E8D8D80075
:10535000FEFEE8E8D8D80000FEFEFE00FF00D8D828
:10536000D8D8FE00FFD800D8D8D8FEFE00D8D80084
:105370000000FEFE00D8E8D8D8D8FEFEFE00D8E82F
:10538000E8E8FEFE000F00000000FEFE000F0F0F19
:1053900000FEFEFEFE000000FEFED8D8D800FF0092
:1053A000FEFED8D800D8FF0000FE0000D8D8000FBD
:1053B00000FED8D8E8D8000F00FEE8E8D800FE00CC
:1053C000FEFE000000FEFEFEFEFEFEFEFEFEFEFEF7
:1053D000FEFEFEFEFEFEFEFEFEFEFEFEFEFEFE00EB
:1053E0000000FEFEFE0000E8E8E8FEFE0000D8E84F
:1053F000F8F8FEFE00D8E8F8F8F8FE00D8E8E8F87B
:10540000F8F8FE00D8D8E8E8F8F8FE0000D8D8E8A8
:10541000E8E8FE00FF00D8D8D8D80000FEFEFEFE67
:10542000FEFEE8E80000FEFEFEFEF8E8D80000FE02
:10543000FEFEF8F8E8D800FEFEFEF8F8E8E8D8002E
:10544000FEFEF8E8E8D8D800FEFEE8E8D8D800006C
:10545000FEFED8D8D800FF00FEFEFEFE00D800D821
:10546000D8D8FEFE00D8D8000000FEFE00D8E8D84C
:10547000D8D8FEFE00D8E8E8F8F8FEFEFE00D8E82E
:10548000E8E8FEFE000F00000000FEFE000F0F0F18
:1054900000FEFEFEFE000000FEFED8D800D800FE92
:1054A000FEFE0000D8D800FEFEFED8D8E8D800FEE8
:1054B000FEFEF8E8E8D800FEFEFEE8E8D800FEFEB2
:1054C000FEFE000000FEFEFEFEFEFEFEFEFEFEFEF6
:1054D000FEFEFEFEFEFEFEFEFEFEFEFEFEFEFEFEEC
:1054E0000000FEFEFEFE0000E8E8FEFEFE00D8E83A
:1054F000F8F8FEFE00D8E8F8F8F8FE00D8D800006A
:105500000000FE00D800FFFFFFFFFE0000FFFF00CD
:105510000000FE0000FF00FF006F00FEFEFEFEFE2A
:10552000FEFEE80000FEFEFEFEFEF8E8D800FEFEED
:10553000FEFEF8F8E8D800FEFEFE000000E8D80005
:10554000FEFEFFFFFF00E800FEFE0000FFFF000080
:10555000FEFE00FF00FF0000FEFEFE0000FFFF0059
:105560000000FE00FF00FFFFFFFFFEFE00D800006E
:105570000000FEFE00E8D8D8D8FFFEFEFE00E8F8E6
:10558000E8FFFEFE000F00000000FEFE000F0F0F00
:1055900000FEFEFEFE000000FEFE0000FFFF00FF1A
:1055A00000FEFFFFFF00FF0000FE000000D8000F1C
:1055B00000FED8D8D8E8000F00FEE8F8E800FE00AA
:1055C000FEFE000000FEFEFEFEFEFEFEFEFEFEFEF5
:1055D000FEFEFEFEFEFEFEFEFEFEFEFEFEFEFEFEEB
:1055E0000000FEFEFEFE0000E8E8FEFEFE00D8E839
:1055F000F8F8FEFE00D8E8F8F8F8FE00D8D8000069
:105600000000FE00D800FFFFFFFFFE0000FFFF00CC
:105610000000FE0000FF00FF000F00FEFEFEFEFE89
:10562000FEFEE80000FEFEFEFEFEF8E8D800FEFEEC
:10563000FEFEF8F8E8D800FEFEFE000000D8D80014
:10564000FEFEFFFFFF00D800FEFE0000FFFF00008F
:10565000FEFE00FF00FF0000FEFEFE0000FF00FF58
:10566000000FFEFE00FFFF000000FE00D800FFFF5D
:10567000FFFFFE0000D800000000FE00FF0000D881
:10568000D8D8FE00000000000000FE000F0F00FE52
:10569000FEFEFEFE0000FEFEFEFE00FF00FF00001C
:1056A000FEFE0000FFFF00FEFEFEFFFFFF00D80031
:1056B000FEFE000000D80000FEFED8D80000FF006B
:1056C000FEFE000000000000FEFEFEFE000F0F00C8
:1056D000FEFEFEFEFE0000FEFEFEFEFEFEFEFE00E4
:1056E0000000FEFEFEFE00E8E8E8FEFEFEFE000012
:1056F0000000FEFEFE00FFFFFFFFFEFEFE000000BA
:1057000000FFFEFEFE006F00FF00FEFEFE00000038
:1057100000FFFEFEFEFE00FFFF00000000FEFEFE9A
:10572000FEFEE8D8D800FEFEFEFEE8E8D8D800FE6F
:10573000FEFE00E8E8D800FEFEFEFF00E8D800FE0E
:10574000FEFEFF00E8D800FEFEFE00D8D8D800FE1E
:10575000FEFED8D8D800FEFEFEFEFEFE0000FF00D2
:105760000000FEFE0000FFE800FFFEFEFE00E8E88D
:1057700000FFFEFEFE00E8E8000FFEFEFE00000057
:105780000000FEFEFE000F0F0F00FEFEFEFE0000FA
:1057900000FEFEFEFEFEFEFEFEFE00000000FEFE1F
:1057A000FEFEFF00D800FEFEFEFEFF00D800FEFE5B
:1057B000FEFE0F00E800FEFEFEFE000000FEFEFE04
:1057C000FEFEFEFEFEFEFEFEFEFEFEFEFEFEFEFEF9
:1057D000FEFEFEFEFEFEFEFEFEFEFEFEFEFEFEFEE9
:1057E000FEFEFEFEFEFEFE000000FEFEFEFE00E8E7
:1057F000E8E8FEFEFEFE00000000FEFEFE00FFFFE9
:10580000FFFFFEFEFE00000000FFFEFEFE006F0038
:10581000FF00FEFEFE00000000FFFEFEFEFEFEFE9C
:10582000FEFE000000FEFEFEFEFEE8D8D800FEFEF2
:10583000FEFEE8E8D8D800FEFEFE00E8E8D800FE4C
:10584000FEFEFF00E8D800FEFEFEFF00E8D800FEE6
:10585000FEFE00D8E8D800FEFEFEFEFEFEFE00FFC3
:10586000FF00FEFEFE00FF000000FEFEFE00FF0047
:10587000FFFFFEFEFE00E800FFFFFEFE000F000F30
:105880000F00FEFEFE0000000000FEFEFEFEFEFE1B
:10589000000FFEFEFEFEFEFEFE00D8E8D800FEFE73
:1058A000FEFE00000000FEFEFEFE00E8D800FEFE48
:1058B000FEFE00E8D800FEFEFEFEE8000000FEFE50
:1058C000FEFE000F00FEFEFEFEFE0F00FEFEFEFED0
:1058D000FEFE00FEFEFEFEFEFEFEFEFEFEFE0000E2
:1058E0000000FEFEFE00E8E8E8E8FEFEFE00000024
:1058F00000E8FEFE00FFFFFFFF00FEFE00000000CC
:10590000FFFFFEFE000F00FF00FFFEFE0000000094
:10591000FF00FEFE00FFFFFF00D80000FEFEFEFEBF
:10592000FEFED8D800FEFEFEFEFEE8D8D800FEFE41
:10593000FEFEE8E8D800FEFEFEFE00E8D800FEFE0F
:10594000FEFE00E8D800FEFEFEFED8E8D800FEFE0F
:10595000FEFED8D80000FEFEFEFE000000000000A3
:105960000000000F0FFFFFFFFF00FE00000000001F
:1059700000E8FEFEFEFEFE00E8E8FEFEFEFEFEFE85
:105980000000FEFEFEFEFEFEFEFEFEFEFEFEFEFE33
:10599000FEFEFEFEFEFEFEFEFEFE00D8D800FEFE6F
:1059A000FEFEE8E8D800FEFEFEFEE8E80000FEFE8F
:1059B000FEFEE8000F00FEFEFEFE000F0F00FEFEE2
:1059C000FEFEFE0000FEFEFEFEFEFEFEFEFEFEFEF3
:1059D000FEFEFEFEFEFEFEFEFEFEFEFEFEFEFEFEE7
:1059E000FEFEFEFEFEFE00000000FEFEFE00E8E8F9
:1059F000E8E8FEFEFE00000000E8FEFE00FFFFFFFC
:105A0000FF00FEFE00000000FFFFFEFE000F00A4EE
:105A100000FFFEFE00000000FF00FEFEFEFEFEFE98
:105A2000FEFE0000FEFEFEFEFEFED8D800FEFEFEDC
:105A3000FEFEE8D8D800FEFEFEFEE8E8D800FEFE36
:105A4000FEFE00E8D800FEFEFEFE00E8D800FEFEE6
:105A5000FEFEE8D8E800FEFEFEFEFE00000000D8D4
:105A6000D8D80000000000000000000F0FFFFFFF6B
:105A7000FF00FE000000000000E8FEFEFEFEFE004B
:105A8000E8E8FEFEFEFEFEFE0000FEFEFEFEFEFE5E
:105A9000FEFEFEFEFEFEFEFEFEFE00D8D800FEFE6E
:105AA000FEFEE8E8D800FEFEFEFEE8E8E800FEFEA6
:105AB000FEFEE80000FEFEFEFEFE000F00FEFEFE03
:105AC000FEFE0F0F00FEFEFEFEFE0000FEFEFEFECE
:105AD000FEFEFEFEFEFEFEFEFEFE0A0A0A0A0A0A9E
:105AE0000A0A0A661466666666660A140A0A0A0ADA
:105AF0000A0A0A660A1D661D141D0A660A0A1D6640
:105B0000141D0A660A1D0A1D661D0A660A1D140A6E
:105B10001D660A660A1D141D661D0A0A0A0A0A0A7B
:105B20000A0A666666660A66140A0A0A0A0A0A14F5
:105B30000A0A141D661D0A66140A14661D0A0A66FE
:105B4000140A661D0A1D0A66140A1D0A141D0A6637
:105B5000140A0A1D141D0A66140A0A660A1D146630
:105B60001D0A0A660A1D661D0A1D0A660A661D0AC6
:105B7000141D0A660A1D0A1D141D0A140A0A0A0ABF
:105B80000A0A0A661466666666660A140A1414141B
:105B900014140A0A0A0A0A0A0A0A1D66141D0A6669
:105BA000140A0A1D661D0A66140A140A1D660A668E
:105BB000140A141D0A1D0A66140A0A0A0A0A0A149B
:105BC0000A0A666666661466140A141414140A1423
:105BD000140A0A0A0A0A0A0A0A0AFEFEFEFEFEFE63
:105BE0000000FEFEFEFE0000C8C8FEFEFE00C8C8A3
:105BF000C8C8FEFE00C8C8C8C8C8000000C8C8C8D9
:105C0000C8C8001E0000C8C8C8C8006F000000C88F
:105C1000C8C8FE0000000000000000FEFEFEFEFE00
:105C2000FEFEC80000FEFEFEFEFEC8C8C800FEFE66
:105C3000FEFEC8C8C8C800FEFEFEC8C8C8C800002E
:105C400000FEC8C8C800001E00FEC8C80000006FE3
:105C500000FE000000000000FEFEFE00FF0000004D
:105C60000000FE00FF0700000000FEFE0007070026
:105C70000000FEFE000707070707FEFE00000707FB
:105C80000707FEFE006F00000000FEFE006F6F6F52
:105C900000FEFEFEFE000000FEFE00000000FFFF12
:105CA00000FE00000007FF0000FE00000707006F75
:105CB00000FE07070707006F00FE07070700000048
:105CC00000FE000000FEFEFEFEFEFEFEFEFEFEFEEC
:105CD000FEFEFEFEFEFEFEFEFEFEFEFEFEFEFE00E2
:105CE0000000FEFEFE0000C8C8C8FEFE00C8C8C80E
:105CF000C8C8FE0000C8C8C8C8C800070000C8C897
:105D0000C8C80017000000C8C8C8FE000000000096
:105D10000000FE00FF00000000000000FEFEFEFE8E
:105D2000FEFEC8C80000FEFEFEFEC8C8C8C800FED1
:105D3000FEFEC8C8C8C80000FEFEC8C8C8000007EC
:105D400000FEC8C80000001700FE000000000000B0
:105D5000FEFE00000000FF00FEFEFE000007000047
:105D60000000FEFE000707000000FEFE0007070718
:105D70000707FEFE000707070707FEFE00000707EC
:105D80000707FEFE006F00000000FEFE006F6F6F51
:105D900000FEFEFEFE000000FEFE00000007000008
:105DA000FEFE0000070700FEFEFE0707070700FED5
:105DB000FEFE0707070700FEFEFE0707070000FEBE
:105DC000FEFE000000FEFEFEFEFEFEFEFEFEFEFEED
:105DD000FEFEFEFEFEFEFEFEFEFEFEFEFEFEFEFEE3
:105DE0000000FEFEFEFE0000C8C8FEFEFE00C8C8A1
:105DF000C8C8FEFE00C8C8C8C8C8000000C8000067
:105E00000000001E000000070707006F001E1E00B4
:105E10000000FE00001E6FFF006F00FEFEFEFEFE93
:105E2000FEFEC80000FEFEFEFEFEC8C8C800FEFE64
:105E3000FEFEC8C8C8C800FEFEFE000000C8000084
:105E400000FE07070000001E00FE00001E1E006F7F
:105E500000FE00FF6F6F0000FEFEFE00FF006FFF00
:105E6000006FFE00FF07006F6F6FFEFE0007070068
:105E70000000FEFE000707FFFFFFFEFE0000070711
:105E80000707FEFE006F00000000FEFE006F6F6F50
:105E900000FEFEFEFE000000FEFE00FF6F00FFFFA2
:105EA00000FE6F6F0007FF0000FE00000707006F95
:105EB00000FEFFFF0707006F00FE07070700000056
:105EC00000FE000000FEFEFEFEFEFEFEFEFEFEFEEA
:105ED000FEFEFEFEFEFEFEFEFEFEFEFEFEFEFEFEE2
:105EE0000000FEFEFEFE0000C8C8FEFEFE00C8C8A0
:105EF000C8C8FEFE00C8C8C8C8C8FE0000C8000068
:105F00000000000700000007070700170007070050
:105F10000000FE00000707FF000700FEFEFEFEFE79
:105F2000FEFEC80000FEFEFEFEFEC8C8C800FEFE63
:105F3000FEFEC8C8C8C800FEFEFE000000C8000083
:105F4000FEFE07070000000700FE0000070700171D
:105F500000FE00FF07070000FEFEFE00000707FF2F
:105F60000007FE00171717FF0007FE001717171787
:105F70001717FE00001717171717FE00FF0000176E
:105F80001717FE00000000000000FE006F6F00FE0B
:105F9000FEFEFEFE000000FEFEFE00FF0707000002
:105FA000FEFE00FF17171700FEFE17171717170042
:105FB000FEFE171717170000FEFE17170000FF0060
:105FC000FEFE000000000000FEFEFEFE006F6F00FF
:105FD000FEFEFEFEFE0000FEFEFEFEFEFEFEFE00DB
:105FE0000000FEFEFEFE00C8C8C8FEFE0000C8C8D5
:105FF000C8C8FE000700C8C8C8C8FE00070700C818
:10600000C8C8FEFE000000000000FEFEFE006F009B
:10601000FF00FEFEFE00006F6F00000000FEFEFEAF
:10602000FEFEC8C8C800FEFEFEFEC8C8C8C800FE06
:10603000FEFEC8C8C8C800FEFEFEC8C8C80000FEF4
:10604000FEFE0000000000FEFEFE1E6F000000FECF
:10605000FEFE6F6F000000FEFEFEFEFE0000FF0071
:106060000000FEFE0000FF0700FFFEFEFE00070727
:106070000000FEFEFE000707006FFEFEFE000000AF
:106080000000FEFEFE006F6F6F00FEFEFEFE0000D1
:1060900000FEFEFEFEFEFEFEFEFE00000000FEFE16
:1060A000FEFEFF000700FEFEFEFE00000700FEFEF3
:1060B000FEFE6F000700FEFEFEFE000000FEFEFE7C
:1060C000FEFEFEFEFEFEFEFEFEFEFEFEFEFEFEFEF0
:1060D000FEFEFEFEFEFEFEFEFEFEFEFEFEFEFEFEE0
:1060E000FEFEFEFEFEFEFE000000FEFEFE0000C8FC
:1060F000C8C8FEFE00C8C8C8C8C8FE000700C8C897
:10610000C8C8FE00070700C8C8C8FEFE000000009F
:106110000000FEFEFE006F00FF00FEFEFEFEFEFE23
:10612000FEFE000000FEFEFEFEFEC8C8C800FEFE29
:10613000FEFEC8C8C8C800FEFEFEC8C8C8C800FE2B
:10614000FEFEC8C8C80000FEFEFE0000000000FE03
:10615000FEFE1E6F000000FEFEFEFEFEFE00006F53
:106160006F00FEFEFE00FF000000FEFEFE00FF00CE
:10617000FFFFFEFEFE00070000FFFEFE006F006F47
:106180006F00FEFEFE0000000000FEFEFEFEFEFEB2
:10619000006FFEFEFEFEFEFEFE006F6F0000FEFEC4
:1061A000FEFE00000000FEFEFEFE00070700FEFEF1
:1061B000FEFE00070700FEFEFEFE07000000FEFEDA
:1061C000FEFE006F00FEFEFEFEFE6F00FEFEFEFE07
:1061D000FEFE00FEFEFEFEFEFEFEFEFEFEFE0000D9
:1061E0000000FEFEFE00C8C8C8C8FE0000C8C8C83F
:1061F000C8C8000700C8C8C8C8C800070700C8C882
:10620000C8C8FE00000000000000FE001700FF07E5
:106210000007FE001717171700170000FEFEFEFE0E
:10622000FEFEC8C800FEFEFEFEFEC8C8C800FEFE98
:10623000FEFEC8C8C800FEFEFEFEC8C80000FEFE86
:10624000FEFE00000000FEFEFEFE07000000FEFE57
:10625000FEFE170000FEFEFEFEFE000017171717D9
:1062600000170000000000000000006F00FFFFFFAB
:10627000FF00FE00000000000007FEFEFEFEFE0024
:106280000707FEFEFEFEFEFE0000FEFEFEFEFEFE18
:10629000FEFEFEFEFEFEFEFEFEFE00000000FEFE16
:1062A000FEFE00000700FEFEFEFE07070700FEFEE2
:1062B000FEFE070000FEFEFEFEFE006F00FEFEFE7C
:1062C000FEFE6F6F00FEFEFEFEFE000000FEFEFE04
:1062D000FEFEFEFEFEFEFEFEFEFEFEFEFEFEFEFEDE
:1062E000FEFEFEFEFEFE00000000FEFEFE00C8C830
:1062F000C8C8FE0000C8C8C8C8C8000700C8C8C8C9
:10630000C8C800070700C8C8C8C8FE0000000000D1
:106310000000FE001700FF070007FEFEFEFEFEFE67
:10632000FEFE0000FEFEFEFEFEFEC8C800FEFEFEF3
:10633000FEFEC8C8C800FEFEFEFEC8C8C800FEFEBD
:10634000FEFEC8C80000FEFEFEFE00000000FEFECD
:10635000FEFE07000000FEFEFEFEFE0017171717E8
:106360000017FE00000000000000006F00FFFFFFAC
:10637000FF00FE00000000000007FEFEFEFEFE0023
:106380000707FEFEFEFEFEFE0000FEFEFEFEFEFE17
:10639000FEFEFEFEFEFEFEFEFEFE17000000FEFEFE
:1063A000FEFE00000700FEFEFEFE07070700FEFEE1
:1063B000FEFE07070000FEFEFEFE07006F00FEFE69
:1063C000FEFE006F6F00FEFEFEFEFE0000FEFEFE03
:1063D000FEFEFEFEFEFEFEFEFEFE000102030004C7
:1063E00005060700050407060108090A0B0009084D
:1063F0000B0A010C0D0E0F000D0C0F0E01101112E7
:1064000013001110131201141516170018191A1B76
:10641000001C1D1E1F002021222300151417160129
:1064200019181B1A011D1C1F1E0121202322010007
:106430000000000101010100020100071400001624
:106440000300100100000000E703FF000200000746
:10645000140000020700010100000000F609FF001F
:10646000020400071400000B0400070100000300F1
:10647000FC0200F906FF00010800072C0000E20101
:1064800000F10100F802050000FF000105000721EE
:106490000000E20100F10100F801050000FF000228
:1064A0000100071000000801002003001001000097
:1064B0000006000000E703FF0002040007160000CA
:1064C000100100120100140100000500FF0200FE8F
:1064D0000200FD0200FC06FF0006FF0001020007AB
:1064E000120000F80100FB01050000FF000106009A
:1064F00007140000F80100FB01050000FF00FF0089
:10650000FF00FF00FF00FF0002010009C8000A377A
:1065100000071400001201001A0200100100000020
:1065200006000000E703FF00020400071400000A51
:106530000200070100040100000100FF0100FE014C
:1065400000FC0200F904FF0002010007140000161D
:106550000300100100000000E703FF00010A00072C
:10656000120000F80100FB01050000FF0001060019
:1065700007120000F80100FB01050000FF00010206
:106580000007120000F80100FB01050000FF00FFFA
:1065900000FF0009B4000A3C0002010007140000DB
:1065A0000B0300110100160100000500EA03FF00C3
:1065B000020400070C0000100400000300F509FFAE
:1065C00000020400070201000401000601000801A6
:1065D000000A01000C0400000006000000F40100A5
:1065E000F60100F80100FA01FF0001010007210097
:1065F00000F10100F802050000FF0001050007217D
:106600000000F10100F802050000FF000109000789
:10661000210000F10100F802050000FF00FF000268
:106620000100071400002104000000060000098C8E
:10663000000A270000E703FF00020100071B01001A
:10664000160300000006000000E703FF000201003F
:1066500007140000160400000006000000E703FF16
:106660000001010007210000F10100F8020500000F
:10667000FF0001050007210000F10100F8020500FC
:1066800000FF00FF00FF00FF00FF00FF000202000C
:10669000000A00082D0200FB0300F300082803088D
:1066A0002D0300EA0308280000E602FF0001FF00B6
:1066B0000000003764000000000000004B64000090
:1066C00000000000005F640000000001000076642C
:1066D000000000000100008A6400000000000000CB
:1066E0009E6400000000000000B86400000000008C
:1066F0000000D96400000000010000DB640000001D
:1067000000010000EC6400000000010000FD6400D6
:10671000000000010000FF64000000000100000113
:10672000650000000001000003650000000001009A
:106730000005650000000000000007650000000083
:106740000000002765000000000000004765000011
:1067500000000100005B65000000000100006C65A6
:10676000000000000100007D650000000001000045
:106770008E65000000000100009065000000000030
:106780000000926500000000000000AF65000000FE
:1067900000000000C06500000000010000E9650085
:1067A000000000010000FA65000000000100000B7D
:1067B00066000000000100001C66000000000000F0
:1067C000001E6600000000000000386600000000A7
:1067D0000000004C66000000000100006066000040
:1067E00000000100007166000000000100008266E8
:1067F00000000000010000846600000000010000AD
:1068000086660000000001000088660000000001AC
:1068100000008A66000000000000008C6600000096
:1068200000010000AD660000000000000000000054
:106830000000000000000000000000000000000058
:1068400000000000000055050000000000002505C4
:1068500000000000000015555500000000553531BE
:1068600052000000002531565500000000555553D8
:1068700000000000000050520000000000005055D1
:106880000000000000000000000000000000000008
:1068900000000000000000000000000000000000F8
:1068A00000000000000000000000000000000000E8
:1068B0000000000000505555000000000050165127
:1068C000000000000050315350550000005031517D
:1068D0005052000000505551555200000000551113
:1068E0001152000000001511155100000000151193
:1068F000555500000000555505000000000000003F
:106900000000000000000000000000000000000087
:106910000000000000000000000000000000000077
:10692000000000000000005555550500000000154E
:106930001111550500005035551511050000506125
:10694000311113050000502152315105000050252E
:10695000521151000000005555555500000000002F
:106960000000000000000000000000000000000027
:106970000000000000000000000000000000000017
:106980000000000000000000000000000000000007
:10699000000000000000000000555500000000004D
:1069A000501551000000000050365100000000005A
:1069B000503551050000000050151305000000007F
:1069C0005032110500000000502224050000000094
:1069D00050555505000000000000000000000000B8
:1069E00000000000000000000000000000000000A7
:1069F0000000000000000000000000000000000097
:106A0000000000000000000000505555000000008C
:106A1000005016550500000000503111050000001F
:106A200000551515550000000025151551000000F2
:106A300000251351510000000025113151000000C4
:106A400000555555550000000000000000000000F2
:106A50000000000000000000000000000000000036
:106A60000000000000000000000000000000000026
:106A700000005055555500000055551111510000AA
:106A80000015115255510000001515151151050042
:106A900000151513531205000015154111150500B9
:106AA0000015521313150500005511111515550544
:106AB0000050515512116105005011115115110569
:106AC00000505555555555050000000000000000C8
:106AD00000000000000000000000000000000000B6
:106AE0000000000000000000000000505555550057
:106AF0000000005511155600000000151115510039
:106B000000000035313151000000001553155100CF
:106B1000000055151315550000002522221105000F
:106B2000000055555555050000000000000000000C
:106B30000000000000000000000000000000000055
:106B40000000000000000000000000000000000045
:106B50000000000000000000000000005055550536
:106B60000000005055111105000000551253155535
:106B70000000002532311156000000251213135574
:106B80000000005555551105000000000050550546
:106B900000000000000000000000000000000000F5
:106BA00000000000000000000000000000000000E5
:106BB00000000000000000000000000000000000D5
:106BC000000000005055555555000000501155115A
:106BD00051000000501131115100000050135515A3
:106BE00053000000505122525100000055512252D2
:106BF0005105000015133111130500001511111571
:106C000016050000555555555505000000000000BB
:106C10000000000000000000000000000000000074
:106C20000000000000000000000000000000000064
:106C300000000000000000000000000000005055AF
:106C4000550500000000501111050000005055339B
:106C500013050000005016231205000000503122D9
:106C6000520500000050551551000000000000556D
:106C700055000000000000000000000000000000BF
:106C80000000000000000000000000000000000004
:106C900000000000010000000000000000000000F3
:106CA00000000000000000000000000000000000E4
:106CB00000000000000050550550555500005511CA
:106CC0000550115100001513555513510000153191
:106CD0002222315100005511111516550000505552
:106CE00055555505000000000000000000000000A0
:106CF0000000000000000000000000000000000094
:106D00000000000000010000000000000000000082
:106D10000000000000000000000000000000000073
:106D2000505555000000005055115600000000500D
:106D300011235105000000501132120500000050CF
:106D400055411305000000005011510500000000DE
:106D50005055550500000000000000000000000034
:106D60000000000000000000000000000000000023
:106D70000000000000000100000000000000000012
:106D80000000000000000000000000000000000003
:106D900000505505000000000050220500000000D2
:106DA0000055215500000000001531520000000080
:106DB0005015135105000000501135130500000057
:106DC00050111611050000005055555505000000E2
:106DD00000000000000000000000000000000000B3
:106DE00000000000000000010000000000000000A2
:106DF0000000000000000000000000000000000093
:106E000000505555550500000050111511050000A2
:106E10000050312213050000005036425105000099
:106E2000005031221305000000501115110500001B
:106E300000505555550500000000000000000000FE
:106E40000000000000000000000000000000000042
:106E50000000000000000000010000000000000031
:106E60000000000000000000000000555555000023
:106E700000000015115155000000001513115100BC
:106E80000000551513555100000025223111510005
:106E90000000252253135500000055555131510073
:106EA00000000050111651000000005055555500CB
:106EB00000000000000000000000000000000000D2
:106EC00000000000000000000001000000000000C1
:106ED00000000000000000000000000000000000B2
:106EE000000000505555050000000050111105002C
:106EF000000000503133550000000050112552555C
:106F000000000050152132510000000015161151EB
:106F1000000000005555555500000000000000001D
:106F20000000000000000000000000000000000061
:106F30000000000000000000000001000000000050
:106F40000000000000000000000000000055555542
:106F50005500000000151125510000005015312288
:106F600052000000501113455200000055513515D4
:106F700055000000151113315100000015111511B5
:106F800051000000555555655100000000000055A6
:106F9000550000000000000000000000000000009C
:106FA00000000000000000000000000100000000E0
:106FB00000000000000000000000000000000000D1
:106FC00000000000005055555500000000502222DE
:106FD00051000000005525225355000000153135A1
:106FE00031510000001533113551000000151151C9
:106FF00011510000005555615155000000005055D9
:107000005505000000000000000000000000000026
:10701000000000000000000000000000010000006F
:107020000000000000000000000000000000000060
:107030000000000000000055555505000000002527
:107040003222050000000025522205000000001534
:107050003313050000000015311105000000001574
:1070600033130500000000155116050000000055FF
:107070005555050000000000000000000000000061
:1070800000000000000000000000000000010000FF
:1070900000000000000000000000000000000000F0
:1070A00000000000000000005055550500000000E1
:1070B0005021220500000055552222050000001530
:1070C00051551355050000151313311305000065C4
:1070D000313111110500001511551511050000552C
:1070E0005505555505000000000000000000000097
:1070F000000000000000000000000000000002008E
:10710000000000000000000000000000000000007F
:107110005055555505000000501111110500000093
:1071200050513311050000005021221505000000C8
:107130005025221355000000001555315100000064
:1071400000351113510000000015511156000000C8
:1071500000555555550000000000000000000000DB
:10716000000000000000000000000000000000021D
:10717000000000000000000000000000000000000F
:107180000000000000000000000055550500000050
:10719000005515115555000000151113135100002D
:1071A00000151311135600000055355355550000B6
:1071B00000001521520000000000252252000000AE
:1071C00000005555550000000000000000000000C0
:1071D00000000000000000000000000000000000AF
:1071E000020000000000000000000000000000009D
:1071F00000505555050055550550111155051521DF
:107200000550111313052522055051111355152151
:107210000550113313111326055055111331152143
:107220000500501153132522050050151111152189
:10723000050000555555555505000000000000009B
:10724000000000000000000000000000000000003E
:10725000000200000000000000000000000000002C
:107260000000000000505555050000505555121102
:107270000500005011255215050000501123121170
:1072800005000050111552510500005515555311B8
:1072900005000015131131130500001535155111A6
:1072A00005000065115555550500005555050000B0
:1072B00000000000000000000000000000000000CE
:1072C0000000020000000000000000000000505517
:1072D00055550555555555561122051511113111A4
:1072E0001122051513355153112205555115115110
:1072F00055220550313155515055055051111551F8
:1073000000000055511111510000001531115105B7
:1073100000000015513551000000001551155100B5
:107320000000005555555500000000000000000009
:1073300000000002000000505555550500000050A7
:107340001111110500000050111313055555555525
:1073500031311105252211555551150522221111E2
:107360001151150525221155315315055555555502
:10737000311161050000505551551505000050317F
:10738000311111050000501113555505000050151D
:107390001105000000000055550500000000000028
:1073A00000000000020000000000000000000000DB
:1073B0000000000000000000505555000000555529
:1073C00050115105000015515551110500001513BC
:1073D00022221555000015512542125100001511A9
:1073E00031555351000015531311135100005561CD
:1073F0005155535100005055555111510000000096
:107400000050555500000000000000000000000082
:107410000000000000020000555500000000555516
:107420001551000000001531315150555505151109
:107430001351502424045531315155424202501306
:1074400013511124240450363111114242055013B6
:107450001351112424045531315155424202151162
:1074600013515024240415313151505555055555AB
:107470001551000000000000155100000000000040
:1074800055550000000002000000555555550500F7
:1074900000001511111105000000353133110500F0
:1074A00000001511151305000000151163130500E8
:1074B00000553531515105000015115353510055F8
:1074C00055151551115100252211155351550025FF
:1074D000222211515100002522221553510000553E
:1074E0005555551151000000000050555500000041
:1074F000000000000000000200000000000000008A
:107500005055550555550500555611551511550041
:10751000151131111513510015311115113151008B
:1075200055155555551151005515551155535500C3
:1075300015135155152205001513131321220500AB
:10754000151151552522050015335100252205003E
:107550001551550055550500555500000000000017
:10756000000000000000000003000050555500001E
:107570000000505511510000000050115151000001
:107580000050551113515555055011351551111114
:10759000055013135511311105551115113133557E
:1075A0000515115155131105001553332252550578
:1075B000001511512222050000151516252205007F
:1075C0000015111123220500005511151111050098
:1075D00000505555555505000003000000000000FF
:1075E00000000050555500000000005011510000EF
:1075F00000000050135100000000005011515500D0
:107600000000505511535500000050111331510026
:1076100000005551515551555505115151555115B0
:1076200021023111131111612102551555555111C6
:10763000210200151111515555050055555555009C
:107640000000000000000000000003000000000037
:10765000000000000000000000000000555505007B
:10766000000000001511555555550500151313114F
:1076700011110555551531513311051511155511B8
:1076800011550525221151153105002522351331DB
:107690001105002522156115510500555555555503
:1076A0005500000000000000000000000000000085
:1076B000000000000000000000000003000055551D
:1076C000050000005555151155555500151111159A
:1076D0005115510515153311311111051551115160
:1076E00015151505151315551131110515113131E4
:1076F0001151510555315111355551005055111544
:10770000151553000050311116225200005031550A
:107710005322520000501511222255000000551529
:1077200022520500000000555555000003000000DE
:1077300000000000000050555505000000005011E9
:1077400011550000000050313151050000555551D0
:1077500053115555001513113111155105151131DE
:107760005131222202551515555522220250153548
:1077700031112255055011151153110500503611C4
:107780001351550500501155555500000050550531
:1077900000000000000000000000000000030000E6
:1077A00000505555550500000050111111050000FD
:1077B000005011131305555555553131110525222A
:1077C000115555511505222211111151150525226A
:1077D00011553153150555555555311161050000A9
:1077E000505551551505000050313111110500005B
:1077F00050111355550500005015110500000000EB
:1078000000555505000000000000000000000300C6
:10781000000000000000000055555500550500000F
:107820002512515065550000251251551151000087
:107830002512111133510000251251513151000010
:107840002552555131510000555531511351000009
:1078500000501153315100000050311113510000FC
:10786000005011551151000000505555555500005C
:107870000000000000000000000000000000000305
:1078800000000000000000000000000000000000F8
:107890000000000000000000005055555505000094
:1078A000005022222205000000501113155500003F
:1078B000005031513151000000503531315100003C
:1078C000000015611151000000005555555500008C
:1078D00000000000000000000000000000000000A8
:1078E0000000000000000000000000000000000098
:1078F0000300000000000000000050555555000036
:10790000000050111151555505005011531111111E
:107910000555551331113513051511311313111375
:107920000515531155515551051556353111135142
:10793000001511111331315100555555555533511D
:107940000000252222222255000025222222220583
:107950000000555555555505000000000000000079
:107960000003000000000000000000000000000014
:107970000000000000000000000000000055550558
:10798000000000000015160500000000003533055A
:10799000000000505515110500000050112135550B
:1079A00000000050313212520000005011252555C0
:1079B0000000005055555505000000000000000073
:1079C00000000000000000000000000000000000B7
:1079D000000004000000000000000050555555054F
:1079E0000000005011111105000000501113115535
:1079F00055050050551511131105005011555331FF
:107A000011050050111156515155055551151313BB
:107A100033110115111551115111011511555555FC
:107A20005555052522520000000000252252000075
:107A30000000005555550000000000000000000047
:107A400000000004005555050000000055151155B3
:107A500000000000151111510000000015335153B2
:107A6000555555055551131313151105252252115E
:107A70003111110525226215515553052522321564
:107A80001113130525223231151111055555151104
:107A9000155353050000555515111305000000003E
:107AA00055151105000000000055550500000000A7
:107AB00000000000040000000000000000505555C8
:107AC00050555505005011515511110500553131D2
:107AD000511335050015316131111355001515513C
:107AE0005122220500155115132555520055111329
:107AF00011212252005031133525225200501151CC
:107B00001151135500505555311111050000005009
:107B100055155105000000000055550000000000FB
:107B200000000000000400000000000000005055AC
:107B300055555555050050221215111105005022BA
:107B40001115551105005022111151110500502237
:107B500011155315050050221235311105005055ED
:107B6000551531130500005511133311050000653B
:107B70003133111505000055315115110500005024
:107B80001111111105000050555555550500000003
:107B9000000000000000040055555555000000008D
:107BA0001511155155000055151513315155001576
:107BB0001151335111510015555311163151001502
:107BC0001131535513550015115351155105001519
:107BD000355121225500001513252222050000559C
:107BE0001122225205000050311555550000005059
:107BF00015110500000000005555050000000000AB
:107C0000000000000000000400000000555555056C
:107C10000000555515111105505515131313130573
:107C200050111531515511055011111611511305EF
:107C30005051555155111105505122225231130501
:107C40005051222252115305555322223211510014
:107C5000151151151551550015131311335100000D
:107C6000551155551551000050550500555500004A
:107C70000000000000000000045055550000000006
:107C80000055115105000000001511115555050052
:107C90000015151131110500001551315115050060
:107CA00000553153221205000050551122120500D3
:107CB0000000505525525555005555552252155125
:107CC0000015515531163551001513151115115167
:107CD000001531113511135500551111135155056A
:107CE0000050555511550000000400000000000030
:107CF000000000000000000000000055555555052B
:107D00000000001511111105000000153131310579
:107D10000000005551531505000000502112225556
:107D2000000000502512225100000000155553514B
:107D300005000000353131110500000015111161F9
:107D400005000000555555550500000000000000D5
:107D50000000000000000000000004555505000070
:107D600050550565115555555511055531111111D0
:107D7000311105505151115555110550111311551F
:107D8000555305501355513131510055311153118F
:107D9000115100151115111151510015115555357D
:107DA00055550055551511151105000000252211D6
:107DB0001305000000252252110500000025225263
:107DC0005505000000555555000000045555555502
:107DD0005505000015115522225555051531112262
:107DE0005215110555351322551515050015552247
:107DF000523511050015151155155105501515135E
:107E00003131510050111515151151005011111536
:107E1000133551005031131553115500505551155C
:107E200051510500005016111151000000505555D8
:107E300055550000000000000000000000C30300D2
:107E4000C20200C10100C00000B0075A0007730061
:107E500090516400B1076400B2077F009221640072
:107E6000FF0601530D9040640743640E4B6400927B
:107E7000246407905264009228640E904764075867
:107E800064009224640D904364075164009221645D
:107E90000E9051640092216407903E640E4C640081
:107EA00092246407905164009228640690506407FD
:107EB00051640758640092246415904A6400922625
:107EC0006407904A64074B640092326407904C64E4
:107ED0000092266407904C64064F64009232640757
:107EE000904B640092276407904B64074F640092A4
:107EF000336407904B640052640092276407904BF0
:107F0000640757640092336407905664075564060B
:107F10005464075364075464075564075664009219
:107F2000216404905464035164034F64044D64035A
:107F30004864044A64009221640AB0075A00077337
:107F40000090420100B0077F0A922101D555FF063B
:107F5000014500FF2F0000C20200C10100C0000067
:107F6000B0077F00903A6400B1075A00B2077F0063
:107F7000921F6400B3077F00FF0601530C903B641F
:107F800007436400914764009304640C903A6400D2
:107F90009147640093046407903B64009226640C4C
:107FA000904364073A6400914764009303640C9023
:107FB0003B6408436400921F640C903A640193038D
:107FC0006402036402046402903B6400914764000D
:107FD000921F64009304640C904364009147640012
:107FE00093046407904164009221640C90406408FB
:107FF0003F640091476400922364009303640C90F3
:108000003E64073C640092246413903C64009148F1
:1080100064009304640C903E6400914864009304EF
:108020006407903F6400921F640C904064084864A9
:1080300000914864009303641390466400922464A2
:108040001390456400914864009224640093046492
:108050000C9148640093046408903F640092236488
:108060000C904064073C64009148640092216400D5
:108070009303640C036407921F640C9047640746E3
:108080006400914764009304640D90476400914735
:10809000640093046407904564009226640C904346
:1080A0006407914764009303640C90476407466437
:1080B00000921F640C9047640193036402036402FE
:1080C00004640390456400914764009304640C9039
:1080D00043640091476400930464079226640C9003
:1080E000456407436400914764009303640A036492
:1080F000029045640847640091486400922464003B
:1081000093046413904864134264134364143F64FB
:108110000C4064073F640C4064073B64143C6413E8
:10812000376400921F640C903664073A64009147EC
:1081300064009304640C903B6400914764009304D2
:108140006407903E64009226640D903B640743648C
:1081500000914764009303641390416400921F648C
:108160000C90376401930364020364020464029078
:10817000406400914764009304640C90376400915C
:1081800047640093046408903E64009226640C9057
:108190003F6407406400914764009303640C903788
:1081A00064073C640092246414903C640091486429
:1081B000009304640C903E6400914864009304644E
:1081C00007903F6400921F640C904064074864006D
:1081D00091486400930364139046640092246414ED
:1081E0009045640091486400922464009304640CF8
:1081F00091486400930464079043640092266413DA
:108200009040640091486400922864009303640CD9
:1082100003640890456400914864009229640093C7
:1082200003641390456400914864009229640093AC
:1082300003640C036402921F640590476400914834
:108240006400922B6400930364139045640091488A
:108250006400922B64009303641490436400914C77
:108260006400922B64009303640C904264029303B5
:10827000640303640290436400914C6400922B6495
:10828000009303640C90456400930364039221649B
:1082900004914C6400922D64009303640C90436439
:1082A00008406400914C6400922D640093036413B1
:1082B000903E6400914A6400922464009303641326
:1082C000903E6400914A6400922464009303640E1B
:1082D00003640690436400914C6400921F64009311
:1082E00003640C903F64073E6400914A6400921F4F
:1082F000640093036413903C6400914C64009224E6
:1083000064009303640A03640990376400914A642B
:1083100000921F64009303641490486400914864C1
:10832000009230640093036426921F6414914764A2
:10833000009304640C9147640093046407922664DC
:10834000139147640093036413921F640D930364B5
:108350000203640204640391476400921F64009363
:1083600004640C91476400930464079221641391A0
:10837000476400922364009303641492246413916D
:108380004864009304640C91486400930464079269
:108390002B64149148640093036413914864009221
:1083A0003064139304640C04641B036409FF060126
:1083B0004500FF2F0000C37500C20000C10600C0C9
:1083C0000500B0077F00B1077F00077E00077E0031
:1083D000B2077E00077E03905064009128700093DE
:1083E000087F00FF0601530990516409506400930F
:1083F000097F099051640093097F089053640093AA
:10840000087F12905164009126700093097F1290AA
:1084100050640091286D0093087F1190516400937F
:10842000097F129050640091296E0093087F12908A
:108430004D640093097F12904C6400912870009362
:10844000087F08904D64094C640093097F09904DA2
:10845000640093097F099050640093087F12904D47
:1084600064009126700093097F11904C640091285C
:108470006D0093087F12904D640093097F12904C19
:10848000640091296E0093087F11904A640093095B
:108490007F12904764009128700093087F099048EC
:1084A000640947640093097F099048640093097F39
:1084B00008904B640093087F1290486400912670E6
:1084C0000093097F129047640091286D0093087F04
:1084D000119048640093097F129047640091296EBF
:1084E0000093087F129045640093097F11904464C3
:1084F000009128700093087F099045640944640046
:1085000093097F099045640093097F0990446400B2
:1085100093087F12904164009126700093097F11A7
:108520009040640091286D0093087F12097F230911
:108530007F12905064009128700093087F09905139
:10854000640950640093097F089051640093097F87
:10855000099053640093087F129051640091267033
:108560000093097F129050640091286D0093087F5A
:10857000119051640093097F129050640091296E0C
:108580000093087F12904D640093097F11904C6412
:10859000009128700093087F09904D64094C640095
:1085A00093097F09904D640093097F0990506400FE
:1085B00093087F11904D64009126700093097F12FB
:1085C000904C640091286D0093087F12904D6400D8
:1085D00093097F11904C640091296E0093087F12DB
:1085E000904A640093097F129047640091287000BC
:1085F00093087F099048640947640093097F0890B5
:1086000048640093097F09904B640093087F12909F
:108610004864009126700093097F1290476400918E
:10862000286D0093087F119048640093097F129091
:1086300047640091296E0093087F1290456400936F
:10864000097F11904464009128700093087F09907D
:1086500045640944640093097F09904564009309C7
:108660007F099044640093087F1190416400912633
:10867000700093097F129040640091286D12930955
:108680007F11087F0408660408660A097F12904774
:1086900064009128700093087F099048640847643B
:1086A0000093097F099048640093097F09904B6407
:1086B0000093087F12904864009126700093097F10
:1086C000129047640091286D0093087F11904864D0
:1086D0000093097F129047640091296E0093087FF0
:1086E000129045640093097F1190446400912870B2
:1086F0000093087F099045640944640093097F0949
:108700009045640093097F099044640093087F11A9
:10871000904164009126700093097F12904064009C
:1087200091286D0093087F12097F11097F12097F3C
:1087300012904764009128700093087F0990486464
:108740000847640093097F099048640093097F09F2
:10875000904B640093087F0E91267004904864004B
:1087600093097F11904B640091286D0093087F124C
:108770009048640093097F129047640091296E002D
:1087800093087F129045640093097F119044640020
:10879000912870099045640944640945640944645A
:1087A00011416400912670129040640091286D2759
:1087B0009309660309660409660B08660A91286630
:1087C000092966092C66092D7F092F7211307F1245
:1087D000337F123072112F661230661234720835F0
:1087E0007F093472093372093066122F66112D66C3
:1087F000092E66092D7F092C660929661127721238
:10880000FF06014500FF2F0000C11800C01700C27D
:108810001900C37306931A6C00B3077F00B2077F79
:108820000092386C00B0077F00B1077F0091206E86
:1088300000FF0601530C931C6C0D1B6C0091246E01
:108840000C931C6C0091276E0D931A6C0091256E91
:1088500006256E07931C6C0091256E0C931B6C0013
:1088600091296E0D931A6C00912C6E0CB3077F004A
:10887000931A6C0091206E0D931C6C0C1B6C009174
:10888000246E0D931C6C0091276E0C931A6C009152
:10889000256E07256E06931C6C00911D6E0C931BB4
:1088A0006C0092366C00911E6E0D931A6C00911F35
:1088B0006E0DB3077F00931A6C0092386C00912004
:1088C0006E0C931C6C0D1B6C0091246E0C931C6C35
:1088D0000091276E0D931A6C0091256E06256E0689
:1088E000931C6C0091256E0D931B6C0091296E0CEE
:1088F000931A6C00912C6E0D931A6C0091206E0CE3
:10890000931C6C0091206E0D931B6C0091246E0DD6
:10891000931A6C0091276E06931A6C061B6C0091DB
:10892000256E06256E07931A6C0091296E0C931B19
:108930006C00912A6E0D931A6C0092366C00912B8C
:108940006E0C931A6C00B3077F0092386C00912074
:108950006E0D931C6C0C1B6C0091246E0D931C6CA3
:108960000091276E0C931A6C0091256E07256E06F8
:10897000931C6C0091256E0D931B6C0091296E0C5D
:10898000931A6C00912C6E0DB3077F00931A6C0044
:1089900091206E0C931C6C0D1B6C0091246E0C933B
:1089A0001C6C0091276E0D931A6C0091256E0625A4
:1089B0006E06931C6C00911D6E0D931B6C0092361D
:1089C0006C00911E6E0C931A6C00911F6E0DB30714
:1089D0007F00931A6C0092386C0091206E0D931CEE
:1089E0006C0C1B6C0091246E0D931C6C0091276E17
:1089F0000C931A6C0091256E06256E07931C6C0073
:108A000091256E0C931B6C0091296E0D931A6C00CE
:108A1000912C6E0C931A6C0091206E0D931C6C00BF
:108A200091206E0C931B6C0091246E0D931A6C00B8
:108A300091276E06931A6C071B6C0091256E062514
:108A40006E06931A6C0091296E0D931B6C00912A8F
:108A50006E0C931A6C0092366C00912B6E0D931A6B
:108A60006C00B3077F0092386C0090486E00912034
:108A70006E0C931C6C0D1B6C0090486E0091246E64
:108A80000C931C6C0091276E0D931A6C0090466E2F
:108A90000091256E06256E07931C6C0090466E00B3
:108AA00091256E0C931B6C0091296E0D931A6C002E
:108AB00090466E00912C6E0CB3077F00931A6C00E9
:108AC00090486E0091206E0D931C6C0C1B6C0090F6
:108AD000486E0091246E0D931C6C0091276E0C93D0
:108AE0001A6C0090496E0091256E07256E06931C46
:108AF0006C0090496E00911D6E0C931B6C00911ED2
:108B00006E0D931A6C0092366C0090496E00911FA6
:108B10006E0DB3077F00931A6C0092386C0090487A
:108B20006E0091206E0C931C6C0D1B6C0090486EB7
:108B30000091246E0C931C6C0091276E0D931A6C9F
:108B40000090466E0091256E06256E06931C6C0003
:108B500090466E0091256E0D931B6C0091296E0C52
:108B6000931A6C0090466E00912C6E0D931A6C0057
:108B700090486E0091206E0C931C6C0091206E0D3D
:108B8000931B6C0090486E0091246E0D931A6C003C
:108B900091276E06931A6C061B6C0090496E00912B
:108BA000256E0690496E0091256E07931A6C009011
:108BB000496E0091296E0690496E06931B6C0090D9
:108BC000496E00912A6E0D931A6C0092366C0090DB
:108BD0004B6E00912B6E0C931A6C00B3077F0092C2
:108BE000386C0090486E0091206E0D931C6C0C1B2D
:108BF0006C0090486E0091246E0D931C6C009127C0
:108C00006E0C931A6C0090466E0091256E07256ECF
:108C100006931C6C0090466E0091256E0D931B6CA4
:108C20000091296E0C931A6C0090466E00912C6E88
:108C30000DB3077F00931A6C0090486E0091206E70
:108C40000C931C6C0D1B6C0090486E0091246E0CF4
:108C5000931C6C0091276E0D931A6C0090496E0066
:108C600091256E06256E06931C6C0090496E00914E
:108C70001D6E0D931B6C00911E6E0C931A6C00926E
:108C8000366C0090496E00911F6E0DB3077F009304
:108C90001A6C0092386C0090486E0091206E0D9313
:108CA0001C6C0C1B6C0090486E0091246E0D931C84
:108CB0006C0091276E0C931A6C0090466E00912503
:108CC0006E06256E07931C6C0090466E0091256E13
:108CD0000C931B6C0091296E0D931A6C0090466EDC
:108CE00000912C6E0C931A6C0090486E0091206ECF
:108CF0000D931C6C0091206E0C931B6C0090486EC1
:108D00000091246E0D931A6C0091276E06931A6CD5
:108D1000071B6C0090496E0091256E0690496E000D
:108D200091256E06931A6C0090496E0091296E068B
:108D300090496E07931B6C0090496E00912A6E0C4F
:108D4000931A6C0092366C00904B6E00912B6E0D56
:108D5000B3077F00077F00077F00077F00077F00C2
:108D6000077F00077F00077F00077F00077F00075E
:108D70007F00077F00077F00077F00077F00077FD6
:108D800000FF06014500FF2F0000C37300C1100063
:108D9000C21100C00F00B0077F00077F009312646C
:108DA00000FF060153109245640093136604924637
:108DB0006404913A64089245640093126410913DF2
:108DC0006400931366109246640091366400931217
:108DD00064089246640091366408931366089242D0
:108DE0006400913564009312641012640891336436
:108DF00000931366109243640091316400931264EF
:108E0000049244640C46640091316400931366102C
:108E1000924764009135640093126408924864009C
:108E2000913864089313660892496408913164008C
:108E300093126410905C64085E6400913564009342
:108E4000126410905B640093126408905C6400915B
:108E500030640093136610912F6400931264109293
:108E60004664009313660492476404913364089245
:108E7000426400931264109136640093136610925A
:108E8000476400912F640093126408924764009134
:108E90002F640893136608924B6400913364009327
:108EA000126410126408913664009313661092499C
:108EB00064009136640093126410924B6400931323
:108EC000661092496400913664009312640A9248D5
:108ED0006400913A64069313660592476400913DDD
:108EE000640B9054640092466400913664009312BF
:108EF00064049055640C57640091366400931366C3
:108F00000890556400913A64009312640812660850
:108F1000905464009312640890536400913D64007F
:108F200093136608905264084E6400912F64009376
:108F300012640813660890526400924A64049053C5
:108F40006400924B640491336408904E640092472D
:108F500064009312640813660891366408905364A1
:108F600000924B6408912F64009312640813660802
:108F700090576400924E6400912F6400931366082A
:108F80009133640093136608905A64009251640010
:108F90009313660813660490596400925064049118
:108FA0003664009313660890576400924E640093F1
:108FB0001366089055640091366400931264109013
:108FC00055640093136608913A64089055640093C1
:108FD00012640C90546404913D64009313660890ED
:108FE00053640857640091336400931264109057DF
:108FF00064009313660891366400931264089057D6
:1090000064089312640490556404913A64009313C5
:1090100066089052640850640091316400931264B1
:109020000890506408931366089052640091356468
:1090300008931264089053640854640091386400E3
:109040009313661090556400913B64009312641072
:109050009057640093136608913364009312641070
:10906000905264009312640890506400913464003C
:1090700093136610904E640091366400931264104E
:10908000136608913A640893126410913D6400934A
:109090001366101264089131640890616400913184
:1090A00064009313660814660490613C04605A00DF
:1090B0009133640093146608146604906037045F6B
:1090C0005000913564009314660C905F3204505543
:1090D0000091366400931466029051640293146602
:1090E0000C913664109050550091366400931466CC
:1090F00002905164029314661C905055009136649E
:109100000093136602905164029312660C904E64B1
:10911000009136640093136608904C6400913A64A1
:109120000093126408126608126408904E6400915D
:109130003D6400931366109050550091366400937F
:109140001264029051640E505500913664009313DE
:1091500066029051640E505500913664009312647B
:10916000029051640E4E640093136608904E6400A2
:1091700091366408904C640093126408904864002F
:109180009136640890486400931366089047640021
:10919000913664009312640890456400913A640823
:1091A000904264009312640890426400913D640010
:1091B00093136608904264084E6400912F640093F4
:1091C000126405904764054E6406476400912F645D
:1091D0000093136605904E64054764034E6403577D
:1091E0006400912F640093126408905764089313ED
:1091F000660890576408576400912F6400931264C6
:109200000890536408536400912F64009313660818
:1092100091336408905A640093126608905A64006F
:1092200093126408905764009136640093136608A3
:10923000905364084E64009132640093126410915C
:1092400032640093146608146608905164009136E5
:10925000640093146608146608905364009139649E
:1092600008346408931264089134640890526400CE
:109270009313660891346400931264089058640054
:10928000913864089312640890596400913B64001B
:1092900093136602905A640E913664009312641020
:1092A000905964009136640093136602905A640EDC
:1092B000913664009312641090596400931366020F
:1092C000905A6406596400913564089312640891B9
:1092D00035640890556400931366089135640093D3
:1092E00012640890526400913A6400931266081266
:1092F0006408905C6400913D640093136602905D85
:1093000064065C64025D64065C64009133640093EF
:10931000126402905D64065C64025D64065C640035
:109320009133640093136602905D64065C64085D8B
:1093300064009133640093126408905D6408931391
:10934000660891336408905D640093126408905D30
:10935000640091336408905A64009313660890582F
:1093600064005A6400913364009312640890586456
:109370000091366408905464009312640890546419
:1093800000913A6400931366089053640851640096
:10939000913264009312641090556400913264001D
:1093A00093136608905564085564009132640093E5
:1093B0001264089055640853640093136608905330
:1093C00064009132640890586400931264089132EA
:1093D00064089055640855640091326400931264E7
:1093E00008905364009136640890556400931264A9
:1093F00008913964009313661091316400931264EC
:10940000089049640093136608904E64009131649B
:109410000890506408506400913664009312640808
:10942000905564009138640093136608905A64085C
:109430005C64086164005C640091376400931264AA
:1094400008906164009137640093146608146608FC
:109450001466089061640091386408905864009123
:109460003164009314660891336400931466089184
:1094700035640093146608FF06014500FF2F0000C5
:10948000C22000C11F00C37300C01E0093226400ED
:1094900091296400FF0601530B9322640B21640C95
:1094A0002264009129640B93226400912C640B9335
:1094B00022640C21640B226400912C640B932264BF
:1094C00000912E640C9322640B21640C22640091A1
:1094D0002E640B932264009130640B9322640091FC
:1094E0002E640693226406226400912C640B93215F
:1094F00064009127640B932264009129640C9322E9
:10950000640B21640B2264009129640C9322640093
:10951000912C640B9322640C21640B226400912C27
:10952000640B93226400912E640C9322640B2164DB
:109530000B226400912E640C932264009130640B22
:109540002E640C93226400912C640B93226400918E
:1095500027640B932264009129640C9322640B21ED
:10956000640B2264009129640C93226400912C64A2
:109570000B9322640B21640C226400912C640B93E6
:10958000226400912E640C9322640B21640B2264EC
:1095900000912E640C932264009130640B9322643A
:1095A00000912E640B93226600912C640C9321642D
:1095B000009127640B904B6400932264009129640E
:1095C0000B904D64009322640C904B6400932164D3
:1095D0000B90486400932264009129640C904B64C2
:1095E0000093226400912C640B904D6400932264DC
:1095F0000B21640C904B640093226400912C640B4B
:1096000093226400912E640B904D64009322640CAD
:10961000904B64009321640B904864009322640093
:10962000912E640C904B6400932264009130640B83
:10963000904D640093226400912E640B904B640063
:1096400093226400912C6406932264069046640081
:10965000932164009127640B904864009322640076
:109660009129640B904864009322640C21640B22BE
:1096700064009129640B93226400912C640C932262
:10968000640B21640C226400912C640B932264000F
:10969000912E640B9322640C21640B226400912EA2
:1096A000640B932264009130640C93226400912E29
:1096B000640B93216400912C640C93226400912725
:1096C000640B904B6400932264009129640B904DCD
:1096D00064009322640C904B64009321640B9048C7
:1096E0006400932264009129640B904B64009322E0
:1096F0006400912C640C904D64009322640B2164EF
:109700000B904B640093226400912C640C932264B0
:1097100000912E640B904D64009322640C904B6476
:10972000009321640B9048640093226400912E649E
:109730000B904B6400932264009130640C904D6454
:109740000093226400912E640B904B64009321647B
:1097500000912C640B90466400932264009127646E
:109760000C90486400932264009129640B93226456
:109770000B21640C2264009129640B9322640091F4
:109780002C640C9322640B21640B226400912C64E2
:109790000C93226400912E640B9322640B21640CC1
:1097A000226400912E640B9322640091306406932E
:1097B0002264069048640093226600912E640B9008
:1097C0004B640093216600912C640B904D640093D0
:1097D0002264009127640C905064009322640091ED
:1097E00029640B9322640B904D64009321640C90C8
:1097F0004B6400932264009129640B904D640093A4
:10980000226400912C640B9322640C904B640093AF
:1098100021640B9048640093226400912C640C90A6
:1098200046640093226400912E640B904864009378
:1098300022640B904464009321640C904164009373
:10984000226400912E640B90466400932264009180
:1098500030640B9048640093226400912E640C9055
:1098600044640093216400912C640B904164009344
:109870002264009127640C90466400932264009156
:1098800029640B904864009322640B21640C2264C9
:10989000009129640B93226400912C640B93226441
:1098A0000C21640B226400912C640B9322640091C0
:1098B0002E640C9322640B21640C226400912E64AC
:1098C0000B932264009130640B90416400932264F6
:1098D00000912E640C9044640093216400912C64E8
:1098E0000B90466400932264009127640B904864B7
:1098F00000932264009129640C9322640B904664C7
:10990000009321640B9044640093226400912964C5
:109910000C9046640093226400912C640B932264A3
:109920000C904464009321640B9041640093226482
:1099300000912C640B9044640093226400912E6487
:109940000C9322640B904164009321640B903F645C
:109950000093226400912E640C9041640093226471
:10996000009130640593226406904464009322645D
:1099700000912E640693226406904664009321644D
:1099800000912C640B90446400932264009127643E
:109990000B29642229640C2C64222C640B2E642273
:1099A00093226400912E640C93226400913064052C
:1099B00093226406226400912E640693226405219A
:1099C0006400912C640C932264009127640BFF06C1
:1099D000014500FF2F003A74C100115F752937F26D
:1099E00037A40AA0B5F0559772237FA30ACA5C7505
:1099F0002937F203117F3D08AA15F05FEA0FAA6527
:109A0000737CCDA8FEA05A36FF8FA90AFF9DEA0FEE
:109A1000AA051177973E9883057065730011175F4B
:109A200097A2C99FFE83A0055F97A20011AA80C8D4
:109A30005B57A60A08F0F35F9A26F47765AA8000C0
:109A40005FD7E9C07765AAF03C179A5AFFFC3DAA98
:109A5000001195A5889D0E335875FA0F285636804B
:109A600015FC0F762A5600116AEAF4A8FF835AA75C
:109A70008CF7978C2A11225A835CA9F237DC3DAA15
:109A80000929303F5F05A0A959FDDFA3A235722A3D
:109A9000305805FCF355A9A9F2373F80AA5805FCB8
:109AA0007F959A2ADF0011FD3C6899F283057F6259
:109AB0000011A39ACAAF60F63DDFA3FE83C6973AB2
:109AC000DC291169CAF3A5F5A4803611C243693DAA
:109AD000503DA6027F6A3D8C095D0D00112DDCE32F
:109AE0007C5A3D227CA60A67AF3532110AC2D608DD
:109AF000FC7DA9FE83A256A70C7C627532C227D6D4
:109B0000E9F0F197AA570FA3627FF598302A1188E0
:109B1000F0D70968735DC2F598A4F28AF017A83DE2
:109B200007118C3098A2FD735697005429503D8040
:109B3000A2FDAB367F9502F25637A4A0D6DF6302B2
:109B40003211A2F40863F5643D0FFAA52908FC89D7
:109B5000560F63652A6C3D50D7F3A05F9AC250A69A
:109B6000C84DD733A397290C1103A0FE950C6AD6D4
:109B7000D0372469D6207F5309A326375F4289D680
:109B8000001170DFC3E895720363A56A3D29FC37B5
:109B90008CD53DAAA2D693C27F03D540F59850AA92
:109BA00089FC370011088A0A1F5A0F9FD85F5D0A87
:109BB000636902F5F3A92600112A685DF608C2550B
:109BC000366001DA73D90B7C8F8A55C027960D1148
:109BD0006ACAFF5C816AAAF50FF2DF40A95682FCCF
:109BE000CF856AA5227F23FF0DA92A9635F237F289
:109BF00073A12A1AA059FFFFCFA92A58AAC05FA0B3
:109C000059FFFFF38985A62603A259FFFF37639208
:109C1000A6A60CA059FFFF3772AA82A2CD7529FF14
:109C20007F43AA821A5AFFFF0F110F3F40955A0A2D
:109C3000FF0D50A9205C056CF58368A5F500F25670
:109C40003FF07509A95A0A5B0F3FF075AA5A0AFF3F
:109C50000D940AC2555A4F0AFF0D001195C2FF73A9
:109C6000A1AAAA5695350020FFFFCF856AA98C9A34
:109C7000F2FFFF73AA969A35C0A829FFFFDFC8A993
:109C8000965A3D0329FCCFA9AA9AF50D940AFCFF28
:109C9000BF6A95590900940AFCFF37726AA9A9D5D1
:109CA000F32500940AFCFF0F112AD40F009AFC55EB
:109CB000A582D68CAA2AF6FF57BD2500A3AAFAFFD3
:109CC00057A5DC00A3AAC9F8F73F0C5F55AA585D59
:109CD0000230AA8AFDFFC3605500FC55A58AD52530
:109CE00000A3AAFEFF03682D7C5500FC55A58AD56C
:109CF0002500A36A327EFF83325705C05F55AA58FC
:109D00005D0230AA62FF7FFDA59A00A3AAFF3FC0B3
:109D10005F8A55C05FA5FA5FAA02A39A8CF73FFC41
:109D2000285605FC55AAFFA52A30AA021122F03FA9
:109D30007C97FEA5F4A08368A9660DF2AF563D435B
:109D40007A29206FFDFDF0A52A6A3D297CD3FFA565
:109D50000011F7FCDFBD225C1CC25781A4AAA6FC3F
:109D6000FFDF40A9AA6067CAFFFF5CA8AA2ACFD973
:109D7000FFDF90AA0A8055F6FFCFA9AA006ACA3F62
:109D800057D9FF3772AA0AA0F65CD9FF73AA0A68EE
:109D9000D9FFFFAA0AA8F673D9FF8D9CAAAA80FC56
:109DA0007395FDDF90AAA60980FC7395FDCFA96A83
:109DB000A63520FFFFAB5A8AD620FF7F23A75A265D
:109DC0005A03F2FF73AA655D0220FFAF5AD680FCEA
:109DD0008D9C5AA97D03C83F118A568D5AFDA40255
:109DE0005FA7AA18FFF0C0275675AA62FCF0237C73
:109DF0006255A7AAFF33207C6255A79A8CFEF0F02B
:109E0000A75875AA180F0F0C5655A72A0F0FC05741
:109E1000A758756A32FAF000FC7FA52A56756A3297
:109E20000E0FFF575AA500306255A762FFF500508C
:109E30000FA86255A7CAF000FC175FAA6255A703D6
:109E40005A010FFFA06255752AF000FF77AA6255EC
:109E5000A700117D56A5DC505A237C2770FFCF85C3
:109E6000AA6A8DFC3F17AAAAF68DFCFF9CAA9A5AF3
:109E700083FCFFF38905C383569D18032A9A5697DE
:109E8000F2FF73C02356A0A26975FF33007655AA6E
:109E90008AC0F33D57A0A229DA5C7529FFFFAA8A80
:109EA000C0839D587529FFBFAA2A3780DC839D583F
:109EB00065FF0F11F7AB880A7F657FC3588AB075BD
:109EC0000F0C20C257559D090380A2FDC25755D9DA
:109ED000002A20F783662F7C55953572A90868F60D
:109EE000C257F637A4080858652F7C657F33002ACF
:109EF0008A55F6C257F6F700C0AFD64F2A7CA78323
:109F000056053C6215C0737CAAA9027F55FC089FC8
:109F100058A718116AA90AFFFFCFA9AA2A30580525
:109F20005AFDFF7F23A72AA062055AFDFF3FA72AFB
:109F3000A0C299D53FA062055AFDFFFFAAAA2ADA5E
:109F4000FFFFDFC8A9020AA055055AFDFF3F114ACD
:109F50008FA862F17FC9A858FC00DA5C75C9A862B5
:109F6000FFF028DA5C75C9A86873F1F7C333AA2A31
:109F7000DA5C75C9A8D87F3F483FA82ADA5C75C962
:109F8000A868730F7FCFA82ADA5C75C9A8FEF737D7
:109F9000C0A82ADA5C75C9A87FFF83F089D5A99A81
:109FA0008C021165CFF0A4025429C873055AFD3DF7
:109FB000D8899D0E5A3620A03083A65AF5FF730526
:109FC0005AFD3DD8899D0E5AA0FEA52250DD0F02F4
:109FD0000A3368AA55FF3F57A0D5DF839DD8E920F3
:109FE000A06AF5FF3DD8899D20A0AA36D72520FF7D
:109FF00073055AFD3D5828A00A336815A05AF5FF8D
:10A0000073055AFD3DD88921A00AA0CD15A05AF5A7
:10A01000FF73055AFD3DD88902AAAA70F6FF7305A1
:10A020005AFD732AC083AA835601AA75F73F57A029
:10A03000D5BF02D083FE973A689DD533942900FCA2
:10A04000973A6855C05F992AA0D6FD2FC05F992A1C
:10A050003057A0D52F00A8835601AA75F73F57A007
:10A06000D503110CF07F3F678FAA70F6BF2AAA02B2
:10A070005FA0D53F673F67A38288055AFD73F6AF9F
:10A08000A22ACC85D63F67DF839DA9FE83A226FF47
:10A090007DA9A6C080D63F672F6A56CF3F83296A25
:10A0A000D6FFAA029AF2FF73F6732A6AD6D7C8AB14
:10A0B000025A650D80FC3F67BFA2AA6DD503C83F59
:10A0C000672F6AD6973A8056D600C8FF7336112A92
:10A0D000D40F009AFC55A582D68CAA2AF6FF57BD4C
:10A0E0002500A3AAFAFF57A5DC00A3AAC9F8F73FE9
:10A0F0000C5F55AA585D0230AA8AFDFFC360550067
:10A10000FC55A58AD52500A3AAFEFF03682D7C5522
:10A1100000FC55A58AD52500A36A327EFF833257FD
:10A1200005C05F55AA585D0230AA62FF7FFDA59A5F
:10A1300000A3AAFF3FC05F8A55C05FA5FA5FAA02CD
:10A14000A39A8CF73FFC285605FC55AAFFA52A3098
:10A15000AA02115D5EC6600CA6AA62F1FF7F293DCE
:10A16000A8AA26FCFDD78CAA8AC5FF7F9502A3AAC0
:10A1700062FF7FD5C0A8AAC9F8FD7F552900A3AA10
:10A1800009DF7F550A50F500A88AFD57293750F599
:10A1900000A8EA7F95D6203750F500A826E3FD57A2
:10A1A000D5008CAA0A1102A3573D2650DFA32930FF
:10A1B0005FA0A9CDF3652908BF5A239F9520377268
:10A1C000D5A3095CCFA7260011C2CFF0F77F595A5B
:10A1D0009DAACAFF035F0E5A9DAAF23F8F58A7AAF5
:10A1E000FE3FF030A88A5AD6A8D6FD7C3F77629D04
:10A1F000AAFC838AF63F7762A7AAFF83AA2AC27FB6
:10A20000816ADDFF3F77629D2A3FF030A88A5A15A8
:10A21000A8D6FDFF732776AAFE030F836AEA835A46
:10A2200015A8D6FDFF7327D6A93CF0C0A8A60A7FC3
:10A23000A73EA855816ADDFF3F7762A7FA030FA00A
:10A24000D62BFC55D6008C6AAAF077EA835A15A85B
:10A25000D6FDFF7327D629030F2ADABFC25F650D2B
:10A26000C0A8A60A7FA73EA855816ADDFF3F776296
:10A27000A73EF0A05AF67327D609E00FAA65CF755E
:10A280003AF000762A56F67305A82A3C57F65C0188
:10A290000A80963D57F65C27A0A0AA65FFFF738150
:10A2A0000A806A5DA502FF7365CF0511D6973E68E7
:10A2B000017C85D62B6ACDAB7CC397CA3C6865A36D
:10A2C00036CF23161150D6D0F7A826A36255F680B4
:10A2D000F0DFFFF7A8AA26A362553600FF3D8C8267
:10A2E000D6657F8F6A322A569D180CFF205C657FE9
:10A2F0008F6A322A56D983F0DF0362055F69322AFA
:10A300005605F00FA0F65C055F69322A56D900FFAA
:10A31000F07F8A055A7D8F6A322A5627C6F0DF3FC2
:10A320008C2A56F09526A3621511D63DAAC29FDD50
:10A33000A30A08F27C569D0AC05C653D2A0F62F1B3
:10A34000A5DFF50CA2DF650AA2F0D599300E7C6876
:10A35000D5F50CA28356D6A3CCDFA33A68D5E9F78E
:10A36000C0A883569D095FCFF7A8806A5D0F8C3A1D
:10A3700068D5990CFCDFF3A99A8C3A68D579CF7F20
:10A380008FAA806A5D0F8C3A6855E7CF57C3A880C3
:10A390006A5D0F8C3A6855F7FC4FAAF0F3A99A8CC6
:10A3A0003A68D5F5FCD53D02A40A3F9FAAC9A88307
:10A3B00056FC575FDD00A40A3F9FAAC9A883161167
:10A3C00097FD7F932583F6A522DD032ADAFF2B0074
:10A3D0005F0E5A36605D29C273056ADDAF96FD0DCA
:10A3E00029C23702AA829675FF5CD9DF9022A85A4B
:10A3F0004F0AFF2FC25FA96622FFBFAA8AF0FF7330
:10A40000052AA6C287D6FF73A1A298FD3F0711D7E0
:10A41000FF20C26BBDC267DD0300A8D625A32A16A4
:10A42000FFC37F55952202A36AC2DF5F6702A38A3A
:10A43000C53FFC57A909A32AF6FF555DAA023FFCB8
:10A440005729C29830AAC9F8FDF5A72630AA09DF16
:10A450005FD5309A302A16FF75552A9402FF0DA356
:10A4600009A38AFD57D96BFD00A309A3EAFFF5975D
:10A470009A00A326E37D95DAD683DC00A326DC5779
:10A480006509F20D30AA00115A650F829A020FDF9A
:10A49000555DCA8F02205A875A3D2F08DF555DCA85
:10A4A000F3CCA8FE652A2808DF555DCA8DBC028F53
:10A4B0009982F05DD5A5DCC8829AF22F08DF555D40
:10A4C000CA8D003C5827566503F00F8A756255A661
:10A4D00030A8F0875AFF82F05D156859CF568ABCC4
:10A4E000F5A03068D6027F99BD3058D9003FFF8F64
:10A4F000A9F09D2A560111FF55AAFF95306A2DFC3F
:10A5000095307A29309A96FD2FFC95307A298C5E09
:10A51000A926F20D543F80A05A95DDC80DF5C30F52
:10A520001C9F68F5307AA50A0AFF157CA58AC59795
:10A53000AA26F24D3FFC8F83D6A9970263F2F5C09D
:10A5400075AA97C2A0DD0FA05AF0DF0FD629D6A9B1
:10A550009702FD00AA75FDC0C360D529D6A9970250
:10A56000FDC003A83D579D629D7A29FC008AFC73BB
:10A57000D529D6A90FA02AF7602716C8FF73D529B9
:10A58000D62911680D20A7C25C683D770957970945
:10A59000302828E35DFD809AC2D95C683D20A2CDB9
:10A5A000D9A8758BF0D797428AF0DF95C25C20DA84
:10A5B0009CCDF15756F7A909C80D655A3780DC7450
:10A5C0003FD8692A7CA709C855AAF2FDA0D937D07F
:10A5D0008326992A9CCDD97F03001108A22AF00571
:10A5E0005ADDE3DF95423DA022F057563DE095024B
:10A5F000A357A9D0FD63029572430F02A83D57806F
:10A60000AAFD73011157D7F75F5FA28AC53FA00269
:10A61000D5F30F0CA66A593DFFC058A59CCA553DFD
:10A6200026205C752A163FA0028355F67375AAD8BA
:10A630003FA0A2C26BFD3058653F57A7295C3CA0E4
:10A64000A25A23BFC25FF673759AC2D91C032AA00F
:10A650005A977223BFC25FF673759AC2D93CA002A3
:10A660000A6255977223BFC25FF673752AF6032AF2
:10A67000002A56752937F22BFC653F57A7A2CD3D1E
:10A68000C00F0C56A0AA2A56752937F22BFC653F3D
:10A6900057A7FA03FCC0A8AA2A56752937F22BFC43
:10A6A000653F57A73E00DFC0A8AA2A56752937F292
:10A6B0002BFC653F57A700113F0000AA68FF37F247
:10A6C0005969A50054F5C0808AF63F970DAA3D77D9
:10A6D00055950A035B593F0080F0899D575F0EAA8C
:10A6E00095F5030020575535025F2600C855DF0F4A
:10A6F000A65E0A0055FFA7A8F58C5E0A806856651D
:10A7000003007F575A0E3C88669535008C68FF66BB
:10A71000550F3C88B656F5F055A93026008C68FFD9
:10A7200069550FFFCF0C5A9DEAA50055570FC3A8D6
:10A730005E0A0011555A45424F5800574F5734345E
:10A74000333333594F553344494433495434340037
:10A75000494633594F5533444944334E4F5433558A
:10A76000534533454D555A45005448454E3347529D
:10A77000454154334A4F4234343400594F553341E4
:10A780005245334C494B454C5933544845334F4E51
:10A790004C5900504552534F4E33544F3345564554
:10A7A000523353454533544849533400434F4E5375
:10A7B0004944455233594F555253454C46335448FA
:10A7C00045334245535400534F4B4F42414E33574C
:10A7D0004F524C4433504C415945523345564552E3
:10A7E00034005448414E4B5333464F5233504C4142
:10A7F00059494E4733414C4C335448450057415911
:10A80000335448524F5547483433534552494F55B6
:10A81000534C59335448414E4B5300534F525259A5
:10A8200033464F5233544845334C414D4533454EE2
:10A8300044494E47004933414D334A555354334FF1
:10A840005554334F463354494D45334E4F570043CB
:10A85000524541544544334259334C45453357459D
:10A86000424552003544454D4F35003544454D4F26
:10A8700035005354414745333333334A4150414EF9
:10A8800000535441474533333333534F55544850A5
:10A890004F4C4500535441474533333333434849C4
:10A8A0004E410053544147453333333345475950A4
:10A8B0005400535441474533333333414D45524996
:10A8C000434100360035003600350036003500368D
:10A8D000003500535441474533333333434C4541EE
:10A8E0005245440050555348455335004D4F564549
:10A8F000533335004350553342455354004F4B3486
:10A9000034004752454154343434003500505553D7
:10A910004845530035004D4F564553004F464600BD
:10A9200051554954004746580042474D00534F4C3B
:10A930005645004749564555500052455452590016
:10A940004241434B00434F4E54494E5545004E45FE
:10A95000573347414D45000011241FBECFEFD0E1D2
:10A96000DEBFCDBF14BE88E10FB6F89480936000BF
:10A97000109260000FBE11E0A0E0B1E0E2EBFFEE4C
:10A9800002C005900D92A031B107D9F71FE0A0E2F7
:10A99000B1E001C01D92AF3BB107E1F70E94665DD7
:10A9A000882311F40E94335EF894E4EEFCE080E02A
:10A9B00090E020E802C02193019632E08C309307AA
:10A9C000D4F384EE9CE09093F10E8093F00E1092FD
:10A9D000F20EE5EFFEE080E090E003C01082019609
:10A9E0003A9684309105D4F39093230F8093220FED
:10A9F00091E09093150F9093160F9093140F10926F
:10AA0000810015BC8FEF87B984B988E98AB95C9A4F
:10AA10008CE081B98BEF82B91092C60C86E08093EE
:10AA2000C70C109285001092840083E08093890007
:10AA30008DE88093880089E08093810082E0809394
:10AA40006F0082E484BD17BC95BD83E88093B0009D
:10AA50001092B3009093B10081E185B91092DB0CA4
:10AA60001092CA0C1092CB0C1092D60C1092D50CEE
:10AA70001092DA0C1092D90C1092E00C0E944B5DEF
:10AA800080E00E942C5D80FF03C084E00E94295D6D
:10AA90000E94066378940E9405630E9462770C947A
:10AAA000D7770C940000ECE4FCE0C0E2D1E0209108
:10AAB000900F0027A081B181AC0FBD1F1C911283A4
:10AAC000021708F4102F1C93339603950E3190F360
:10AAD0000BE216E01A95F1F70A95D9F7C0E2D1E03A
:10AAE00000EEA02E662778E055D233E23A95F1F7D2
:10AAF0000E94B4553FE03A95F1F700C0AA94A9F03E
:10AB00000000639500000000683029F0C895C895E2
:10AB1000C8950000E9CF662700243EE1C30FD01D91
:10AB20000000000000000000DFCFC895C895C89560
:10AB3000C895C895000000002DD20E94EE6211E079
:10AB40000091C90C01270093C90C2091CA0C002365
:10AB500009F021272093CA0CE1E0E093C80CE2E061
:10AB6000E093360011240895DE01679F00000091F4
:10AB7000D00C1091D10C00581740000D111D180178
:10AB80000CEC14E0000D111D280130E41EE12D91A4
:10AB90002E316FB660FA239FA1010EF4A201040EBC
:10ABA000151EF001F6F0059108B92D91059108B92F
:10ABB000239F059108B92E316FB6059108B908F4A5
:10ABC000A201059108B960FA040E059108B9151E95
:10ABD0001A95059108B9059139F1F00108B91EF7E8
:10ABE00000C0019108B92D910191000008B9239F7F
:10ABF0000191000008B92E316FB660FA019108B9D1
:10AC00000EF0A1010191040E08B9151E00C00191BA
:10AC100008B9000000C0019108B901911A9521F00E
:10AC2000F00108B906F6DDCF08B90027C895000085
:10AC300008B905E00A95F1F7089520E4E091D00CF9
:10AC4000F091D10C8E51829FE00DF11DACECB4E07F
:10AC5000629FA00DB11D002405900D9205900D92EC
:10AC600005900D9205900D9205900D9205900D9214
:10AC700005900D9205900D9205900D9205900D9204
:10AC800005900D9205900D9205900D9205900D92F4
:10AC900005900D9205900D9205900D9205900D92E4
:10ACA00005900D9205900D9205900D9205900D92D4
:10ACB00005900D9205900D9205900D9205900D92C4
:10ACC00005900D9205900D9205900D9205900D92B4
:10ACD00005900D9205900D9205900D9205900D92A4
:10ACE00005900D9205900D9205900D9205900D9294
:10ACF00005900D9205900D9205900D9205900D9284
:10AD000005900D9205900D9205900D9205900D9273
:10AD100005900D9205900D9205900D9205900D9263
:10AD200005900D9205900D9205900D9205900D9253
:10AD300005900D9205900D9205900D9205900D9243
:10AD400005900D9205900D9205900D9205900D9233
:10AD500005900D9205900D92112408950F931F9365
:10AD600095E0899FE8E6F4E0E00DF11D0481828121
:10AD70009381E0E48E9FD0019E9FB00DE091A60CE0
:10AD8000F091A70CEA0FFB1FACECB4E090E4699FD4
:10AD9000A00DB11D1124403051F4A20FB11D822F1E
:10ADA000122F00FF11C0379610E1121B0DC088E072
:10ADB000821B00FD04C0182FE80FF11D05C018E02C
:10ADC000120FE20FF11D3197503031F498E0939F4C
:10ADD000A00DB11D932F06C098E0931B58E0599F1A
:10ADE000E00DF11D11243EEFE89400FD689458E059
:10ADF000591B48E0481B3EF0259123132C931196D4
:10AE00004A95D1F707C02491319723132C931196BB
:10AE10004A95C9F7E10FF11DA80FB11D5A9549F7E1
:10AE200011241F910F910895D857E257F0571857E2
:10AE300028980E949A59E7E1EA95F1F7289A0FD1EC
:10AE4000E0E0F6E0F2D0E0FF32D0E0FF2FC02F9339
:10AE50003F934F935F936F937F938F939F93AF93A2
:10AE6000BF9378941124E091CC0CF091CD0CE115B6
:10AE7000F10509F009950E9417640E945E5D0E9429
:10AE8000655D0E94C7581124E091CE0CF091CF0C63
:10AE9000E115F10509F00995BF91AF919F918F914F
:10AEA0007F916F915F914F913F912F910895EF9313
:10AEB000E091C70CE93EE0F5E930D0F12F923F92E6
:10AEC0004F925F926F927F928F929F92AF92BF92BA
:10AED000CF92DF92EF92FF920F931F932F933F93A6
:10AEE0004F935F936F937F938F939F93AF93BF9392
:10AEF000CF93DF930E945355DF91CF91BF91AF91D4
:10AF00009F918F917F916F915F914F913F912F9181
:10AF10001F910F91FF90EF90DF90CF90BF90AF9077
:10AF20009F908F907F906F905F904F903F902F9069
:10AF3000EF910895FF93EF93EFB7EF93E0918400C3
:10AF4000EE50E13000F0E23000F0E33000F0E430A9
:10AF500000F0E53000F0E63000F0E73000F0E830D7
:10AF600000F0E93000F005D0EF91EFBFEF91FF91D5
:10AF700018950F921F92E8E2FEEA0090C60C000CB2
:10AF80001124E00DF11D05901490F00109951F901A
:10AF90000F90089528980E949A59E5E1EA95F1F7F3
:10AFA000E091C70CEA95E093C70C289A00C0089579
:10AFB00028980E94C159289A0000E1E0F6E035D0B7
:10AFC00047D0089528980E94C159E0EB0000EA9507
:10AFD000E9F700000000289AF6E0E2E026D00895A4
:10AFE00028980E94C159289A0000E3E0FDEF1DD087
:10AFF000E091C70CE53091F4E091C90CE13000001C
:10B00000F091DB0C19F4F091DB0CF195E3E0E093A7
:10B010008900EDE8EF0FE09388000895E3E0E09306
:10B020008900EDE8E093880008950090C70C0A9429
:10B0300010905F0011FC0F2E0092C70C0090C60C00
:10B0400011FC0E2E0092C60CE0E011FCE1E0089528
:10B05000E3E0E0938900EDE8E09388000895E7E0FD
:10B06000E0938900EBE1E093880008950000000080
:10B0700000000000000000000000000000000000D0
:10B0800000000000000000000000000000000000C0
:10B0900000000000000000000000000000000000B0
:10B0A00000000000000000000000000000000000A0
:10B0B0000000000000000000000000000000000090
:10B0C0000000000000000000000000000000000080
:10B0D0000000000000000000000000000000000070
:10B0E0000000000000000000000000000000000060
:10B0F0000000000000000000000000000000000050
:10B1000099277727833008F00895E0E0F9EB660F80
:10B11000771FE60FF71FA591B491E5EFFEE02AE057
:10B12000289FE00DF11DA183B28311240895909111
:10B13000140F9170880F892B8093140F089599270D
:10B140007727E5EFFEE02AE0289FE00DF11D6E3F36
:10B1500031F46091140F6E7F6093140F0BC06F3F3A
:10B1600031F46091140F6E6F6093140F03C074EB91
:10B17000760F75831124089599277727E5EFFEE070
:10B180002AE0289FE00DF11D6083112408950E949C
:10B19000E55F0090F20E002019F4A4EEBCE002C0BE
:10B1A000AAEEBDE021E002260092F20E22E02093FA
:10B1B000F30E2F923F924F925F926F927F928F92F7
:10B1C0009F92AF92BF92CF92DF92EF92FF920F9336
:10B1D0001F93CF93DF935091130F6091150F7091D0
:10B1E000160F8091170F2090F60E3090F70E4090BA
:10B1F000F90E5090FA0E6090F80E1091F50E7090C6
:10B20000000F8090010F9090020FA090030FB0905C
:10B21000040F2091FF0EC0900A0FD0900B0FE0900A
:10B220000D0FF0900E0F00910C0F3091090F9FEF52
:10B23000620C431CF2014491410300240008C12D1B
:10B24000D02D970CA81CF50144914203002400085E
:10B25000C10DD01D0C0DED1CF701449143030024DA
:10B260000008C10DD01D8A956AF44091140F842FF7
:10B270008695062E0694062600FA7695679576F949
:10B2800040FF66F940E860FD4FE7450300240008F1
:10B29000C10DD01D0024C038D0050CF0CFE70A94B2
:10B2A000C038D0050CF4C0E8C058CD939A9509F089
:10B2B000BFCF4091F30E4A954093F30E97E009F00B
:10B2C000B7CF6092F80E4092F90E9092020FA092C2
:10B2D000030F00930C0FE0920D0F6093150F709306
:10B2E000160F8093170FDF91CF911F910F91FF9051
:10B2F000EF90DF90CF90BF90AF909F908F907F9016
:10B300006F905F904F903F902F900895E091F00ED6
:10B31000F091F10E019100000093B3000EE0E03FC8
:10B32000F00704EE1CE008F0F801E093F00EF09353
:10B33000F10E08950C949C590C949E590F931F93F1
:10B340002F93E091F00EF091F10E01910093B30074
:10B350000EE0E03FF00710F40000000010F0E4EE13
:10B36000FCE0E093F00EF093F10EC895C895C895F7
:10B37000C895C895C895000000002F911F910F91A6
:10B3800008950000E091C70CE0FFD8CFE1E1EA9515
:10B39000F1F7000000000895000000000000000028
:10B3A000000000000000000000000000000000009D
:10B3B000000000000000000000000000000000008D
:10B3C000000000000000000000000000000000007D
:10B3D000000000000000000000000000000000006D
:10B3E000000000000000000000000000000000005D
:10B3F000000000000000000000000000000000004D
:10B40000808182838485868788898A8B8C8D8E8FC4
:10B41000909192939495969798999A9B9C9D9E9FB4
:10B42000A0A1A2A3A4A5A6A7A8A9AAABACADAEAFA4
:10B43000B0B1B2B3B4B5B6B7B8B9BABBBCBDBEBF94
:10B44000C0C1C2C3C4C5C6C7C8C9CACBCCCDCECF84
:10B45000D0D1D2D3D4D5D6D7D8D9DADBDCDDDEDF74
:10B46000E0E1E2E3E4E5E6E7E8E9EAEBECEDEEEF64
:10B47000F0F1F2F3F4F5F6F7F8F9FAFBFCFDFEFF54
:10B48000000102030405060708090A0B0C0D0E0F44
:10B49000101112131415161718191A1B1C1D1E1F34
:10B4A000202122232425262728292A2B2C2D2E2F24
:10B4B000303132333435363738393A3B3C3D3E3F14
:10B4C000404142434445464748494A4B4C4D4E4F04
:10B4D000505152535455565758595A5B5C5D5E5FF4
:10B4E000606162636465666768696A6B6C6D6E6FE4
:10B4F000707172737475767778797A7B7C7D7E7FD4
:10B5000000020406080A0C0E10121416181A1C1E4B
:10B5100020222426282A2C2E30323436383A3C3E3B
:10B5200040424446484A4C4E50525456585A5C5E2B
:10B5300060626466686A6C6E70727476787A7C7E1B
:10B540007F7D7B79777573716F6D6B6967656361FB
:10B550005F5D5B59575553514F4D4B4947454341EB
:10B560003F3D3B39373533312F2D2B2927252321DB
:10B570001F1D1B19171513110F0D0B0907050301CB
:10B58000FFFDFBF9F7F5F3F1EFEDEBE9E7E5E3E1BB
:10B59000DFDDDBD9D7D5D3D1CFCDCBC9C7C5C3C1AB
:10B5A000BFBDBBB9B7B5B3B1AFADABA9A7A5A3A19B
:10B5B0009F9D9B99979593918F8D8B89878583818B
:10B5C00080828486888A8C8E90929496989A9C9E8B
:10B5D000A0A2A4A6A8AAACAEB0B2B4B6B8BABCBE7B
:10B5E000C0C2C4C6C8CACCCED0D2D4D6D8DADCDE6B
:10B5F000E0E2E4E6E8EAECEEF0F2F4F6F8FAFCFE5B
:10B600007F7F7F7F7F7F7F7F7F7F7F7F7F7F7F7F4A
:10B610007F7F7F7F7F7F7F7F7F7F7F7F7F7F7F7F3A
:10B620007F7F7F7F7F7F7F7F7F7F7F7F7F7F7F7F2A
:10B630007F7F7F7F7F7F7F7F7F7F7F7F7F7F7F7F1A
:10B640007F7F7F7F7F7F7F7F7F7F7F7F7F7F7F7F0A
:10B650007F7F7F7F7F7F7F7F7F7F7F7F7F7F7F7FFA
:10B660007F7F7F7F7F7F7F7F7F7F7F7F7F7F7F7FEA
:10B670007F7F7F7F7F7F7F7F7F7F7F7F7F7F7F7FDA
:10B6800080808080808080808080808080808080BA
:10B6900080808080808080808080808080808080AA
:10B6A000808080808080808080808080808080809A
:10B6B000808080808080808080808080808080808A
:10B6C000808080808080808080808080808080807A
:10B6D000808080808080808080808080808080806A
:10B6E000808080808080808080808080808080805A
:10B6F000808080808080808080808080808080804A
:10B700007F7F7F7F7F7F7F7F7F7F7F7F7F7F7F7F49
:10B710007F7F7F7F7F7F7F7F7F7F7F7F7F7F7F7F39
:10B720007F7F7F7F7F7F7F7F7F7F7F7F7F7F7F7F29
:10B730007F7F7F7F7F7F7F7F7F7F7F7F7F7F7F7F19
:10B740007F7F7F7F7F7F7F7F7F7F7F7F7F7F7F7F09
:10B750007F7F7F7F7F7F7F7F7F7F7F7F7F7F7F7FF9
:10B760007F7F7F7F7F7F7F7F7F7F7F7F7F7F7F7FE9
:10B770007F7F7F7F7F7F7F7F7F7F7F7F7F7F7F7FD9
:10B780007F7F7F7F7F7F7F7F7F7F7F7F7F7F7F7FC9
:10B790007F7F7F7F7F7F7F7F7F7F7F7F7F7F7F7FB9
:10B7A0007F7F7F7F7F7F7F7F7F7F7F7F7F7F7F7FA9
:10B7B0007F7F7F7F7F7F7F7F7F7F7F7F7F7F7F7F99
:10B7C0008080808080808080808080808080808079
:10B7D0008080808080808080808080808080808069
:10B7E0008080808080808080808080808080808059
:10B7F0008080808080808080808080808080808049
:10B800000309131E28313A40464C5054585B5E6180
:10B81000636567696B6C6E6F707172737475767740
:10B82000777879797A7A7B7B7C7C7C7D7D7D7E7E66
:10B830007E7E7F7F7F7F7F7F7F7F7F7F7F7F7F7F1A
:10B840007F7F7F7F7F7F7F7F7F7F7F7F7F7E7E7E0B
:10B850007E7D7D7D7C7C7C7B7B7A7A79797877773D
:10B86000767574737271706F6E6C6B696765636106
:10B870005E5B5854504C46403A31281E1309030071
:10B88000C6CCD5DBDFE3E5E7E9EAEBECEDEEEFEF85
:10B89000F0F0F0F1F1F1F1F2F2F2F2F2F2F2F2F391
:10B8A000F3F3F3F3F3F3F3F3F3F3F3F3F3F3F3F368
:10B8B000F3F3F3F3F3F3F3F3F3F3F3F3F3F3F3F358
:10B8C000F3F3F3F3F3F3F3F3F3F3F3F3F3F3F3F348
:10B8D000F3F3F3F3F3F3F3F3F3F3F3F3F3F3F3F338
:10B8E000F2F2F2F2F2F2F2F2F1F1F1F1F0F0F0EF45
:10B8F000EFEEEDECEBEAE9E7E5E3DFDBD5CCC60004
:10B9000022002400260028002B002D0030003300E8
:10B91000360039003D004000440048004C00510012
:10B9200056005B00600066006C00730079008100C7
:10B93000880090009900A200AC00B600C100CC00C5
:10B94000D800E500F300010110012101320144019A
:10B9500057016C0181019801B001CA01E5010202A1
:10B960002102410264028802AE02D70203033003BF
:10B9700061039403CB03050442048304C704100548
:10B980005D05AF0505066106C20629079607090889
:10B99000830805098E09200ABA0A5D0B0A0CC10C3E
:10B9A000840D510E2B0F121007110A121D13401493
:10B9B0007415BA1614188319071BA31C571E2420CC
:10B9C0000E22142439267F28E82A752D29300633C3
:10B9D0000F364539AD3C49401B442848734CFE5056
:10B9E000CF55EA5A51600C661D6C8B725A79928061
:10B9F00037885090E598FDA19FABD3B5A3C0000058
:10BA00008093A60C9093A70C0895E8E4F3E0A0E2DD
:10BA1000B1E06EE16D933197E9F71124089599270C
:10BA200077272EE1629F080E191EA0E2B1E0A00D5B
:10BA3000B11D425E4C93112408958093D00C9093D5
:10BA4000D10C08958091C80C089511241092C80C4F
:10BA500008958093DB0C0895882329F48091D30CFA
:10BA60009091D40C08958091D70C9091D80C0895A2
:10BA7000F999FECF92BD81BD60BDF894FA9AF99A0A
:10BA800078940895F999FECF92BD81BDF894F89A03
:10BA900080B578940895129A129880E090E020E0A2
:10BAA000969587951398009B9068139A2F5F203185
:10BAB000B9F79093D40C8093D30C08958091000132
:10BAC000882311F00E944B5D089508951F9380E034
:10BAD00090E00E94425D182F81E090E00E94425D5C
:10BAE00090E0382F20E0210F311D2A55354509F40B
:10BAF00091E0892F1F910895A0E0B0E0E2E8FDE514
:10BB00000C94A9776C01062FB72E0E94665D8823DE
:10BB1000F1F18FEFC8168FEFD80611F481E03AC02B
:10BB2000EE24FF24C7010E94425D182FC701019631
:10BB30000E94425DD82FC0E0CE01810F911D8C156F
:10BB40009D0521F4E114F10459F423C080E290E052
:10BB5000E80EF91E90E0E91694E0F90619F719C00D
:10BB6000802F9B2D9C01E90140E2C42ED12CC20EF6
:10BB7000D31E87010F5F1F4FC7010E94425D89934B
:10BB8000CC15DD0511F480E005C07801F2CF84E02A
:10BB900001C083E0CDB7DEB7E9E00C94C577A0E043
:10BBA000B0E0E5EDFDE50C94A9776C010E94665DBF
:10BBB000882311F484E04EC0F60180819181FFEF6B
:10BBC0008F3F9F0709F445C08A55954509F441C048
:10BBD00002E010E060E4E62EF12CC7010E94425D15
:10BBE000B82EC70101960E94425DD82FC0E09E0189
:10BBF0002B0D311DF601808191812817390719F429
:10BC00001123B1F00EC02F5F3F4F19F4112309F437
:10BC1000102F0F5F80E290E0E80EF91E0034E9F685
:10BC20001EC0E12EFF2455E0EE0CFF1C5A95E1F7F3
:10BC3000C0E0D0E0F601EC0FFD1FCE018E0D9F1D80
:10BC400060810E94385D2196C032D10599F780E06D
:10BC500001C081E0CDB7DEB7E9E00C94C5771123D0
:10BC600001F782E0F7CFCF93DF93C0E0D0E0FE0191
:10BC7000E059FF4FE491CE016E2F0E94385D21966E
:10BC8000C531D105A1F7C0E4D0E0CE016FEF0E942D
:10BC9000385DCE0101966FEF0E94385DA09688E076
:10BCA000C030D80791F7DF91CF91089590E026E159
:10BCB00030E0829FF001839FF00D929FF00D1124E0
:10BCC000EA5DF04F628708956093140F089590E045
:10BCD00026E130E0829FF001839FF00D929FF00DEE
:10BCE0001124EA5DF04F13861182089590E026E159
:10BCF00030E0829FF001839FF00D929FF00D1124A0
:10BD0000EA5DF04F81E0838B089590E026E130E01A
:10BD1000829FF001839FF00D929FF00D1124EA5D48
:10BD2000F04F6187089590E026E130E0829FF001B6
:10BD3000839FF00D929FF00D1124EA5DF04F648314
:10BD4000089590E026E130E0829FF001839FF00D9E
:10BD5000929FF00D1124EA5DF04F65830895909352
:10BD6000810F8093800F8FE68093860F1092E30CF3
:10BD7000E6E2FFE021E08FEF98E1208310868683E2
:10BD8000878314861182958376963FE0EE37F3071A
:10BD9000A1F708951092270F10923D0F1092530FA4
:10BDA0001092690F019690938A0F8093890F909358
:10BDB000250F8093240F90938D0F80938C0F1092FA
:10BDC000880F1092870F10927F0F10927E0F1092A3
:10BDD000820F81E08093E30C1092850F1092840F04
:10BDE00008958091300F87FD03C08AEF8093300F54
:10BDF0008091460F87FD03C08AEF8093460F8091A4
:10BE00005C0F87FD03C08AEF80935C0F8091720FF7
:10BE100087FD03C08AEF8093720F1092E30C0895A0
:10BE2000DC01ED91FC911197AF014F5F5F4F1196CF
:10BE30005C934E93E4912E2F30E0E7FF13C02F77F1
:10BE400030703695322F222737952795FA014F5FAC
:10BE50005F4FE4918E2F8F77280F311DE7FDF1CFD3
:10BE60004D935C93C90108958093860F08950E94B5
:10BE70009F580895EF92FF920F931F93CF93DF93F4
:10BE8000182F062FF42EE22EC82FD0E086E190E086
:10BE9000C89FF001C99FF00DD89FF00D1124EA5DF5
:10BEA000F04F8385882321F08181882309F088C0A1
:10BEB000EE2091F486E190E0C89FF001C99FF00D5B
:10BEC000D89FF00D1124EA5DF04F138A82858823F4
:10BED00009F076C0108674C0133059F481E091E007
:10BEE0009093160F8093150F81E08093140F0F2D00
:10BEF00008C0812F60E00E949F58812F6F2D0E9403
:10BF000080580F3799F486E190E0C89FF001C99FEF
:10BF1000F00DD89FF00D1124EA5DF04F8091830F52
:10BF2000878784E89FE0958B848B30C089E0089FE9
:10BF3000C0011124E091800FF091810FE80FF91FEB
:10BF40003396459154914115510571F486E190E085
:10BF5000C89FF001C99FF00DD89FF00D1124EA5D34
:10BF6000F04F158A148A12C0FA01249186E190E0FC
:10BF7000C89FF001C99FF00DD89FF00D1124EA5D14
:10BF8000F04F27874F5F5F4F558B448B86E190E0E2
:10BF9000C89FF001C99FF00DD89FF00D1124EA5DF4
:10BFA000F04F108A1286048711829FEF9187E086F6
:10BFB000F282118A81E08387138A128A148296831F
:10BFC000CDB7DEB7E6E00C94C877CF92DF92FF9250
:10BFD0000F931F93CF93DF93EFE2FFE08181282F30
:10BFE000332727FD30958081280F311D2F3F3105E4
:10BFF00019F014F02FEF30E0C90137FF02C080E0E4
:10C0000090E0808376964FE0E738F40739F7809127
:10C01000E30C882309F028C144C1E091890FF09115
:10C020008A0F9F012F5F3F4F30938A0F2093890F14
:10C0300044914F3F69F5A9014F5F5F4F50938A0FBD
:10C040004093890FF90184918F3219F41092E30C17
:10C0500019C1863009F0FBC0FA013196CF01019673
:10C0600090938A0F8093890FE491E33529F490939C
:10C070008D0F80938C0FEBC0E53409F0E8C0809100
:10C080008C0F90918D0F90938A0F8093890FDFC052
:10C0900047FF02C04093820F542F5F70842F90E0BF
:10C0A000807F9070803B910531F1803C910581F15A
:10C0B0008039910509F043C0C9010196F901449105
:10C0C000019690938A0F8093890F0197FC01249128
:10C0D000852F90E08C9FF0018D9FF00D9C9FF00DBF
:10C0E0001124EA5DF04F8081882309F4B0C0220F4B
:10C0F000852F648553C0C9010196F90144910196C9
:10C1000090938A0F8093890F0197FC01249153C06B
:10C110002F5F3F4F30938A0F2093890F215030407B
:10C12000F9012491852F90E08C9FF0018D9FF00DF7
:10C130009C9FF00D1124EA5DF04F248788C0809108
:10C14000820F582F5F7090E0807F9070803B910548
:10C1500041F1803C910509F46EC08039910509F0E8
:10C1600076C02F5F3F4F30938A0F2093890F215065
:10C170003040F9012491852F90E08C9FD0018D9F54
:10C18000B00D9C9FB00D1124AA5DB04F8C918823F7
:10C1900009F45DC0220F852F1C966C910E943A5FB6
:10C1A00056C02F5F3F4F30938A0F2093890F215045
:10C1B0003040F9012491473071F4852F90E08C9F35
:10C1C000F0018D9FF00D9C9FF00D1124EA5DF04F62
:10C1D000220F27833CC04B3071F4852F90E08C9F59
:10C1E000F0018D9FF00D9C9FF00D1124EA5DF04F42
:10C1F000220F26832CC04C3571F4852F90E08C9F44
:10C20000F0018D9FF00D9C9FF00D1124EA5DF04F21
:10C21000220F24831CC04436D1F4852F90E08C9FDC
:10C22000F0018D9FF00D9C9FF00D1124EA5DF04F01
:10C23000220F25830CC0852F90E08C9FF0018D9FED
:10C24000F00D9C9FF00D1124EA5DF04F448789E8C2
:10C250009FE00E94105F9093880F8093870F109249
:10C260007F0F10927E0F02C0C6E1D0E060917E0F7A
:10C2700070917F0F8091870F9091880F68177907D1
:10C2800009F4CBCE6F5F7F4F70937F0F60937E0F6B
:10C290008091840F9091850F01969093850F8093E4
:10C2A000840F05EF1EE0C7E2DFE0FF24BFEFCB2ED7
:10C2B000D12C8A89882309F05EC08B899C89892BBF
:10C2C00009F456C09F858E85981708F04CC050C061
:10C2D0008B852B893C898F37E9F4D9018D91BC8BF3
:10C2E000AB8B8F3F01F1F90161811196BC8BAB8B58
:10C2F000E82FF0E0EE0FFF1FEB57FF4F0190F081AA
:10C30000E02D8F2D0995EB89FC8981918E87FC8B1F
:10C31000EB8B28C0A9014F5F5F4F5C8B4B8BF90102
:10C3200084918F3F21F418821C8A1B8A21C04F5FA1
:10C330005F4F5C8B4B8B41505040FA01649190E011
:10C34000880F991F8B579F4FFC01259134918F2D9A
:10C35000F9010995EB89FC893196FC8BEB8B3197C0
:10C36000E491EE871F869F858E85981709F4B0CFDC
:10C370008F858F5F8F878A85882319F420E030E0CE
:10C380006BC088898F3F11F08F5F888B9F819923C5
:10C3900009F45CC02885222309F458C08E818823C3
:10C3A00009F454C04091860F442309F44FC0899F7B
:10C3B000C001112480509F4F892F992730E0B90187
:10C3C000869F9001879F300D969F300D112420503D
:10C3D0003F4F232F33278D8190E0FC012E9FC0011A
:10C3E0002F9F900D3E9F900D112480509F4F892FBD
:10C3F0009927242F30E0AC01429FC001439F900D4C
:10C40000529F900D112480509F4F292F33278B81ED
:10C410008823F1F0EA81F0E0E050FC44E491E05838
:10C42000E89FC001112480509F4F892F9927B601A2
:10C43000681B790B629FC001639F900D729F900DE6
:10C44000112480509F4F292F332702C020E030E075
:10C450008A819C81890F8A83F8012083F394065F87
:10C460001F4F6696F4E0FF1609F023CFDF91CF91BE
:10C470001F910F91FF90DF90CF9008951F93CF935E
:10C48000DF93582F89E0589FC00111242091800F1D
:10C490003091810F280F391FC9010396FC01A59126
:10C4A000B491F90184918150823010F413E01DC0E1
:10C4B00080913D0F8823B1F08091490F851711F4C9
:10C4C000442381F48091530F882371F080915F0F92
:10C4D000851711F4442341F490914D0F8091630F1F
:10C4E000891710F411E001C012E0212F30E0FD01A6
:10C4F000449186E190E0289FE001299FD00D389F6C
:10C50000D00D1124CA5DD04F4F871196BD8BAC8BD7
:10C51000188A80E58A8368878FEF89871A861B8A45
:10C52000198A21E02B871A8A5D8729831C828E83D2
:10C53000133049F481E091E09093160F8093150F2A
:10C540002093140F08C0812F60E50E948058812F2E
:10C550006A890E949F58DF91CF911F910895FF92A1
:10C560000F931F93082FF62E0E94805810E086E14B
:10C5700090E0089FF001099FF00D189FF00D112425
:10C58000EA5DF04FF2821F910F91FF900895962F70
:10C59000482F50E026E130E0429FF001439FF00D2C
:10C5A000529FF00D1124EA5DF04F6281691B628396
:10C5B0000E9480580895482F50E026E130E0429FC5
:10C5C000F001439FF00D529FF00D1124EA5DF04FF2
:10C5D0009281690F62830E94805808953091900F74
:10C5E00020E010C0822F90E0FC01EE0FFF1FE80F4B
:10C5F000F91FE45BF34FA081B181A05EBE4F828141
:10C600008C932F5F231770F308950895E8E6F4E004
:10C6100080EF8083359694E0EC3CF907D1F70895DC
:10C6200080938E0F1092920F81E08093910F66237A
:10C6300021F08091910F8823E1F70895982F8823A6
:10C6400019F48FEF87B9089581E08093930F809359
:10C650008F0F892F0E9410630895982F882311F45B
:10C6600017B808958CE08093930F8FEF80938F0F0E
:10C67000892F0E94106308958091910F8823F9F00B
:10C680008091920F8823C1F480918E0F8093920F36
:10C690009091930FE92FF0E0EF5FFE4F808187B913
:10C6A00080918F0F890F8093930F882311F08D3025
:10C6B00031F41092910F089581508093920F089554
:10C6C0000F931F93CF93DF938C01C0E0D0E007C09E
:10C6D0000E94225D8823E1F30E94255D2196C01708
:10C6E000D107B4F3DF91CF911F910F910895A3E08B
:10C6F000B0E0EDE7F3E60C94A0771092900F8091F4
:10C700000101882309F48FC0A8E68A2EA4E09A2E9E
:10C710007724F4018081803F09F47AC09181F82F59
:10C72000F695F695F695F983282F277019F0F2E023
:10C730002F2E02C022242394392F36953695369514
:10C74000892F877019F0E2E06E2E02C06624639490
:10C75000B82EAA242501420E511CC32EEE24FF241C
:10C760004DC02BE12C1510F09C2D01C0932D4DE1F7
:10C770004D1510F08D2D02C08D2D8E51EEE19E9F36
:10C7800090011124280F311D8901005E1E4FF80110
:10C7900060816E31F0F04091900F4E3100F5842FA2
:10C7A00090E0FC01EE0FFF1FE80FF91FE45BF34F71
:10C7B000318320836283862F642F0E941D566091EF
:10C7C000900FF80160836F5F6093900F61506E313E
:10C7D00030F4872D4A815B8192010E94AE568A8196
:10C7E0009B8101969B838A83D394821508F4B9CFE9
:10C7F0000894E11CF11CC394E61450F480E09E2DD3
:10C800009C013B832A83D98054EE352E3C0CA9CF62
:10C810007394E5E0F0E08E0E9F1EF4E17F1609F0C0
:10C8200078CF0E94EE622396E2E10C94BC770E94DE
:10C830003C630E9477630895EF920F93CF93DF9349
:10C84000382FEE2DF0E0A6E0EE0FFF1FAA95E1F7DE
:10C85000E556FF4FA22FB0E076E0AA0FBB1F7A95F6
:10C86000E1F7A453BB4FED0190E0849189939F5F62
:10C8700031969034D1F7862F90E0FC0155E0EE0F11
:10C88000FF1F5A95E1F7880F991FE81BF90BE30F7B
:10C89000F11DE05EFE4F2083E42FF0E066E0EE0F36
:10C8A000FF1F6A95E1F7E55EFD4D90E084918013EE
:10C8B0008C939F5F319611969034C1F7DF91CF91A1
:10C8C0000F91EF900895282F30EF0DC0822F90E048
:10C8D000FC01EE0FFF1FEE0FFF1FE80FF91FE859D5
:10C8E000FB4F30832F5F261788F3089590E0835025
:10C8F000823008F491E0892F089590E0843009F4A3
:10C9000091E0892F089590E0853009F491E0892F16
:10C9100008951F93182F0E947664882349F4812F6D
:10C920000E947D64882321F4812F0E94836401C0CA
:10C9300081E01F910895A62FB0E096E0AA0FBB1FDB
:10C940009A95E1F7A453BB4FE82FF0E086E0EE0F95
:10C95000FF1F8A95E1F7E556FF4F90E08C91841711
:10C9600011F484918C939F5F119631969034B1F7B6
:10C970000895DB01FC01E556FF4FA453BB4F03C0F4
:10C9800084918D933196415050408FEF4F3F58071F
:10C99000B9F70895AF92CF92EF92FF920F931F9342
:10C9A000CF93DF93F82E122FA22FB0E096E0AA0FBC
:10C9B000BB1F9A95E1F78EE1689F90011124BA019F
:10C9C000205E3E4FFB018491882389F18F7780524E
:10C9D000E82FFF27E7FDF09586E0EE0FFF1F8A9511
:10C9E000E1F7E55AF34EAD014F5F5F4FED01C453E0
:10C9F000DB4F90E08491801711F4E88205C08C151C
:10CA000011F4A88201C08883DA019F5F31964F5FDD
:10CA10005F4F2196903471F7F901EF0DF11D1083EE
:10CA20001F5FF3946F5F7F4FFDE1FF1558F6812F75
:10CA3000DF91CF911F910F91FF90EF90CF90AF902A
:10CA40000895A0E0B0E0E7E2F5E60C94A977F22EB5
:10CA5000B02EDE2CC22FD0E0B6E0CC0FDD1FBA9591
:10CA6000E1F79EE1699F80011124E42FF52FBF01BA
:10CA70008F5F005E1E4F03C06F5F7F4F8F5FE82E9A
:10CA8000EA94FB0194919333B9F39923C1F1EC2D0E
:10CA9000F0E0E55AFB4CC3945491F3E0FC1508F424
:10CAA000CC249F779052E92FFF27E7FDF095A6E071
:10CAB000EE0FFF1FAA95E1F7E55AF34E9E012F5F97
:10CAC0003F4FDE01A453BB4F40E094919B1511F4FE
:10CAD000DC9205C09F3F11F45C9301C09C93E90177
:10CAE0004F5F31962F5F3F4F1196403471F7F80139
:10CAF000EE0DF11DF082F3948E3108F4BDCF8F2D31
:10CB0000CDB7DEB7E9E00C94C5778091970F83FD30
:10CB100003C080E090E008958091950F9091960F6A
:10CB200023E0969587952A95E1F780958170089581
:10CB30008091970F82FD03C080E090E0089580917E
:10CB4000950F9091960F96958795969587958095D8
:10CB5000817008958091970F84FD03C080E090E07C
:10CB600008958091950F9091960F44E09695879542
:10CB70004A95E1F78095817008958091970F85FD22
:10CB800003C080E090E008958091950F9091960FFA
:10CB900055E0969587955A95E1F7809581700895AF
:10CBA0008091970F86FD03C080E090E0089580910A
:10CBB000950F9091960F66E0969587956A95E1F7A7
:10CBC0008095817008958091970F87FD03C080E064
:10CBD00090E008958091950F9091960F880F892F7E
:10CBE000881F990B919580958170089570E090E071
:10CBF000880F991FFB01B6E0EE0FFF1FBA95E1F712
:10CC0000660F771F660F771FE61BF70BE80FF91FFC
:10CC1000E05EFE4F90819E51969596958091AD0F66
:10CC20002AEF3FEF829F802D1124890F0895A0E005
:10CC3000B0E0EDE1F6E60C94A477182FC62EA42EF2
:10CC4000622E80E49FE160E876E040E051E00E94DF
:10CC5000B9644EE1742EC79C60011124C10ED11C31
:10CC600030E2832E31E0932E7401EC0CFD1CF701B1
:10CC70000083102F1F5F8091A40F602F40E00E945F
:10CC80009B64BB24EA0CFB1CF70110830E5F8091B0
:10CC9000A50F612F40E00E949B64679CE001112476
:10CCA000CC0DDD1DC80DD91D08831E5F8091A60F18
:10CCB000602F40E00E949B64CA0DDB1D18838091A9
:10CCC000A70F612F40E00E949B64CDB7DEB7EEE076
:10CCD0000C94C077FF920F931F93CF93DF93F82E9E
:10CCE00010E0A6E0000F111FAA95E1F7862FC0E023
:10CCF000D0E070E0620F711DAF2DB0E0A40FB11D48
:10CD00000BC0E40FF51FC08321969F5FE92FF0E071
:10CD1000EA17FB07B4F38F5F282F30E02617370799
:10CD200084F4A901F5E0440F551FFA95E1F7220FAD
:10CD3000331F421B530B400F511F9F2D405E5E4F10
:10CD4000E5CFCDB7DEB7E5E00C94C97770E0FB0125
:10CD500096E0EE0FFF1F9A95E1F7660F771F660FBB
:10CD6000771FE61BF70B90E0880F991FE80FF91F5C
:10CD7000440F440F8091AD0F28E1829FC001112420
:10CD8000825E840FE05EFE4F80838F5F81838F5FC2
:10CD9000868F8F5F878F0895AF92BF92CF92DF9279
:10CDA000EF92FF920F931F93F090B90F00919D0F98
:10CDB000A090A30FBA2CA0FE1BC0002309F4B3C09F
:10CDC000C02ECA948F2D6C2D0E94F665E82E01307E
:10CDD00039F0602F62508F2D0E94F665182F06C023
:10CDE0000E947664882309F09EC011E002501FC0A3
:10CDF000A1FE1FC00D3009F496C0C02EC3948F2D24
:10CE00006C2D0E94F665E82E0A3111F411E00EC077
:10CE1000602F6E5F8F2D0E94F665182F0C3031F455
:10CE20008E2D0E947664882309F07DC00E5FDF2C72
:10CE300040C0A2FE1DC0FF2009F475C0DF2CDA94AB
:10CE40008D2D602F0E94F665E82E81E0F81639F0EE
:10CE50008F2D8250602F0E94F665182F07C08E2DEF
:10CE60000E947664882309F05EC011E08EEF1FC037
:10CE70008EE0F81609F457C0DF2CD3948D2D602F67
:10CE80000E94F665E82E8CE1F81611F411E00EC050
:10CE90008F2D8E5F602F0E94F665182F8DE0F8169B
:10CEA00029F48E2D0E9476648823E9F582E0F80E3D
:10CEB000C02E8E2D0E947664882341F1812F0E941E
:10CEC0008964882381F58E2D0E947D64882359F022
:10CED0008D2D6C2D42E00E94A6668091AE0F8F5F73
:10CEE0008093AE0F05C08D2D6C2D41E00E94A6668B
:10CEF000D0929C0FC092B20FF092B70F0093BA0F6E
:10CF00008091A30F80628093A30F05C08E2D0E9495
:10CF10008964882311F481E007C0B5FE04C080E273
:10CF2000A826A092A30F80E01F910F91FF90EF9091
:10CF3000DF90CF90BF90AF900895582F3091A00F01
:10CF4000343110F080E00895832F90E0FC01EE0F63
:10CF5000FF1FEE0FFF1FE80FF91FE859FB4F50832B
:10CF600061834283138224833F5F3093A00F81E06B
:10CF70000895A0E0B0E0EFEBF7E60C94A977C82E97
:10CF8000E62E9091AD0F85E0489FA0011124FA0193
:10CF9000E252FC49E4918A0106521C49CE2FD0E0AE
:10CFA000CC0FDD1FCC0FDD1FC15DDB49FF2484E208
:10CFB000989FD02C1124E8E0BE2EBC0C02C088E063
:10CFC000E80EF8014491FE0184914D0D20E081119D
:10CFD00021E08C2D6E2D0E949D670F5F1F4FF80181
:10CFE0004491015010402196FE01849121974D0DEE
:10CFF00020E0811121E08B2D6E2D0E949D67F3941E
:10D000000E5F1F4F2296F2E0FF16C9F6CDB7DEB7CE
:10D01000E9E00C94C5770F931F938091940F8823B8
:10D0200009F04BC08091A30F282F20FF06C010915C
:10D03000B30F119500E091E013C021FF05C01091DE
:10D04000B30F00E095E00CC08091B30F22FF05C044
:10D05000082F019510E099E003C0082F10E09DE033
:10D060004091BC0F490F25FD4E5F1092A00F80919B
:10D07000B90F8295807F60919D0F6295607F610FEF
:10D08000800F0E94B96790919C0F9F3F69F0929525
:10D09000907F8091B20F8295807F180F802F890F2B
:10D0A000612F40E00E94B9678091A00F64E10E9467
:10D0B000636481E090E00E9460631F910F91089586
:10D0C000EF92FF920F931F93F82E81E090E00E9461
:10D0D0006063E090AD0F00E020C0E092AD0F812FC3
:10D0E000602F0E94F665482FF092AD0F812F602FC0
:10D0F0000E94A6661F5F1F3081F780919D0F081761
:10D1000029F40E940B6881E090E002C082E090E088
:10D110000E9460630F5F0E3011F010E0DECFF092DE
:10D12000AD0F1F910F91FF90EF9008959091AD0F6B
:10D1300088E1989F90011124225E3F4FE0E2F1E0E8
:10D140009081892F8E51883710F4921B90833196ED
:10D1500084E0E836F807A1F781E090E00E94606380
:10D1600008959091AD0F88E1989FF0011124A6E0F9
:10D17000EE0FFF1FAA95E1F7E556FF4FACECB4E0C8
:10D1800084918D9331968AE0AC3CB807C9F781E071
:10D1900090E00E9460630895A0E0B0E0E2EDF8E660
:10D1A0000C94A877182FD62EA42EB22EC02E0E9433
:10D1B000B1680E949668A12FB0E093E0AA0FBB1F50
:10D1C0009A95E1F741C0FE018491E82EFF248B017E
:10D1D00083E0000F111F8A95E1F740E050E0C7019E
:10D1E000042E02C0959587950A94E2F780FF15C03A
:10D1F0009A01200F311F80E090E024533B4FFC0147
:10D20000689415F8EE0FFF1F1694E1F7E20FF31F75
:10D21000108201968831910591F74F5F5F4F48303A
:10D220005105E9F66F5F7F4F21966830710559F619
:10D23000ED012896BB2011F0ED0128978A2D90E092
:10D240000E946063DA94DE01DD2031F0ED01C65208
:10D25000DB4C60E070E0B7CFCC2021F08C2D90E06B
:10D260000E946063CDB7DEB7EAE00C94C477EF921A
:10D270000F93DF93CF9300D000D000D0CDB7DEB7AF
:10D2800081E090E00E94606380E064E10E9463645A
:10D290000E94B1680E9496689091A80F86E0989FBE
:10D2A000F0011124E856FB4CDE0111969E01295F26
:10D2B0003F4F84918D933196A217B307D1F781E048
:10D2C00090E00E94606320E08C81811121E090E079
:10D2D0008E81811191E089816A814B810D81E92ED6
:10D2E0000E94CC688091A80F8F5F8093A80F8B302D
:10D2F00010F01092A80F26960FB6F894DEBF0FBE5E
:10D30000CDBFCF91DF910F91EF9008951092BD0F97
:10D3100081E08093940F8093B80F0E94376981E079
:10D3200090E00E94606381E00895FF920F931F9345
:10D33000F82E00E00CC0802F612F4F2D50E00E948E
:10D340000F5D1F5F1C31B9F70F5F0E3111F010E058
:10D35000F2CF1F910F91FF900895A0E0B0E0E3EBB2
:10D36000F9E60C94A477982EA62E142F022FC62E21
:10D37000DD24682E7724C601880F991F960165E089
:10D38000220F331F6A95E1F7281B390B260D371D35
:10D39000F901E05EFE4FE081EE51E83710F0E13830
:10D3A00011F4E093A40FC12FD0E0F901E05EFE4F2D
:10D3B000EC0FFD1FE081EE51E83710F0E13811F479
:10D3C000E093A50FE02EFF24C701880F991FD70116
:10D3D00045E0AA0FBB1F4A95E1F7A81BB90BA20FA6
:10D3E000B31FFD01E05EFE4FE081EE51E83710F023
:10D3F000E13811F4E093A60FA05EBE4FAC0FBD1F45
:10D40000EC91EE51E83710F0E13811F4E093A70FFA
:10D41000892D6A2D4DE750E00E940F5DB12EB90CA9
:10D420008B2D6A2D4EE750E00E940F5D0A0D892D6D
:10D43000602F4FE750E00E940F5D8B2D602F40E87A
:10D4400050E00E940F5D892C8394182D6C0E7D1E78
:10D450000DC0812F6A2D48E750E00E940F5D812F9B
:10D46000602F49E750E00E940F5D1F5F812F90E021
:10D470008615970574F30A2D0F5F102FE701CC0D69
:10D48000DD1D0DC0892D612F4AE750E00E940F5D20
:10D490008B2D612F4BE750E00E940F5D1F5F812FA6
:10D4A00090E08C179D0774F30DC0812F602F42E828
:10D4B00050E00E940F5D1F5F812F90E08615970559
:10D4C000A4F30F5F802F90E08C179D0714F4182DA4
:10D4D000F3CFCDB7DEB7EEE00C94C077A0E0B0E0BC
:10D4E000E4E7FAE60C94A377C82ED62E742E622EAB
:10D4F000E8015E2CE02EF02E11E0842E9924AA245F
:10D50000BB24AC1ABD0A1FC08C2D6D2D412F21E00C
:10D510000E94AD69552039F08C2D6D2D412F21E0F1
:10D520000AE10E941766D7FF04C0C5010E9460632C
:10D5300009C0FF2031F481E090E00E946063FE2C7E
:10D5400001C0FA941F5F812F90E088169906E4F6D7
:10D55000FE2C11E0862C9924AA24BB24AC1ABD0A07
:10D560001FC08C2D6D2D472D212F0E94AD69552098
:10D5700039F08C2D6D2D472D212F0AE10E94176661
:10D58000D7FF04C0C5010E94606309C0FF2031F4C9
:10D5900081E090E00E946063FE2C01C0FA941F5F5E
:10D5A000812F90E088169906E4F6CDB7DEB7EFE05C
:10D5B0000C94BF770F931F93CF93DF93182F062FF1
:10D5C000EA01FE0144912196442369F0812F1F5FF7
:10D5D0004F774052552747FD509541595F4F602F77
:10D5E0000E940F5DEECFDF91CF911F910F910895B3
:10D5F000CF93DF9383E060E00E941E6382E80E9485
:10D60000956981E090E00E946063C0E0D0E0FE0197
:10D61000E55CF845E4914E2F50E04F775070415B48
:10D620005F4F9E012A5F822F64E00E940F5D88E0B9
:10D6300090E00E9460632196C431D10541F7C0E0BB
:10D64000D0E0FE01E05BF845E4914E2F50E04F77CB
:10D650005070415B5F4F9E012C5F822F65E00E94FE
:10D660000F5D88E090E00E9460632196C831D1058B
:10D6700041F7C0E0D0E0FE01E759F845E4914E2FB4
:10D6800050E04F775070415B5F4F9E01285F822FC3
:10D6900066E00E940F5D88E090E00E946063219642
:10D6A000C131D10541F7C0E0D0E0FE01E558F845B1
:10D6B000E4914E2F50E04F775070415B5F4F9E01D9
:10D6C0002C5F822F68E00E940F5D88E090E00E944E
:10D6D00060632196C731D10541F7C0E0D0E0FE017B
:10D6E000ED56F845E4914E2F50E04F775070415B76
:10D6F0005F4F9E012C5F822F69E00E940F5D88E0E2
:10D7000090E00E9460632196C831D10541F7C0E0E6
:10D71000D0E0FE01E455F845E4914E2F50E04F77FC
:10D720005070415B5F4F9E012D5F822F6CE00E9425
:10D730000F5D88E090E00E9460632196CA31D105B8
:10D7400041F7C0E0D0E0FE01E953F845E4914E2FE7
:10D7500050E04F775070415B5F4F9E012D5F822FED
:10D760006DE00E940F5D88E090E00E94606321966A
:10D77000CA31D10541F78CE390E00E946063C0E0BC
:10D78000D0E0FE01EE51F845E4914E2F50E04F7786
:10D790005070415B5F4F9E012D5F822F6FE00E94B2
:10D7A0000F5D88E090E00E9460632196CA31D10548
:10D7B00041F7C0E0D0E0FE01E350F845E4914E2F80
:10D7C00050E04F775070415B5F4F9E012F5F822F7B
:10D7D00060E10E940F5D88E090E00E946063219606
:10D7E000CD31D10541F7C0E0D0E0FE01E55EF7455F
:10D7F000E4914E2F50E04F775070415B5F4F9E0198
:10D800002D5F822F62E10E940F5D88E090E00E9410
:10D8100060632196C931D10541F7C0E0D0E0FE0137
:10D82000EB5CF745E4914E2F50E04F775070415B31
:10D830005F4F9E012D5F822F63E10E940F5D88E0A4
:10D8400090E00E9460632196C931D10541F784E0E0
:10D8500068E14FE458EA0E94DA6A8FEF90E00E9494
:10D860006063DF91CF910895FF920F931F93CF9341
:10D87000DF93082FF62EEA0183E0483E580714F0A4
:10D88000C7EED3E010E01C161D0614F0112361F45E
:10D89000CE016AE070E00E948D77482F50E04A5731
:10D8A0005F4F802F6F2D04C0802F6F2D42E850E016
:10D8B0000E940F5D1F5F0150143039F0CE016AE005
:10D8C00070E00E948D77EB01DECFCDB7DEB7E5E0EB
:10D8D0000C94C977FF920F931F93082FF62E142FE5
:10D8E000842F6AE00E946D77492F50E04A575F4FBE
:10D8F000802F8F5F6F2D0E940F5D812F6AE00E9445
:10D900006D77882329F4802F6F2D42E850E006C000
:10D91000482F50E04A575F4F802F6F2D0E940F5DB8
:10D920001F910F91FF900895AF92CF92EF920F93B6
:10D930001F9381E80E94956982E060E00E941E6367
:10D9400018E08DE06EE044E357EA26E10FEFE12EA8
:10D95000F0ECCF2EAA240E94CA648AE090E00E94D4
:10D9600060631150153069F78DE290E00E946063AA
:10D9700014E08DE06EE044E357EA26E10FEFE12E7C
:10D98000E0ECCE2EAA240E94CA648AE090E00E94B5
:10D99000606311501E3F69F78CE390E00E94606362
:10D9A00083E061E00E942D6381E060E00E941E63DD
:10D9B0001F910F91EF90CF90AF9008950E94055D59
:10D9C0001092990F1092AA0F81E08093B80F809364
:10D9D000940F1092AD0F8093A90F82E38093AF0F45
:10D9E00080EB96E60E94AF5E8AED96E30E94005DB2
:10D9F0008BE990E00E941D5D80EC0E94345F0E94E4
:10DA0000946C0895EF92FF921F93DF93CF93CDB75D
:10DA1000DEB7A0970FB6F894DEBF0FBECDBF182FAC
:10DA20008EE390E09A8389837E010894E11CF11CC7
:10DA3000B7010E947C5D882319F0C7010E94CF5D69
:10DA4000812F877021E030E002C0220F331F8A95BA
:10DA5000E2F7FE013396169516951695E10FF11D26
:10DA60008081822B8083CE0101960E94CF5DA0969B
:10DA70000FB6F894DEBF0FBECDBFCF91DF911F91DF
:10DA8000FF90EF900895885C0E94026D0895A0E2D7
:10DA9000B0E0EDE4FDE60C94AF77182F8EE390E054
:10DAA0009A838983BE016F5F7F4F0E947C5DFE0178
:10DAB0003396882389F4812F869586958695E80F7D
:10DAC000F11D808190E01770012E02C09595879519
:10DAD0000A94E2F781700BC0CE0181961192E8178B
:10DAE000F907E1F7CE0101960E94CF5D80E0A09694
:10DAF000E3E00C94CB771F9310E0812F0E94476DD9
:10DB0000882321F01F5F1233C1F781E01F91089530
:10DB1000885C0E94476D0895A0E0B0E0E2E9FDE670
:10DB20000C94A877F42E122FC02E1092AA0F1092E8
:10DB3000AC0F1092AB0F10929F0F10929E0F10928D
:10DB4000AE0F1092B30F10929D0F1092B90F8091EB
:10DB5000B00F833318F081E38093B00F8091B00F42
:10DB60000E94476D8093BE0F8091B00F0E94886D18
:10DB70008093A20F8FEF80939C0F82E08093A30F7E
:10DB8000E091B00F81E7E89FF00111245F01089454
:10DB9000A11CB11CE65DF749949180911F0F882369
:10DBA00011F49093AD0F80911D0F8823A9F5EE20FD
:10DBB00099F52091A90F80911E0F882329F080915B
:10DBC000200F8093A90F03C09F5F9093A90F8091AE
:10DBD0000E01882321F08091A90F2817E9F0809188
:10DBE000A90F813019F486E59FE711C0823019F43E
:10DBF00085EB93E80CC0833019F489E89DE807C0F1
:10DC0000843019F488E098E802C08FE794E90E9414
:10DC1000CA5E81E080930E01E12ED12EDF0C44C05C
:10DC2000F02E802F8695CC2039F4FE01E80FF11DEF
:10DC3000E65DF749849106C09E01280F311DC90198
:10DC40000E94425D282F30E0C80181709070880FDB
:10DC5000991F880F991F02C0359527958A95E2F77D
:10DC6000422F4F70463050F0F092B90FE0929D0F66
:10DC7000463011F441E009C042E007C0423029F4C7
:10DC80008091AE0F8F5F8093AE0F8F2D6D2D0E9410
:10DC9000A6660F5F1F4F0F30110509F0C1CFE39447
:10DCA000D3943DE03E1560F0CE2DD0E0A3E0CC0F44
:10DCB000DD1FAA95E1F7CA0DDB1D00E010E0B0CF33
:10DCC000CDB7DEB7EAE00C94C477EF920F9383E010
:10DCD00061E00E942D6381E090E00E94606381E03A
:10DCE00061E040E020E000E0EE24E3940E948C6DCF
:10DCF00081E090E00E9460630E940B6883E060E036
:10DD00000E941E630F91EF9008958091970F90915C
:10DD1000980F9093960F8093950F80E00E942C5D52
:10DD20009093980F8093970F0895CF92EF92FF9260
:10DD30000F931F9381E090E00E94606381E060E0B8
:10DD40000E941E6381E80E94956981E090E00E9434
:10DD50006063F090B00F81E060E040E020E000E020
:10DD6000EE24E3940E948C6D80E060E04DE122E0BF
:10DD700000E010E0EE240E946E6A8091BE0F8823BE
:10DD800029F08AE161E041ED58EA04C08AE161E0EE
:10DD90004FEC58EA0E94DA6A8091A20F882349F07A
:10DDA0008BE161E04DEC58EA0E94DA6ACC241EE176
:10DDB00005C08BE161E04BEC58EAF6CF0E94856E1E
:10DDC0002091970F3091980F32FF10C08091950FDE
:10DDD0009091960F92FD0AC0FF2041F089E08F15C7
:10DDE00010F0FF2445C086EFF80E42C033FF16C086
:10DDF0008091950F9091960F93FD10C04091AF0FB9
:10DE00002F2D30E0842F90E001972817390734F444
:10DE10008AE0F80EF41660F1F42E1EC00E948565AB
:10DE20008823A1F01092940F1092B80FF092B00FC7
:10DE300081E061E040E020E000E0EE240E948C6D93
:10DE40001F910F91FF90EF90CF9008950E94D065A1
:10DE5000882321F0FF2011F0FA940AC00E94E365A4
:10DE6000882309F451C080E38F1508F44DC0F39462
:10DE700080E060E04DE122E00E94AD690E943769D8
:10DE800081E090E00E946063F092B00F81E061E079
:10DE900040E021E000E0EE24E3940E948C6D80E0FD
:10DEA00060E04DE122E00E94AD698091BE0F8823C1
:10DEB00029F08AE161E049EC58EA04C08AE161E0B6
:10DEC00047EC58EA0E94DA6A8091A20F882329F071
:10DED0008BE161E045EC58EA04C08BE161E043EC82
:10DEE00058EA0E94DA6A8091B90F60919D0F70E044
:10DEF000660F771F880F42E022E009E10E946A6600
:10DF000081E090E00E9460631123E1F58091AD0F04
:10DF1000882339F41C2D1F5F86E061E042EB58EA4C
:10DF20001FC0813039F41C2D1F5F86E061E043EA99
:10DF300058EA16C0823039F41C2D1F5F86E061E07C
:10DF400044E958EA0DC01C2D1F5F833029F486E098
:10DF500061E041E858EA04C086E061E042E758EA3F
:10DF60002BE000E0EE240E942165C12E4F2D4F5F73
:10DF70008CE061E00E946A6C83E0811708F4CC2495
:10DF80001EE101C011501092A00F8091B90F609155
:10DF90009D0F1F3010F445E001C046E070E004E042
:10DFA000660F771F0A95E1F78295807F0E94B96717
:10DFB00081E090E00E94606301CFA0E0B0E0E3EE7A
:10DFC000FFE60C94A6770E94F15E8091B90F90E075
:10DFD000E4E0880F991FEA95E1F78093B30F109260
:10DFE000B90F8FEF80939C0F88E08093A30F10925E
:10DFF000940F14E017C08E5F8093B30F8091B40F1D
:10E00000882321F081508093B40F0AC01093B40F7D
:10E0100090E08091BC0F882309F491E09093BC0FAD
:10E020000E940B688091B30F803E28F380E064E18A
:10E030000E9463648CE39EE70E94CA5E10920E0108
:10E040008AE090E00E9460638EE08093B90F86E0E2
:10E0500080939D0F1092B30F84E08093A30F0E94D2
:10E06000376981E090E00E94606381E80E949569D1
:10E0700081E061E00E942D63C0919E0FD0919F0FBF
:10E08000C090AB0FD090AC0F8091B00F0E94307257
:10E0900081E80E94956910920E018091B00F0E9454
:10E0A000026D80919A0F90919B0F8C179D0724F021
:10E0B0008091B00F0E94436D81E061E00E941E6379
:10E0C00089E06FE04BE02AE00EEF1FEFEE240E94A4
:10E0D0006E6A8AE060E146E159EA0E94DA6A80915C
:10E0E0009A0F90919B0F8C179D0734F080E160E1AF
:10E0F00044E159EA0E94DA6A8AE061E14DE059EAB6
:10E100000E94DA6A8091B50F9091B60F8C159D052B
:10E1100034F080E161E14BE059EA0E94DA6A83E180
:10E1200060E1AE010E94346C83E161E1A6010E94CE
:10E13000346C80919A0F90919B0F8C179D0764F01F
:10E140008091B50F9091B60F8C159D052CF08BE04A
:10E1500063E142E059EA04C08DE063E14DEF58EA23
:10E160000E94DA6A8BE065E144EF58EA0E94DA6ABD
:10E170008AE067E14CEE58EA0E94DA6A8AE068E1D8
:10E1800044EE58EA0E94DA6A40919A0F50919B0F30
:10E1900083E167E10E94346C4091B50F5091B60F56
:10E1A00083E168E10E94346C81E090E00E9460634A
:10E1B000D090B00FD3948D2D6AE00E946D77982E89
:10E1C0008D2D0E946D77A92E7DE1F72EBB246FE97E
:10E1D000862E49C0899282E0C63AD807D9F78B2D9E
:10E1E00065E00E946D778F2D6CE043ED58EA20E0EA
:10E1F00000ECEE24C92E0E942165FE01819282E08E
:10E20000E43CF807D9F784E18F15D0F089E08D154B
:10E2100050F48F2D8A5F6CE0492D25E100EC51E828
:10E22000E52E0E941C648F2D895F6CE04A2D24E14D
:10E2300000EC31E8E32E0E941C6487E08F1508F49F
:10E24000FA9410E00E94856E0E948565882371F41F
:10E2500081E090E00E9460631F5F163099F7B394ED
:10E260008AE5B81619F0C8E8D2E0B4CF0E94F15E92
:10E2700081E090E00E946063CDB7DEB7ECE00C94E3
:10E28000C277EF920F938091940F882309F0E5C035
:10E290008091AE0F882309F041C08091AA0F86FDBE
:10E2A0003DC08091BD0F882309F0D7C085E090E084
:10E2B0000E9460630E94DD6F82E061E00E942D6336
:10E2C0002091B00F2F5F2093B00F4091AF0F30E03F
:10E2D000842F90E00197281739077CF04150409334
:10E2E000B00F0E947B6D882311F00E94F86A81E0D4
:10E2F0008093940F82E08093B80F81E090E00E94B9
:10E30000606381E061E040E020E000E0EE240E94F4
:10E310008C6D82E060E00E941E639FC08091B40F0C
:10E32000882321F081508093B40F0BC087E0809345
:10E33000B40F90E08091BC0F882309F491E0909392
:10E34000BC0F9091A30F94FF82C08091B30F8823DC
:10E3500089F40E94CC66882369F49091A30F80E130
:10E3600098279093A30F95FF78C080E28927809328
:10E37000A30F73C09091B30F9F5F9093B30F8091E1
:10E38000AA0F87FF03C09F5F9093B30F8091B30FD5
:10E39000803108F462C01092B30F8091A30F90E116
:10E3A00089278093A30F80FF04C080919D0F815027
:10E3B00005C081FF06C080919D0F8F5F80939D0FE8
:10E3C00009C09091B90F82FF02C0915001C09F5FB8
:10E3D0009093B90F80919E0F90919F0F019690930B
:10E3E0009F0F80939E0F80919C0F8F3F61F18091D2
:10E3F000AB0F9091AC0F01969093AC0F8093AB0F45
:10E400000091B70FE090BA0F802F6E2D0E94F66535
:10E410008230A1F4802F6E2D44E00E94A666809188
:10E42000AA0F86FD05C088E26CE340E00E943E62D0
:10E430008091AE0F81508093AE0F05C0802F6E2D5E
:10E4400043E00E94A6668FEF80939C0F06C095FF65
:10E4500004C080E298279093A30F0F91EF90089546
:10E46000A0E0B0E0E6E3F2E70C94AB77982F80935E
:10E47000B00F81E08093BD0F20E030E007C02F5F38
:10E480003F4F849131968131D1F79150E901CA52C1
:10E49000D646992311F0FE01F2CF80E060E040E023
:10E4A00020E000E0EE24E3940E948C6D8091AA0F9E
:10E4B00080648093AA0F8E01F0E1DF2EF801949121
:10E4C0008091AE0F882379F1913169F1C0E0D0E0FD
:10E4D000E92EFF248091AE0F8823F1F0C7010C2EA6
:10E4E00002C0959587950A94E2F7837011F481E153
:10E4F00009C0813011F482E105C0823011F088E159
:10E5000001C084E18093A30F1092B30F0E94417168
:10E51000D092B30F0E9441712296C830D105D1F636
:10E520000F5F1F4FCBCF80919E0F90919F0F9093C5
:10E530009B0F80939A0F8091AB0F9091AC0F9093AB
:10E54000B60F8093B50F1092AA0F1092BD0FCDB7E2
:10E55000DEB7E7E00C94C7776F927F929F92AF92FD
:10E56000BF92CF92DF92EF92FF920F931F93CF93C0
:10E57000DF93182F81E08093BD0F80E064E10E945B
:10E58000636481E090E00E9460631093B00F20E02C
:10E5900030E007C02F5F3F4F849131968131D1F732
:10E5A0001150E901CA52D646112311F0FE01F2CFF3
:10E5B00081E061E040E020E000E0EE240E948C6D0C
:10E5C00081E061E00E941E630E940B688CE06BE1B9
:10E5D0004BE658EA28E100ECCC240E9421658CE34C
:10E5E00090E00E9460635E01DD2410E03EE1E32ED6
:10E5F000FF24F50194918091AE0F882381F1913130
:10E6000071F1C0E0D0E0692E77248091AE0F8823AD
:10E61000C1F0C3010C2E02C0959587950A94E2F7CC
:10E62000837019F421E1D22E0CC0813019F492E1EB
:10E63000D92E07C0823019F088E1D82E02C004E13B
:10E64000D02ED092A30FCF2C99240E94856E0E94C9
:10E6500085658823A1F081E090E00E9460630E94BC
:10E660008669DF91CF911F910F91FF90EF90DF901E
:10E67000CF90BF90AF909F907F906F9008950E9431
:10E6800041712091970F3091980F33FF0CC080910A
:10E69000950F9091960F93FD06C0112391F01130C4
:10E6A000A1F017E013C032FF13C08091950F909135
:10E6B000960F92FD0DC0113011F410E007C0133019
:10E6C00011F411E003C0173009F413E00E940B6845
:10E6D00000E003C00E9441710F5F0117D8F3109250
:10E6E000A00F0E940B68EE2099F4F3948CE06BE18C
:10E6F00044E658EA28E100EC0E942165F3E0FF15AA
:10E7000020F4BEE1EB2EFF2404C0AEE1EA2E01C0EE
:10E71000EA941F5F910E11508FE0891510F0CF2CF5
:10E7200094CF2296C830D10509F06FCF0894A11C70
:10E73000B11C5FCF8091990F823311F41092990F21
:10E740008091990F8F5F8093990F81500E94AC72D6
:10E750000895A0E0B0E0EFEAF3E70C94A9771092F7
:10E76000B10FC090AD0FB090A90FC0E8D3E005E0A5
:10E770000EC0812F602F0E94F665F70181937F0103
:10E780001F5F1A30B1F725960F5F0A3041F0FCEC9D
:10E79000EF2EF4E0FF2EEC0EFD1E15E0EACF80E038
:10E7A00064E10E9463648AE06AE048E028E000E0F7
:10E7B00010E0EE24E3940E946E6A81E090E00E94F3
:10E7C00060638BE06BE040E459EA0E94DA6A8BE018
:10E7D0006CE04AE359EA0E94DA6A8BE06DE043E3B9
:10E7E00059EA0E94DA6A8BE06EE04DE259EA0E9433
:10E7F000DA6A8BE06FE049E259EA0E94DA6A8BE05C
:10E8000060E145E259EA0E94DA6A8BE061E140E2A8
:10E8100059EA0E94DA6ADC2C0E94856E0E94AA6581
:10E82000882331F08091B10F882311F0815009C005
:10E830000E94BD65882341F08091B10F863020F49D
:10E840008F5F8093B10FB5C00E948565882309F45E
:10E85000B0C0C0E8D3E005E00EC0812F602FF70103
:10E8600041917F010E94A6661F5F1A30B1F725967D
:10E870000F5F0A3041F0ECECEE2EE4E0FE2EEC0EE1
:10E88000FD1E15E0EACF1092940F1092B80F109170
:10E89000B10F112329F4B092A90FC092AD0F34C16A
:10E8A000113019F40E94656E2FC1123041F40E949C
:10E8B000376981E08093940F1093B80F25C113300E
:10E8C00079F48091B00F0E94AC7280E064E10E9404
:10E8D000636481E08093940F82E08093B80F14C149
:10E8E000143009F043C00E94F15E82E090E00E9483
:10E8F000606351E050930E0150931E0F4091A90F99
:10E900004093200F80911D0F882369F0242F30E061
:10E910008091AD0F90E001962817390721F41092ED
:10E920001D0F10921E0F413019F486E59FE704C0B9
:10E93000423029F485EB93E80E94CA5EE5C043307B
:10E9400019F489E89DE8F8CF443019F488E098E894
:10E95000F3CF453019F48FE794E9EECF10920E0112
:10E9600081E080931D0F10921E0FCEC0153091F4E0
:10E9700011E010931F0F8091AD0FD81641F00E9447
:10E980000B688D2D0E94606810931F0FBDC0109200
:10E990001F0FBAC081E08093B80F8093940F0E943C
:10E9A000376980E064E10E94636481E80E949569B0
:10E9B000ABC08091B10F8430A1F41091A90F112345
:10E9C00041F00E94D065882311F0115007C0153026
:10E9D000C8F40E94E3658823A9F01F5F1093A90F74
:10E9E00011C0853079F4DD2049F00E94D06588237C
:10E9F00011F0DA9407C0F3E0FD1520F00E94E36502
:10EA00008111D3948091A90F81508E3F38F08FE00F
:10EA10006FE04CE159EA0E94DA6A36C080E16FE0AB
:10EA200042E850E00E940F5D8091B00F90E09C01A1
:10EA300074E0220F331F7A95E1F7F90163E0EE0FDE
:10EA4000FF1F6A95E1F7E21BF30BE80FF91FE65D84
:10EA5000F749E4912091A90F30E08E2F90E00196C4
:10EA60002817390729F481E16FE044E850E004C039
:10EA700081E16FE042E850E00E940F5D8FE06FE0BF
:10EA80004091A90F0E946A6C4D2D4F5F8FE060E1AD
:10EA90000E946A6C8091B00F90E09C0154E0220FBC
:10EAA000331F5A95E1F7F90143E0EE0FFF1F4A9536
:10EAB000E1F7E21BF30BE80FF91FE65DF749E4917C
:10EAC000ED1529F481E160E144E850E004C081E102
:10EAD00060E142E850E00E940F5D1BE08AE0612F98
:10EAE0004AE750E00E940F5D1F5F1231B9F7609155
:10EAF000B10F655F8AE04CE750E00E940F5D81E056
:10EB000090E00E94606388CECDB7DEB7E9E00C9458
:10EB1000C577A0E0B0E0EFE8F5E70C94A577109298
:10EB2000B10F1092AD0F10921F0F10921E0F80E0C8
:10EB300064E10E94636481E80E94956981E090E04D
:10EB40000E94606382E060E00E941E638091210F5A
:10EB5000882359F486E59FE70E94CA5E81E080938E
:10EB60000E018093A90F8093210F81E090E00E9415
:10EB7000606380E064E10E946364DD24D39454E028
:10EB8000F52E06E1C6E1D3E044E0742E3FE9832E82
:10EB90009924939464C0849189538D933196A617D8
:10EBA000B707C9F7425E5F4F225F3F4FBD01625E0C
:10EBB0007F4F84E32839380729F0DA01A05EBE4F81
:10EBC000F901E9CF1092A00F1092AD0F802F880F9E
:10EBD000880F880F10E020E2A22EA80EB72CBD18D7
:10EBE00090E1C92EC80E83E0E82EED0C113049F0FB
:10EBF000113028F0133039F0143071F408C080E47B
:10EC000007C080E601C080E86A2D4B2D03C080EA72
:10EC10006C2D4E2D0E94B9678091AD0F8F5F809350
:10EC2000AD0F1F5F153011F781E090E00E94606327
:10EC3000FE01E05EFE4FCE01865D9E4F8192E81799
:10EC4000F907E1F7FA9419F4D924B4E0FB2E81E036
:10EC500090E00E94606301506E97023049F0AE016F
:10EC60004A57504020E634E3BE016C547F4FA5CF95
:10EC700084E190E00E94606384E164E149E023E084
:10EC80000CEF1FEFEE240E946E6A85E165E14EE411
:10EC900059EA0E94DA6A85E166E145E459EA0E9490
:10ECA000DA6A88E290E00E946063C0E0D0E0CC24A1
:10ECB000C394A8E3EA2E0E94856E0E94AA65882369
:10ECC00021F40E94BD65882359F090E08091B10F36
:10ECD000882309F491E09093B10FC0E0D0E02CC0FC
:10ECE0000E948565882341F181E08093940F82E042
:10ECF0008093B80F1092B00F8091B10F813099F4CA
:10ED000003C09F5F9093B00F8091B00F0E94476D3A
:10ED10009091B00F8823A9F78091AF0F981718F042
:10ED200081508093B00F81E061E00E942D6380E00C
:10ED300064E10E94636465C084E165E14AE750E0F4
:10ED40000E940F5D84E166E14AE750E00E940F5D9A
:10ED50006091B10F6B5E84E14CE750E00E940F5D63
:10ED6000219681E0CD32D80784F081E061E00E94F5
:10ED70002D6380E064E10E9463641092940F0E940E
:10ED80009A7381E08093940F3CC081E090E00E94F0
:10ED900060631092A00FF39487E08F1510F4DC24C9
:10EDA000FF2410E00D2D0B5F123009F11093AD0F11
:10EDB000112329F421E030E090E140E00AC0143052
:10EDC000F1F440E120E030E0143011F421E030E0D3
:10EDD00090E0812F8295807F805B891B922F929596
:10EDE000907F6E2D691B840F402F0E94B9671F5FB3
:10EDF0001530D1F681E090E00E9460635CCF40E086
:10EE0000E1CFCDB7DEB7EDE00C94C1778091B80FBC
:10EE10008823B9F0823069F0833018F4813089F4A6
:10EE200005C0853049F0873061F409C00E948975BA
:10EE300008950E94956E08950E94DD6F08950E94C6
:10EE4000A97308950E94856E0E948565882331F01C
:10EE500081E08093940F87E08093B80F0E949865BB
:10EE6000882319F00E94656E08952091970F3091C4
:10EE7000980F33FF0FC08091950F9091960F93FDDF
:10EE800009C08091AA0F87FF02C0805801C0806826
:10EE90008093AA0F8091B30F882399F424FF02C0B6
:10EEA00081E107C025FF02C082E103C026FF04C044
:10EEB00084E18093A30F089527FF03C088E1809326
:10EEC000A30F08950E94DE6C0E9422770E940677AD
:10EED0000E9441710E940B68F7CF991B79E004C032
:10EEE000991F961708F0961B881F7A95C9F7809589
:10EEF0000895AA1BBB1B51E107C0AA1FBB1FA61781
:10EF0000B70710F0A61BB70B881F991F5A95A9F7D2
:10EF100080959095BC01CD01089597FB092E072699
:10EF20000AD077FD04D0E5DF06D000201AF47095F2
:10EF300061957F4F0895F6F7909581959F4F0895BD
:10EF40002F923F924F925F926F927F928F929F92F9
:10EF5000AF92BF92CF92DF92EF92FF920F931F93E7
:10EF6000CF93DF93CDB7DEB7CA1BDB0B0FB6F89498
:10EF7000DEBF0FBECDBF09942A88398848885F84D8
:10EF80006E847D848C849B84AA84B984C884DF8049
:10EF9000EE80FD800C811B81AA81B981CE0FD11D2D
:10EFA0000FB6F894DEBF0FBECDBFED010895F89403
:02EFB000FFCF91
:10EFB200010100408891D2E4ADB5B6BEBFFF0100A9
:00000001FF
